:020000040800F2
:1000000000A000204510000891100008DD480008FD
:1000100091100008911000089110000800000000E5
:100020000000000000000000000000009110000827
:10003000911000080000000091100008E15700082E
:10004000911000089110000891100008911000080C
:1000500091100008911000089110000891100008FC
:1000600091100008911000089110000891100008EC
:100070009110000891100008FD220008911000085E
:10008000911000083D23000891100008911000080D
:1000900091100008911000089110000891100008BC
:1000A000BD2A0008C92A0008D52A0008852A0008A8
:1000B000912A0008992A0008A52A00089110000832
:1000C000911000089110000891100008911000088C
:1000D00091100008012400080D2400089110000868
:1000E000911000089110000891100008911000086C
:1000F0009110000891100008B12A00089110000822
:100100000000000000000000000000009110000846
:10011000911000089110000891100008911000083B
:10012000911000089110000891100008911000082B
:10013000911000089110000800000000000000006D
:1001400091100008911000089110000800000000B4
:10015000000000000000000000000000000000009F
:10016000000000000000000091100008911000083D
:1001700091100008000000000000000000000000D6
:080180000000000091100008CE
:1001880010B5054C237833B9044810B10448AFF3CF
:1001980000800121217010BDD4050020000000005E
:1001A800702C010808B5064B1BB106480649AFF389
:1001B80000800648016811B1054A02B1904708BDA0
:1001C80000000000702C0108D8050020D40500208C
:1001D8000000000081F0004102E000BF83F000430E
:1001E80030B54FEA41044FEA430594EA050F08BFCA
:1001F80090EA020F1FBF54EA000C55EA020C7FEA8E
:10020800645C7FEA655C00F0E2804FEA5454D4EB0A
:100218005555B8BF6D420CDD2C4480EA020281EAD4
:10022800030382EA000083EA010180EA020281EA0C
:100238000303362D88BF30BD11F0004F4FEA01315E
:100248004FF4801C4CEA113102D0404261EB41016D
:1002580013F0004F4FEA03334CEA133302D05242F3
:1002680063EB430394EA050F00F0A780A4F10104AF
:10027800D5F1200E0DDB02FA0EFC22FA05F28018E9
:1002880041F1000103FA0EF2801843FA05F35941CF
:100298000EE0A5F120050EF1200E012A03FA0EFC4E
:1002A80028BF4CF0020C43FA05F3C01851EBE37178
:1002B80001F0004507D54FF0000EDCF1000C7EEB95
:1002C80000006EEB0101B1F5801F1BD3B1F5001FD3
:1002D8000CD349085FEA30004FEA3C0C04F10104F2
:1002E8004FEA445212F5800F80F09A80BCF1004F1B
:1002F80008BF5FEA500C50F1000041EB045141EA9D
:10030800050130BD5FEA4C0C404141EB010111F49D
:10031800801FA4F10104E9D191F0000F04BF014648
:100328000020B1FA81F308BF2033A3F10B03B3F126
:1003380020020CDA0C3208DD02F1140CC2F10C02B6
:1003480001FA0CF021FA02F10CE002F11402D8BF14
:10035800C2F1200C01FA02F120FA0CFCDCBF41EAE0
:100368000C019040E41AA2BF01EB0451294330BDAF
:100378006FEA04041F3C1CDA0C340EDC04F114048C
:10038800C4F1200220FA04F001FA02F340EA030063
:1003980021FA04F345EA030130BDC4F10C04C4F1A9
:1003A800200220FA02F001FA04F340EA0300294689
:1003B80030BD21FA04F0294630BD94F0000F83F4D3
:1003C800801306BF81F480110134013D4EE77FEAB6
:1003D800645C18BF7FEA655C29D094EA050F08BF02
:1003E80090EA020F05D054EA000C04BF19461046E3
:1003F80030BD91EA030F1EBF0021002030BD5FEA27
:10040800545C05D14000494128BF41F0004130BD4E
:1004180014F580043CBF01F5801130BD01F00045A2
:1004280045F0FE4141F470014FF0000030BD7FEA15
:10043800645C1ABF194610467FEA655C1CBF0B4610
:10044800024650EA013406BF52EA033591EA030F27
:1004580041F4002130BD00BF90F0000F04BF00211F
:10046800704730B54FF4806404F132044FF0000552
:100478004FF0000150E700BF90F0000F04BF0021CB
:10048800704730B54FF4806404F1320410F0004531
:1004980048BF40424FF000013EE700BF42004FEA2C
:1004A800E2014FEA31014FEA02701FBF12F07F43A9
:1004B80093F07F4F81F06051704792F0000F14BFA6
:1004C80093F07F4F704730B54FF4607401F00045EA
:1004D80021F0004120E700BF50EA010208BF704741
:1004E80030B54FF000050AE050EA010208BF704736
:1004F80030B511F0004502D5404261EB41014FF49F
:10050800806404F132045FEA915C3FF4DCAE4FF0A2
:1005180003025FEADC0C18BF03325FEADC0C18BF89
:10052800033202EBDC02C2F1200300FA03FC20FADA
:1005380002F001FA03FE40EA0E0021FA02F1144427
:10054800C1E600BF70B54FF0FF0C4CF4E06C1CEA3C
:1005580011541DBF1CEA135594EA0C0F95EA0C0FB1
:1005680000F0DEF82C4481EA030621EA4C5123EA24
:100578004C5350EA013518BF52EA033541F4801153
:1005880043F4801338D0A0FB02CE4FF00005E1FB06
:1005980002E506F00042E0FB03E54FF00006E1FB50
:1005A80003569CF0000F18BF4EF0010EA4F1FF0493
:1005B800B6F5007F64F5407404D25FEA4E0E6D41D3
:1005C80046EB060642EAC62141EA55514FEAC520E4
:1005D80040EA5E504FEACE2EB4F1FD0C88BFBCF560
:1005E800E06F1ED8BEF1004F08BF5FEA500E50F111
:1005F800000041EB045170BD06F0004646EA0101D7
:1006080040EA020081EA0301B4EB5C04C2BFD4EB08
:100618000C0541EA045170BD41F480114FF0000E01
:10062800013C00F3AB8014F1360FDEBF002001F06F
:10063800004170BDC4F10004203C35DA0C341BDCE9
:1006480004F11404C4F1200500FA05F320FA04F0BB
:1006580001FA05F240EA020001F0004221F00041EF
:1006680010EBD37021FA04F642EB06015EEA430E62
:1006780008BF20EAD37070BDC4F10C04C4F1200592
:1006880000FA04F320FA05F001FA04F240EA020045
:1006980001F0004110EBD37041F100015EEA430E16
:1006A80008BF20EAD37070BDC4F1200500FA05F236
:1006B8004EEA020E20FA04F301FA05F243EA0203B5
:1006C80021FA04F001F0004121FA04F220EA0200C4
:1006D80000EBD3705EEA430E08BF20EAD37070BD0A
:1006E80094F0000F0FD101F00046400041EB0101EA
:1006F80011F4801F08BF013CF7D041EA060195F0CC
:10070800000F18BF704703F00046520043EB030385
:1007180013F4801F08BF013DF7D043EA0603704772
:1007280094EA0C0F0CEA135518BF95EA0C0F0CD07D
:1007380050EA410618BF52EA4306D1D181EA0301C3
:1007480001F000414FF0000070BD50EA410606BFBD
:100758001046194652EA430619D094EA0C0F02D102
:1007680050EA013613D195EA0C0F05D152EA033647
:100778001CBF104619460AD181EA030101F0004165
:1007880041F0FE4141F470014FF0000070BD41F0AE
:10079800FE4141F4780170BD70B54FF0FF0C4CF488
:1007A800E06C1CEA11541DBF1CEA135594EA0C0FA7
:1007B80095EA0C0F00F0A7F8A4EB050481EA030EF4
:1007C80052EA03354FEA013100F088804FEA0333DB
:1007D8004FF0805545EA131343EA12634FEA0222A9
:1007E80045EA111545EA10654FEA00260EF000416A
:1007F8009D4208BF964244F1FD0404F5407402D2BC
:100808005B084FEA3202B61A65EB03055B084FEA4C
:1008180032024FF480104FF4002CB6EB020E75EB49
:10082800030E22BFB61A754640EA0C005B084FEA71
:100838003202B6EB020E75EB030E22BFB61A7546EE
:1008480040EA5C005B084FEA3202B6EB020E75EB39
:10085800030E22BFB61A754640EA9C005B084FEAB1
:100868003202B6EB020E75EB030E22BFB61A7546BE
:1008780040EADC0055EA060E18D04FEA051545EAAD
:1008880016754FEA06164FEAC30343EA52734FEA56
:10089800C2025FEA1C1CC0D111F4801F0BD141EACF
:1008A80000014FF000004FF0004CB6E711F4801F34
:1008B80004BF01430020B4F1FD0C88BFBCF5E06F14
:1008C8003FF6AFAEB5EB030C04BFB6EB020C5FEA24
:1008D800500C50F1000041EB045170BD0EF0004E79
:1008E8004EEA113114EB5C04C2BFD4EB0C0541EAAB
:1008F800045170BD41F480114FF0000E013C90E6A8
:1009080045EA060E8DE60CEA135594EA0C0F08BF6B
:1009180095EA0C0F3FF43BAF94EA0C0F0AD150EA6A
:1009280001347FF434AF95EA0C0F7FF425AF1046FD
:1009380019462CE795EA0C0F06D152EA03353FF425
:10094800FDAE1046194622E750EA410618BF52EAA2
:1009580043067FF4C5AE50EA41047FF40DAF52EA76
:1009680043057FF4EBAE12E74FEA4102B2F1E043F0
:1009780024BFB3F5001CDCF1FE5C0DD901F0004C7E
:100988004FEAC0024CEA5070B2F1004F40EB8300CE
:1009980008BF20F00100704711F0804F21D113F1FA
:1009A8003872BCBF01F00040704741F480114FEA33
:1009B8005252C2F11802C2F1200C10FA0CF320FABC
:1009C80002F018BF40F001004FEAC1234FEAD323D9
:1009D80003FA0CFC40EA0C0023FA02F34FEA430343
:1009E800CCE77FEA625307D150EA01331EBF4FF0CC
:1009F800FE4040F44000704701F0004040F0FE40E7
:100A080040F40000704700BF80F0004002E000BFE3
:100A180081F0004142001FBF5FEA410392EA030FE1
:100A28007FEA226C7FEA236C6AD04FEA1262D2EB2B
:100A38001363C1BFD218414048404140B8BF5B4230
:100A4800192B88BF704710F0004F40F4000020F0C9
:100A58007F4018BF404211F0004F41F4000121F0DF
:100A68007F4118BF494292EA030F3FD0A2F1010229
:100A780041FA03FC10EB0C00C3F1200301FA03F167
:100A880000F0004302D5494260EB4000B0F5000F8A
:100A980013D3B0F1807F06D340084FEA310102F149
:100AA8000102FE2A51D2B1F1004F40EBC25008BFFB
:100AB80020F0010040EA03007047490040EB0000C5
:100AC80010F4000FA2F10102EDD1B0FA80FCACF1F4
:100AD800080CB2EB0C0200FA0CF0AABF00EBC250F3
:100AE80052421843BCBFD0401843704792F0000FE1
:100AF80081F4000106BF80F400000132013BB5E734
:100B08004FEA41037FEA226C18BF7FEA236C21D0A9
:100B180092EA030F04D092F0000F08BF084670470E
:100B280090EA010F1CBF0020704712F07F4F04D1DC
:100B3800400028BF40F00040704712F100723CBFEF
:100B480000F50000704700F0004343F0FE4040F419
:100B5800000070477FEA226216BF08467FEA2363D7
:100B68000146420206BF5FEA412390EA010F40F4C2
:100B7800800070474FF0000304E000BF10F000430E
:100B880048BF40425FEA000C08BF704743F09643F5
:100B980001464FF000001CE050EA010208BF704710
:100BA8004FF000030AE000BF50EA010208BF704797
:100BB80011F0004302D5404261EB41015FEA010CAC
:100BC80002BF84460146002043F0B64308BFA3F1A4
:100BD8008053A3F50003BCFA8CF2083AA3EBC25386
:100BE80010DB01FA02FC634400FA02FCC2F12002A5
:100BF800BCF1004F20FA02F243EB020008BF20F0DC
:100C08000100704702F1200201FA02FCC2F1200241
:100C180050EA4C0021FA02F243EB020008BF20EA36
:100C2800DC7070474FF0FF0C1CEAD0521EBF1CEA64
:100C3800D15392EA0C0F93EA0C0F6FD01A4480EA52
:100C4800010C400218BF5FEA41211ED04FF000633B
:100C580043EA501043EA5111A0FB01310CF0004067
:100C6800B1F5000F3EBF490041EAD3715B0040EA8D
:100C7800010062F17F02FD2A1DD8B3F1004F40EB5D
:100C8800C25008BF20F00100704790F0000F0CF030
:100C9800004C08BF49024CEA502040EA51207F3AF4
:100CA800C2BFD2F1FF0340EAC250704740F40000CF
:100CB8004FF00003013A5DDC12F1190FDCBF00F0C0
:100CC80000407047C2F10002410021FA02F1C2F16E
:100CD800200200FA02FC5FEA310040F1000053EA0A
:100CE8004C0308BF20EADC70704792F0000F00F058
:100CF800004C02BF400010F4000F013AF9D040EA5E
:100D08000C0093F0000F01F0004C02BF490011F4F1
:100D1800000F013BF9D041EA0C018FE70CEAD153EF
:100D280092EA0C0F18BF93EA0C0F0AD030F0004C6F
:100D380018BF31F0004CD8D180EA010000F0004023
:100D4800704790F0000F17BF90F0004F084691F0E1
:100D5800000F91F0004F14D092EA0C0F01D142021B
:100D68000FD193EA0C0F03D14B0218BF084608D1E4
:100D780080EA010000F0004040F0FE4040F400002E
:100D8800704740F0FE4040F4400070474FF0FF0CC1
:100D98001CEAD0521EBF1CEAD15392EA0C0F93EA08
:100DA8000C0F69D0A2EB030280EA010C49024FEA5A
:100DB800402037D04FF0805343EA111143EA101313
:100DC8000CF000408B4238BF5B0042F17D024FF4CB
:100DD800000C8B4224BF5B1A40EA0C00B3EB510FA6
:100DE80024BFA3EB510340EA5C00B3EB910F24BF8F
:100DF800A3EB910340EA9C00B3EBD10F24BFA3EB14
:100E0800D10340EADC001B0118BF5FEA1C1CE0D1DB
:100E1800FD2A3FF650AF8B4240EBC25008BF20F08E
:100E2800010070470CF0004C4CEA50207F32C2BFE2
:100E3800D2F1FF0340EAC250704740F400004FF07F
:100E48000003013A37E792F0000F00F0004C02BFB0
:100E5800400010F4000F013AF9D040EA0C0093F07A
:100E6800000F01F0004C02BF490011F4000F013BD4
:100E7800F9D041EA0C0195E70CEAD15392EA0C0F3C
:100E880008D142027FF47DAF93EA0C0F7FF470AF74
:100E9800084676E793EA0C0F04D14B023FF44CAFB7
:100EA80008466EE730F0004C18BF31F0004CCAD14C
:100EB80030F000427FF45CAF31F000437FF43CAF88
:100EC8005FE700BF4FF0FF3C06E000BF4FF0010CAA
:100ED80002E000BF4FF0010C4DF804CD4FEA40028C
:100EE8004FEA41037FEA226C18BF7FEA236C11D0D6
:100EF80001B052EA530C18BF90EA010F58BFB2EB89
:100F0800030088BFC81738BF6FEAE17018BF40F008
:100F1800010070477FEA226C02D15FEA402C05D1BC
:100F28007FEA236CE4D15FEA412CE1D05DF8040B41
:100F3800704700BF844608466146FFE70FB5FFF7D4
:100F4800C9FF002848BF10F1000F0FBD4DF808ED8C
:100F5800FFF7F4FF0CBF012000205DF808FB00BF7D
:100F68004DF808EDFFF7EAFF34BF012000205DF8D7
:100F780008FB00BF4DF808EDFFF7E0FF94BF012024
:100F880000205DF808FB00BF4DF808EDFFF7D2FF21
:100F980094BF012000205DF808FB00BF4DF808ED64
:100FA800FFF7C8FF34BF012000205DF808FB00BF31
:100FB8004FEA4002B2F1FE4F0FD34FF09E03B3EB5E
:100FC80012620DD94FEA002343F0004310F0004F9E
:100FD80023FA02F018BF404270474FF000007047F4
:100FE80012F1610F01D1420205D110F0004008BF93
:100FF8006FF0004070474FF00000704742000ED27B
:10100800B2F1FE4F0BD34FF09E03B3EB126209D43B
:101018004FEA002343F0004323FA02F070474FF0F1
:101028000000704712F1610F01D1420202D14FF066
:10103800FF3070474FF00000704700BF002100F0FC
:1010480004B80C4B5B58435004310B480B4B421807
:101058009A42FFF4F6AF0A4A00F003B8002342F8B8
:10106800043B084B9A42FFF4F9AF0AF0D1FA03F0B7
:101078002BFC7047942C010800000020D4050020A8
:10108800D4050020F41F0020FFF7FEBF084B98424C
:1010980001D1084904E0084988420CBF07490849BA
:1010A8000A88501C83B20B80098888B2704700BF39
:1010B80000300140F205002000380040F40500200F
:1010C800F005002038B5054641F201041148022117
:1010D8000AF0A4FD20B9601E84B2002CF6D10EE0FF
:1010E8000C4829460AF091FD41F201040948012102
:1010F8000AF094FD40B9013CA4B2002CF6D1054891
:10110800FFF7C4FFC0B238BD0248BDE838400AF056
:1011180080BD00BF003001402DE9F041012188B0B9
:101128004FF480500AF0ACFC01214FF400300AF073
:101138009BFC05210A464FF090400AF052FA06211E
:1011480005224FF090400AF04CFA052207214FF093
:1011580090400AF046FA02200026E02303258DF885
:10116800080001A94FF0904001938DF809508DF8BF
:101178000A608DF80B600AF0E3F901214FF40010C2
:101188000AF072FC8DF80950394D3A4F8DF80A6013
:1011980008244FF00108284601A901948DF8088019
:1011A8008DF80B600AF0CCF9214628460AF015FAAA
:1011B80038460AF09DFC07204FF482714FF4E06234
:1011C8004FF40073ADF80E10ADF81C0003A93846B3
:1011D800ADF81020ADF81630ADF80C60ADF812601F
:1011E800ADF81460ADF81840ADF81A600AF0B2FC1A
:1011F80038464FF480510AF0FDFC384641460AF063
:10120800EDFC214628460AF0EAF92420FFF75AFFA8
:101218008020FFF757FF214628460AF0DEF96420B0
:1012280004F002FB214628460AF0D9F92020FFF7EE
:1012380049FFAF20FFF746FF214628460AF0CDF9BF
:10124800404604F0F1FA214628460AF0C8F923205E
:10125800FFF738FF5020FFF735FF284621460AF0F0
:10126800BCF9642004F0EBFA08B0BDE8F08100BFD7
:10127800001000480030014037B5082105461948DC
:101288000AF0ADF9E820FFF71DFF00240020FFF762
:1012980019FF0DF804000134062CF7D11148082174
:1012A8000AF09BF99DF800209DF8013043EA0220DE
:1012B80001B2082391FBF3F29DF802009DF8031098
:1012C8002A8041EA002210B290FBF3F19DF8052034
:1012D8009DF80400698042EA002108B290FBF3F30C
:1012E800AB803EBD00100048034B0449044A03602C
:1012F8004160C26001207047211100088112000876
:101308001944923113B506220446282132206B462F
:1013180000F058FAF0B19DF801209DF8003043EA3A
:10132800022001B2022391FBF3F29DF803009DF81D
:101338000210228041EA002210B290FBF3F19DF8DE
:1013480004209DF80500618042EA002108B290FB64
:10135800F3F3A3801CBD000008B5242180223220AD
:1013680000F0B6F9642004F06AFA202197223220AE
:1013780000F0AEF90A2004F062FA1022232132208C
:1013880000F0A6F9642004F05AFA024B4FF4805298
:101398001A8008BD0400002013B501220446272145
:1013A80032200DF1070300F00DFA20B10248034B7B
:1013B8006060236001201CBD0D1300086113000844
:1013C800044B054903EB4000427831F8123098B2DB
:1013D800704700BF2C1500202615002030B55C4D45
:1013E8005C4B2878062207211A7099700822811C04
:1013F800441C9BB01A7159715870DC70C31C564854
:101408002B70564C0BF0FCF80FA80BF091F92A78CA
:10141800534810940024012A8CBF802121460F9044
:1014280014914FF480604FF400514FF48073ADF87D
:101438004820169020221891474817920FA9159313
:101448001194139419940BF053F9012142480BF0AD
:101458007CF968460AF0B7F803200F238DF80400DA
:101468006946404800938DF807400AF069F8012161
:101478004FF0A0400AF050FC0A2004F0E0F94FF0C9
:10148800A04021460AF03DFC4FF0A0400AF034FC91
:101498004FF0A0400AF03DFC04460028F8D1214650
:1014A8004FF0A0400AF038FC02A80AF015FC4FF4EF
:1014B80000414FF44032022304914FF0A04002A9AA
:1014C8000392059302948DF818400AF0D7FB07A8F9
:1014D8000AF0C8FB1E4A0894117809944FF400508A
:1014E80007908DF838104FF0A04007A90A940B9484
:1014F8000C940D940AF098FB154B1878A0420BD960
:10150800144A12F814100134E4B24FF0A0402246F5
:1015180006230AF00EFCEFE74FF0A04001210AF085
:10152800E2FB4FF0A04001210AF081FC0028F8D02E
:1015380002214FF0A0400AF072FC4FF0A0400121B8
:101548000AF064FC4FF0A0400AF05BFC1BB030BD11
:10155800F60500202C150020080002402615002062
:101568004000005000080048024B1A88501C81B205
:1015780019807047F805002070B5494B98428AB029
:10158800054637D14FF4802001210AF06DFA4FF457
:10159800001001210AF080FA01214FF480200AF09E
:1015A80063FA10200AF046FA3E48062104220AF09F
:1015B80018F8042207213B480AF013F801A80AF09A
:1015C80002F803A80AF0E8FF0224032640218DF858
:1015D80008408DF80960019132480126002401A9CC
:1015E8008DF80A608DF80B4009F0AAFF802201925D
:1015F8002C483CE02C4885424FD14FF480200121F3
:101608000AF032FA4FF4800001210AF045FA01216C
:101618004FF484000AF028FA24480AF00BFA244808
:101628000621042209F0DDFF0A2104224FF0904030
:1016380009F0D7FF01A809F0C6FF03A80AF0ACFF1C
:1016480002218DF808100322402319488DF809203B
:101658000126002401A98DF80A608DF80B4001933A
:1016680009F06EFF4FF4806001904FF0904001A99F
:1016780009F066FF03A80AF08FFF0E4B0694284670
:1016880003A90494059407940894099403930AF011
:1016980053FF284631460AF08AFF0AB070BD00BFE2
:1016A800005400400004004800580040200000108A
:1016B800001400487A25E0000148FFF75DBF00BF2D
:1016C80000540040014B188880B27047F80500208C
:1016D8003A4BF7B516464FF4204205460F461A60B6
:1016E8003748364C4FF400410AF081FF40B1236877
:1016F800581E2060002BF3D1FFF736FF00205BE077
:101708004FF40050009029462D4801224FF0807375
:101718000AF056FF4FF4204121602948274C022146
:101728000AF065FF28B921684A1E22600029F4D111
:10173800E2E7234839460AF055FF4FF42042226079
:101748001F481E4C80210AF052FF28B92368581EF2
:101758002060002BF4D1CFE70023009318482946D6
:1017680001224FF000730AF02BFF4FF42040206055
:101778001348124C02210AF03AFF28B921684A1E80
:1017880022600029F4D1B7E731460D480AF02AFF54
:101798004FF4204121600A4820210AF028FF30B97F
:1017A800064A1368581E1060002BF4D1A4E70448B9
:1017B80020210AF022FF0120FEBD00BFFC05002009
:1017C800005400402DE9F3411F463E4B14464FF4A8
:1017D800204280460D461A603B483A4E4FF400417D
:1017E8000AF005FF034640B133685A1E3260002BE9
:1017F800F2D1FFF7B9FE002061E04FF400500090ED
:101808004146314801220AF0DBFE4FF420413160A5
:101818002D482C4E02210AF0EAFE28B93168481EEC
:1018280030600029F4D1E4E7012C88BF45F0800539
:10183800254829460AF0D6FE4FF420423260224855
:1018480040210AF0D4FE30B91E480268531E0360D6
:10185800002AF4D1CDE74FF4105300931A484146BB
:1018680022464FF000730AF0ABFE16484FF42041B1
:101878000160CCB1144804210AF0B9FE30B9114A0C
:101888001368591E1160002BF4D1B2E70E480AF014
:10189800ABFE013C07F8010BE4B2E6E7094A13681E
:1018A800581E1060002BA4D0074820210AF09FFE84
:1018B8000028F3D0044820210AF09FFE0120BDE84B
:1018C800FC8100BFFC05002000540040F8B5134B14
:1018D8009B8905460E461446ECB116B116F8017BF5
:1018E80000E0FF270D4802210AF098F90028F9D0F6
:1018F8000A4839460AF08BF9084801210AF08EF99E
:101908000028F9D005480AF086F9C0B20DB105F8EB
:10191800010B013CE0E70120F8BD00BF00380040A2
:101928002DE9F047012188B04FF480400AF0B4F85F
:10193800364C374F01214FF480400AF0C5F8032098
:101948004FF420434FF0020A8DF803006946204601
:10195800ADF800308DF802A000F05CF84FF480413B
:101968000025ADF80010204669464FF480564FF028
:1019780001098DF8025000F04DF869462046ADF88F
:1019880000608DF8029000F045F838460AF0B0F88B
:1019980007214FF482724FF400704FF4E063ADF802
:1019A8000E20ADF816001022ADF81C10384603A919
:1019B800ADF81030ADF81820ADF80C50ADF81A504D
:1019C800ADF812A0ADF814900AF0C4F838464946AC
:1019D8000AF004F99F238DF804308DF805508DF82E
:1019E80006508DF8075001A90422268502A8FFF7A2
:1019F8006DFFA6619DF80900B0F1EF014A42A846C3
:101A080052EB010008B0BDE8F08700BF00040048B1
:101A18000038004073B506460D4600240123298886
:101A280003FA04F20A421AD0A878E978009200F082
:101A380003028DF804208A1ED1B299429CBF0A4B3A
:101A48005B5C800800F00C028DF8053030460023FE
:101A580069468DF806308DF8072009F071FD0134CC
:101A6800102CDBD17CBD00BFB80301082DE9F84379
:101A7800044643796278002B14BF0220002002B18B
:101A880001303849002551F82090A8462F462E46A7
:101A980019F80620FF2A02F00F0002F0F0035FD0C9
:101AA800A17821B1A0F1080CBCF1030F55D902F0BF
:101AB8002002D2B21AB12278002A08BF002303F00C
:101AC8001002D2B21AB16278002A08BF0023E27865
:101AD8004AB162793AB909B1011F01E0A0F10801E0
:101AE800012998BF802322792AB1617919B9021F87
:101AF800032A98BF802303F01001CAB212B100F084
:101B0800C9F92AE003F02001CAB222B1F9B200F003
:101B18008BF9013721E003F04001CAB282B1228972
:101B2800114B4FEA0010B2F5FA7F1844E9B2A389C5
:101B380002D900F0DFF801E000F0F2F801350CE01E
:101B48001B060AD5084B628903EB00105FFA88F17F
:101B5800E38900F0FBF808F1010801360E2E97D151
:101B6800BDE8F883D403010834040108064B53F890
:101B7800200083880268A1F57A714B434FF47A708C
:101B880093FBF0F11160704704060020024B53F8F4
:101B98002000026811607047040600202DE9F04F0C
:101BA80004464648464F057889B08E46691C017040
:101BB8009246114620680193724600F0AFFEA26873
:101BC8006068ADF808204FF0020802A90C268DF8CD
:101BD8000A808DF80B80FFF71DFF03A86E4394F869
:101BE8000CB025680AF086FA7023019A0393012045
:101BF80000214FF4807307EB0609ADF81000ADF82B
:101C080012100592ADF81880ADF81C30BBF10C0F1E
:101C18002BD8DFE80BF0072A2A2A102A2A2A192AA1
:101C28002A2A2200284603A90AF094F928460821FE
:101C38000AF06AFA19E0284603A90AF0C9F9284601
:101C480008210AF067FA10E0284603A90AF0F6F915
:101C5800284608210AF065FA07E0284603A90AF091
:101C680021FA284608210AF062FAA07B18B12068F8
:101C780001210AF0F2FA012120680AF05EF9217BBD
:101C88000C2914D8DFE801F0071313130A131313F0
:101C98000D13131310002268343207E0226838321B
:101CA80004E022683C3201E022684032BA51A9F8C7
:101CB80004A0484609B0BDE8F08F00BF0006002028
:101CC8005406002008B5044B53F820301BB10B28EC
:101CD80001D89A68904708BD04060020044B53F8C1
:101CE80020201AB107289CBF12681160704700BFF6
:101CF8003406002010B50C460649B1FBF2F292B248
:101D08000821FFF74BFF044B044943F82400816086
:101D180010BD00BF00127A0004060020751B0008E1
:101D280010B50C460649B1FBF2F292B20121FFF759
:101D380035FF044B044943F82400816010BD00BFFF
:101D480040420F0004060020951B000810B50C4601
:101D5800054991FBF2F292B20121FFF71FFF034BF5
:101D680043F8240010BD00BF40420F003406002095
:101D78000A4A0B4813681160C91A40F68C2291422E
:101D88000360084B01DD002006E01A780B2A9CBF8F
:101D9800054820F81210501C18707047880700205A
:101DA800E4060020A40700208C0700207FB5044625
:101DB80001A80D4616460AF0C1F9002003210123A7
:101DC800ADF80A00ADF80C10204601A9ADF8045092
:101DD800ADF80660ADF808300AF0E5F97FBD0000FF
:101DE80010B50F4B142202FB00308278036932B918
:101DF8004160012181701868197B02220BE0446858
:101E08008160084A091B4478C16022F81410002236
:101E180082701868197BBDE81040FFF7C7BF00BF84
:101E2800E80600208C0700202DE9F341164F0D46E7
:101E38004FEA0018142208EB07046A431349606844
:101E480001268B188E54E17BA2685D701C618DF8A9
:101E58000610022301A98DF80730ADF80420FFF71A
:101E6800D9FD58F80700217B0022FFF79FFF204685
:101E780032464FF6FF7100F071FD20462946044AAC
:101E880000F02EFDBDE8FC8134040108E8060020BE
:101E9800E91D0008F7B5124E124B0701BC190025C1
:101EA800A168E27B1D701C616068ADF80410022314
:101EB80001A98DF807308DF80620FFF7ABFDB8595A
:101EC800217B2A46FFF772FF204601224FF6FF7159
:101ED80000F044FD20462946034A00F001FDFEBDFE
:101EE80034040108E8060020791D0008014B33F886
:101EF800100070478C070020036B13B15A68006C00
:101F080001E0026AC069101A18BF01207047436BCC
:101F180013B190F844007047826A406A111A4B4224
:101F280053EB01007047026B034610B5406942B19C
:101F38001A6CD9688C1A013A18BF1146005D1964E9
:101F480010BD196ADA68405C0131B1FBF2F402FB9A
:101F58001411196210BD0000F0B51D465A4B984285
:101F680093B00F46164604D11046294600F004F9EE
:101F780007E05649884240F0A3801046294600F001
:101F880061F9044605F0040200206571A660A0719D
:101F980001962062E061A0626062E762029002F04E
:101FA800FF062AB14FF4005703974FF4806600E00C
:101FB80003960023049615F00106069301D10596B1
:101FC80001E00421059105F0020505F0FF071DB1A8
:101FD800059840F00802059201A9206D0AF092F9CF
:101FE80007A80AF0A5FBE36C00254FF48051802078
:101FF8000793109111950B950D950C900E9536B38E
:10200800206BD8B16369E668089320220F92ADF877
:10201800286009950AF0F4FA206B07A90AF068FB12
:10202800206B01210AF091FB206D402101220AF06A
:10203800D6F9206B0AF096FB206408E0206D24494D
:102048000AF0ECF9206D224901220AF0D0F907A81C
:102058000AF06EFB4FF48055A16C10958026002580
:10206800079111950B950D950C960E951FB3606B06
:10207800E0B122690F9510230993ADF828200AF0E2
:10208800BFFA606B07A90AF033FB0122606B0221DB
:102098000AF06BFB606B29460AF062FB606B314605
:1020A80045600122206D0AF09AF904E0206D094983
:1020B80001220AF09CF9206D01210AF083F900E061
:1020C8000024204613B0F0BD003801400044004011
:1020D800050105000701070007B502460B465171C7
:1020E80081790091D16A006D9268FFF735FF0EBDC6
:1020F80013B504460A46A160817943790091006DC1
:10210800E16AFFF729FF1CBD836A8169426BC91820
:10211800D160416A994203D9CB1A5360816204E0C5
:102128000169CB1A536000228262002180F84410B2
:10213800406B01210AF009BB10B5426A8469A154B9
:10214800416A02690131B1FBF2F402FB1411426BDE
:10215800416232B11368DA070AD4BDE81040FFF7CC
:10216800D3BF006D03490122BDE810400AF03FB912
:1021780010BD00BF0701070030B52C4B2C4A9860F2
:102188000D462C492C4899612C491A6058614FF426
:1021980080722B481965243185B0DA601A610A1DEE
:1021A80018639A64143801225863D96403200223FF
:1021B80000218DF80F20AA078DF80C308DF80D003E
:1021C8008DF80E100FD504AC4FF4007344F8083D99
:1021D8004FF090400921072209F003FA4FF0904090
:1021E800214609F0ADF9EB070FD504AC4FF4806038
:1021F80044F8080D0A214FF09040072209F0F1F940
:102208004FF09040214609F09BF901220E2101A8C8
:102218008DF804108DF805208DF806208DF807201C
:102228000AF03CF8014805B030BD00BF280A00207C
:1022380004040108A50700202509002000380140F2
:102248005800024030B5254B254A986080200D463D
:10225800D860402123481A6085B01961224A234971
:10226800986100205A6119650322022301218DF823
:102278000E00A8078DF80C308DF80D208DF80F1082
:102288000CD504AC202344F8083D19480521072241
:1022980009F0A7F91648214609F052F9E9070CD5C3
:1022A80004AC402244F8082D11480621072209F001
:1022B80098F90F48214609F043F9262001218DF8A5
:1022C800040001A88DF805108DF806108DF8071088
:1022D80009F0E4FF014805B030BD00BF7C0A0020CA
:1022E80004040108D00A0020A5080020004400408A
:1022F800000C004810B54FF400500C4C0AF03EFAA0
:1023080000210B480AF021FA0021606B0AF01DFA3F
:10231800626AA36A9A4204D02046BDE81040FFF7DB
:10232800F3BE012084F8440010BD00BF280A002035
:102338004400024010B54FF000700C4C0AF01EFA31
:1023480000210B480AF001FA0021606B0AF0FDF940
:10235800626AA36A9A4204D02046BDE81040FFF79B
:10236800D3BE012084F8440010BD00BF7C0A0020C1
:102378008000024038B5026B036D0446DD69A2B9DE
:10238800A80612D5E16A19B19A8C90B288470CE078
:102398009B8CE2696069D9B28154E069E368421CA8
:1023A800B2FBF3F103FB1120E061626BBAB92906B5
:1023B80015D5A36A616A8B420DD0A069C15C206DF6
:1023C8000AF009F8A26A2369501CB0FBF3F103FB79
:1023D8001102A26203E0206D05490AF008F82B07F4
:1023E80005D5206D0349BDE838400AF017B838BD57
:1023F80007010700000303000148FFF7BBBF00BF48
:10240800280A00200148FFF7B5BF00BF7C0A00205A
:1024180041717047426A806A131A594251EB0300AE
:1024280070477FB5044601A80D46164609F086FE9A
:1024380000200123ADF80A00ADF80C0001A92046E0
:10244800ADF80450ADF80660ADF8083009F0ABFE01
:102458007FBD437913F001010BD0026AC3699A4228
:1024680005D09CBFC0681218D01AC0B270470020AF
:10247800704708467047437913F0010110B50446C8
:102488000ED0FFF7E6FF60B1E3696269E168D05CEE
:102498004A1E934201D2013300E00023E36110BDDC
:1024A800084610BD43799A070AD5436A8269D15410
:1024B800416A03694A1CB2FBF3F103FB1122426231
:1024C80070478379012B03D1D1F1010138BF002175
:1024D800D0F83401426811B183689361704701896B
:1024E8001185704707B50346042299684068ADF81E
:1024F8000410022301A98DF806208DF80730FFF794
:1025080089FA0EBD2DE9F743914698464FF41272A9
:102518003B4B42430646D41808B93A4802E0012822
:1025280004D1394820631030C4F83401374D84F899
:1025380046620327D55067710023D4F8347184F8B4
:102548003C32012584F8393284F83852E1624FF47C
:102558008071E1602161B968236204F1340204F5F5
:102568009C70E361A3626362A4F84232A4F8443227
:102578006261A06102227868ADF80410C4F808907E
:1025880001A984F806808DF807208DF80650FFF71A
:1025980041FA206BFFF7A6FF20462946FFF791FF77
:1025A800322003F04CF91A4BD4F8347118680346FA
:1025B800B3FBF9F1B1F5803F03D3012BF8D95B08E0
:1025C800F6E7144DB0FBF5F289B23846D2B200F006
:1025D800C5F938463146104A00F082F9256BB8F142
:1025E800010F14BF022200222868297BFFF719FF78
:1025F80028463146094A00F073F92046BDE8FE83B3
:1026080034150020B4040108D40401081C0401088E
:102618006C01002040420F0051280008D92600080C
:1026280003460A4690F84602D96A9B79FFF76ABFC3
:10263800C268036A511E8B4201D3002300E00133B4
:102648000362704710B590F83C220446AAB9836A21
:10265800416A994225D080692169C05C01338B4267
:10266800A36228BFA26242000A2342F4007084F8E1
:102678003D32A4F83E02012311E090F93D3273B1D6
:10268800B0F83E124A08A0F83E2201F00101FFF717
:1026980018FF94F83D02431E84F83D3210BD84F8BB
:1026A8003C3210BD90F83B3210B583B990F83A32FD
:1026B80090F8392293420AD2B0F84042012101FA37
:1026C80003F121430133A0F84012DBB2F2E710BD59
:1026D8002C4B10B54FF4127404FB00346079C10719
:1026E8004FD594F8381219B3236B0021186809F0F4
:1026F80022FC94F83C1221B1B4F84202421CA4F81E
:102708004222236BA2791868197B012A0CBF022286
:102718000022FFF786FE0020012184F83B1284F88E
:10272800390284F83A02A4F8400284F8380210BD4D
:1027380094F83B22012A08BF94F83922204608BFA2
:1027480084F83A22FFF7AEFF94F83B02236B50B9A6
:102758000120A27984F83B021868197B012A0CBF72
:102768000222002209E0002184F83B12A2791868AD
:10277800197B012A14BF02220022BDE81040FFF78E
:1027880050BE10BD3415002090F83B1200230122E2
:10279800012980F8393280F838220BD180F83B3291
:1027A800036B8279197B1868012A14BF0222002260
:1027B800FFF737BE70474279D20708B503461BD5E5
:1027C800B0F8402202F4007189B209B9D10705D4E2
:1027D800B3F84402421CA3F8442208BDC16AC2F3FC
:1027E800470211B11046884708BD4169036ACA54B7
:1027F800BDE80840FFF71CBF08BD10B590F8383297
:102808000446002B1ED190F839124A1CD3B2092B6A
:1028180080F8393203D1BDE81040FFF743BF0A2BD7
:1028280010D190F83B0228B9B4F8401241F00102E7
:10283800A4F840222046FFF7BEFF2046BDE810401E
:10284800FFF7A2BF10BD0000064B10B54FF412747D
:1028580004FB00342046FFF7F5FE2046BDE8104093
:10286800FFF7CBBF3415002030B500240E4D55F8C6
:102878002450854202D00134E4B2F7E700200B4D22
:1028880035F810508D4202D0451CE8B2F7E707250D
:1028980005FB0040C0B21B2805D8054C04EB00100E
:1028A80083600171027330BD140501083005010809
:1028B800100B00200C2912D8DFE801F007111111C4
:1028C800091111110B1111110D00022104E004214D
:1028D80002E0082100E01021012209F0C7BC70477E
:1028E80038B504460D461346217B00682A46FFF793
:1028F800BBFF2068217BBDE83840FFF7DBBF07B589
:102908008DF80400012000238DF806008DF80700DB
:1029180001A88DF8053009F0C1FC0EBD7FB504464D
:1029280001A80D46164609F0FDFA0A480A4B016847
:102938005E43B1FBF6F20023013D561E204601A975
:102948000295ADF80460ADF80C30ADF8063009F02A
:10295800A3FA7FBD6C01002040420F0010B5044669
:102968000068FFF7DBFF2068012109F0E6FA607BC9
:10297800BDE81040FFF7C3BF00230C4A52F82320DC
:10298800824202D00133DBB2F7E70022084830F870
:102998001200884202D00132D2B2F7E7072101FBC8
:1029A80002330448DAB200EB02107047140501083C
:1029B80030050108100B002070B5044600262E4B88
:1029C8009D5D95B90221204609F059FC01284FD197
:1029D8002046022109F05DFC29462046FFF7CCFF7E
:1029E8000546204609F0B2FB3DE0042D12D12046F1
:1029F800294609F044FC01283AD12046294609F025
:102A080048FC29462046FFF7B7FF0546204609F04F
:102A18009FFB28E0082D12D12046294609F02FFCFB
:102A2800012825D12046294609F033FC29462046AD
:102A3800FFF7A2FF0546204609F08CFB13E00C2D9A
:102A480016D11021204609F01AFC012810D1204681
:102A5800102109F01EFC29462046FFF78DFF054688
:102A6800204609F079FBAA6801460AB1287B9047FD
:102A78000236082EA3D170BD300501080148FFF7C2
:102A88009BBF00BF002C01404FF08040FFF794BF70
:102A98000148FFF791BF00BF000400400148FFF75D
:102AA8008BBF00BF000800400148FFF785BF00BF8B
:102AB800003401400148FFF77FBF00BF00400140DC
:102AC8000148FFF779BF00BF004401400148FFF704
:102AD80073BF00BF00480140024800214FF4E07274
:102AE8000BF098BE100B00202E4B2DE9F341054644
:102AF8001878002838D0002426462746A0463221D8
:102B0800082253206B46FEF75DFE9DF801109DF8E4
:102B180000009DF8032000EB01239DF8021001340A
:102B280001EB022008FA83F89DF805209DF804308F
:102B3800E4B207FA80F79DF8070003EB0221202C86
:102B480006FA81F600F07F0201D0002AD7D1164B91
:102B580098FBF4F897FBF4F796FBF4F6A5F80080D9
:102B68006F80AE801C701AE0322106226B4653201B
:102B7800FEF728FE9DF801209DF800109DF803003F
:102B880001EB02239DF802202B8002EB00219DF827
:102B980004309DF80500698003EB0022AA80BDE897
:102BA800FC8100BFD00C0020D10C002008B5134BCD
:102BB8001B7853202D2108227BB1FEF789FD312196
:102BC8000A225320FEF784FD2C210C225320FEF705
:102BD8007FFD53203821902209E0FEF779FD31214D
:102BE8000A225320FEF774FD53202C210A22FEF7F7
:102BF8006FFD034840F20912028008BDD00C002086
:102C08000400002037B5104B05461A680F480C46DB
:102C1800002182428DF8071001D1002013E05320D3
:102C280001220DF10703FEF7CDFD0028F5D09DF830
:102C38000710E529F1D12A780548064B0649206096
:102C48001A70616001203EBD68010020001BB700BA
:102C5800B52B0008D00C0020F12A000813B5062275
:102C6800044602216B461820FEF7ACFD9DF80030A3
:102C78009DF8012098089DF8023000EB02219DF88C
:102C88000320218098089DF8043000EB02219DF86C
:102C980005206180980800EB0221A1801CBD00007E
:102CA80008B50F2108221820FEF712FD0E22182061
:102CB8001021FEF70DFD024B4FF480521A8008BD1B
:102CC8000400002037B502AB0024054603F8014D87
:102CD800182021460122FEF775FD50B19DF80730F6
:102CE800FB2B05D10348044928606960012000E0F6
:102CF80020463EBDA92C0008652C000813B5062205
:102D0800044601216B461C20FEF75CFD9DF800205F
:102D18009DF8013043EA022040F38D01042391FB22
:102D2800F3F29DF802009DF80310228041EA002288
:102D380042F38D0090FBF3F19DF805209DF8040007
:102D4800618042EA002141F38D0090FBF3F3A380F8
:102D58001CBD000037B52023022500244FF0904009
:102D680001A9ADF804308DF807508DF80640FEF73C
:102D780051FE2A2122461C20FEF7AAFC0E212A46D3
:102D88001C20FEF7A5FC0F2103221C20FEF7A0FC47
:102D98002B2112221C20FEF79BFC2C212A461C20EA
:102DA800FEF796FC2D2101221C20FEF791FC2E2116
:102DB80022461C20FEF78CFC05221C202A21FEF747
:102DC80087FC02484FF4807202803EBD0400002058
:102DD80013B5044610481149026800238A428DF849
:102DE800073001D1002015E01C200D2101220DF132
:102DF8000703FEF7E7FC0028F4D09DF807302A2BDC
:102E080001D01A2BEED10648064A074920606260B5
:102E18000B7001201CBD00BF68010020001BB7001B
:102E28005D2D0008052D0008D20C002013B50222E4
:102E380004461B2101AB6820FEF7C4FC9DF8042062
:102E48009DF8053043EA022000F54E5110314FF449
:102E58008C7291FBF2F3233323801CBD13B5062239
:102E680004461D216B466820FEF7ACFC9DF8002047
:102E78009DF8013043EA022001B2042391FBF3F2EA
:102E88009DF802009DF80310228041EA002210B24A
:102E980090FBF3F19DF805209DF80400618042EA5B
:102EA800002108B290FBF3F3A3801CBD08B51920DC
:102EB80002F0C5FC682015210022FEF709FC10B9B4
:102EC800032002F0BDFD0C4B1A781621682042F051
:102ED8001802FEF7FDFB172100226820FEF7F8FB19
:102EE8003D2101226820FEF7F3FB68203E210122E4
:102EF800BDE80840FEF7ECBB0000002038B50546E9
:102F080019200C4602F09BFC682015210022FEF7D0
:102F1800DFFB18B3124B13481349144A2B60622C79
:102F28006860A960EA60124B0FD004D80A2C12D04E
:102F3800142C0CD10DE0BC2C04D0B4F5807F06D144
:102F4800002009E00120187038BD022004E00320A9
:102F580002E0042000E005201870012038BD00BF01
:102F6800B52E0008652E0008352E00081844923149
:102F780000000020064B187820B1012806D14FF434
:102F8800805201E04FF4006202490A80704700BF96
:102F9800D30C00200400002007B5232002F04FFCCA
:102FA8006820752101220DF10703FEF70BFC30B1F3
:102FB8009DF80700B0F16803594251EB03000EBDBC
:102FC80013B50622044643216B466820FEF7FAFB38
:102FD8009DF800209DF8013043EA022001B2042345
:102FE80091FBF3F29DF802009DF80310228041EA5C
:102FF800002210B290FBF3F19DF805209DF8040023
:10300800618042EA002108B290FBF3F3A3801CBD63
:1030180013B5062204463B216B466820FEF7D2FB17
:103028009DF800209DF801309DF8021043EA022027
:103038009DF80320208042EA01239DF804009DF8B2
:103048000510638041EA0022A2801CBD07B5204A12
:1030580002204FF40053ADF804308DF807001368D0
:103068001C48002183428DF8061001D11A4803E05C
:103078001A498B4203D11A4801A9FEF7CBFC6B21F0
:1030880080226820FEF724FB052002F0D8FB1921D6
:1030980000226820FEF71CFB6B2103226820FEF744
:1030A80017FB372102226820FEF712FB0D4A1A216E
:1030B80068201278FEF70CFB1B2118226820FEF707
:1030C80007FB68201C211022FEF702FB0EBD00BF83
:1030D8006801002000127A0000040048001BB700B5
:1030E800000800480100002030B585B00446FFF70D
:1030F80053FF002841D006210A46682002ABFEF79C
:1031080061FB9DF80B309DF80D5003F0010105F0AF
:1031180001004A0042EA80059DF8090000F0010319
:103128001D4307D0012D164801D1002318E0022DB8
:103138000CD114E00C21682001220DF10703FEF7E1
:1031480041FB9DF8071011F00F0203D1052002F092
:1031580077FC06E0042A0A4801D1057001E0012342
:103168000370074807490378074A2160002B14BFFA
:103178006E216F2162602172012005B030BD00BF51
:10318800D30C00207D2F00081930000838B50546FB
:103198000C46FFF701FF28B3134B144814492B6062
:1031A800142C6860E960134B15D004D8052C16D090
:1031B8000A2C0ED111E0BC2C08D0B4F5807F03D0C6
:1031C800622C06D102220BE0002209E001201870CF
:1031D80038BD032204E0042202E0052200E00622B2
:1031E8001A70012038BD00BF55300008C92F0008EB
:1031F800194492310100002013B506220446A82183
:103208006B466820FEF7DEFA9DF800209DF8013035
:1032180043EA022001B2042391FBF3F29DF8020075
:103228009DF80310228041EA002210B290FBF3F1CE
:103238009DF805209DF80400618042EA002108B24B
:1032480090FBF3F3A3801CBD08B5642002F0F7FAE5
:1032580068202321F022FEF73BFA10B9032002F080
:10326800EFFB052002F0EBFA044B1A7868202021C6
:1032780042F00F02BDE80840FEF72ABAD40C00203D
:1032880037B5054619200C4602F0D9FA68200F21F7
:1032980001220DF10703FEF795FA9DF80730D32BAD
:1032A80016D10C480C490D4A28604E2C6960EA601A
:1032B8000B4B07D05D2C09D0362C01D0002002E042
:1032C800402000E080201870012002E0C020FAE7CA
:1032D80000203EBD5132000801320008DDE9A73167
:1032E800D40C002010B5FDF749FC0A49FDF79AFCFB
:1032F8000949FDF74BFD094B044618680078FDF7AE
:103308003DFC01462046FDF78DFCFDF777FE80B2B7
:1033180010BD00BF3333534000F07F45E80C002058
:1033280038B50D4C00202578FEF74AF805F007035C
:103338000A4A013522F81300002325701846D15A8D
:1033480002334018102B80B2F9D1C008FFF7CAFF2A
:10335800034A107038BD00BFD50C0020D60C0020E1
:10336800C4190020074B084A19781088884207D3E7
:10337800064B1A68907888428CBF0020012070475D
:1033880000207047C4190020C6190020E80C00204E
:1033980038B5114B2024186000250020FEF710F8DE
:1033A8002D180A2002F04BFA013CF6D1C5F34F1054
:1033B800FFF798FF08490A68517801236418A0426A
:1033C80002D30133062BF9D10448927804490370DB
:1033D80053430B8038BD00BFE80C002002000020DA
:1033E800C61900202DE9F04F0446008885B048B979
:1033F800B4F9023043B9B4F90420D2F1010138BF5D
:10340800002102E0002100E0014611F0010377D11C
:103418003D4D00B22B7000F0BFFD0646B4F9020026
:1034280000F0BAFD0546B4F9040000F0B5FD044605
:10343800304609F0ADF90746304609F01DFA8046D6
:10344800284609F0A5F90646284609F015FA054662
:10345800204609F09DF98246204609F00DFA3946C2
:1034680081465046FDF7DEFB394683464846FDF760
:10347800D9FB514601904046FDF7D4FB49460290DE
:103488004046FDF7CFFB314603905046FDF7CAFB97
:103498001E4C4946206006F10040FDF7C3FB294653
:1034A8006060A5600298FDF7BDFB01460198FDF735
:1034B800B1FA2946E0600398FDF7B4FB0146584687
:1034C800FDF7A6FA3146206108F10040FDF7AAFB96
:1034D800294660615846FDF7A5FB01460398FDF7AC
:1034E80097FA2946A0610198FDF79CFB01460298CE
:1034F800FDF790FA3946E0613046FDF793FB20620C
:1035080005B0BDE8F08F00BF03000020EC0C0020E0
:103518002DE9F8434D4B0C46016819608088013A43
:103528009880072A30D8DFE802F004080F14191E23
:103538002226188820805A8803E0598821801A8812
:10354800524262809A881EE01988484220805A8830
:10355800F6E75988484220801A88F2E719884842D5
:10356800208058880CE05A882280188808E019883A
:1035780021805A8803E05988484220801A8850429E
:1035880060809B885A42A280314B1A78002A5AD10F
:10359800B4F900002F4DFDF7F1FA8046B4F90200A6
:1035A800FDF7ECFA0746B4F90400FDF7E7FA2968D5
:1035B80006464046FDF736FBE96881463846FDF782
:1035C80031FB01464846FDF725FAA9698146304690
:1035D800FDF728FB01464846FDF71CFA09F00CF9EF
:1035E800696820804046FDF71DFB296981463846F9
:1035F800FDF718FB01464846FDF70CFAE9698146D4
:103608003046FDF70FFB01464846FDF703FA09F07F
:10361800F3F8A96860804046FDF704FB69698046B5
:103628003846FDF7FFFA01464046FDF7F3F9296AE7
:1036380007463046FDF7F6FA01463846FDF7EAF93F
:1036480009F0DAF8A080BDE8F88300BF100D00206B
:1036580003000020EC0C002070B5144D144C2B789E
:103668000646ABB102F0DAF82268B31898421CD3C8
:103678000020287002F09EF802F0D0F820600D4873
:10368800017809B14A1E02700B4B0120187070BDF9
:1036980002F0C4F821683231884206D3012028702C
:1036A80002F088F802F0BAF8206070BD170D00200B
:1036B800240D00201B0D0020190D002037B58DF8B2
:1036C800051022498DF807300B788DF8040002A800
:1036D8008DF80620C2180D4612F8044C443CE0B29E
:1036E8000A282CD81A49022B31F8104003D814B1F3
:1036F8002046FFF7B1FF2B78022B0BD9154D2D680B
:1037080002F08CF8021B954204D21049124B00209B
:103718000870187011480278012A014600D094B93F
:103728000A4B1878022801D8421C1A700020087029
:103738000B49087003B0BDE8304002F03BB83224B2
:10374800022BD5D9D7E703B030BD00BF1C0D002030
:1037580038050108240D00201B0D0020190D00203C
:10376800170D0020014B1860704700BF200D002086
:1037780070B53F4B5A7B04463E4802B101220270A5
:103788004FF4007000F074F9002828D03A4E3B4BF3
:10379800316858780D68003018BF01206A68904772
:1037A80048B13368364D18680121C26829709047BE
:1037B80008B102212970304D2B681868826890473B
:1037C80028B12E494B7813B92D4A02201070296868
:1037D8000B689869804710B1294900220A70202097
:1037E80004F04AFE60B12248264B827A0AB9C17AAF
:1037F80021B12248C27A0AB9012100E000211970DA
:103808001F4B1878022802D14C204E211DE00128B8
:1038180007D14D2153204C220B46BDE87040FFF7DD
:103828004DBF184A1178012903D1532001464E2271
:1038380006E0104B1878012804D1532001460246AF
:103848004D23EAE724B153204D210A464423E4E7F7
:103858000D4A117821B13220BDE87040FFF7FCBE57
:103868000A4B20461C70BDE8704001F0A3BF00BFA2
:10387800881F0020160D0020200D0020771F002033
:103888001A0D0020180D00201B0D0020170D002018
:10389800014B1870704700BF1B0D00200F4B1A78A2
:1038A800432A17D15888B0F56C7F13D11979BE29EE
:1038B80010D193F8AD230020EF2A0DD113F8011B86
:1038C800074A934280EA0100F8D1D0F1010038BFDD
:1038D8000020704700207047704700BF00FC0308B5
:1038E800B0FF0308C82314211E220380012381701E
:1038F800C270037164214FF496722823C18002813B
:103908004381704710B50446272005F0A9FE2070B2
:10391800102005F0A5FE6070002005F0A1FEA07043
:10392800002005F09DFE4FF4E133E0705220636003
:10393800A360E360207510BD7FB51B4D1B4C284666
:1039480004F0D0FD214628461F3D04F0E5FD2E4633
:1039580004F1240001F092FD04F1680005F018FA62
:1039680016F8C40B02F088FA304603F0C5FC681C50
:1039780003F080FD05F1B80000F012FE04F1280004
:1039880001F076FD04F14B0304F1380005F1C201A2
:1039980000930190029105F17800A11D224605F1DE
:1039A800C00302F0FBFE7FBD9B1D0020981A00207B
:1039B80008B5054B0549D02202FB003000F59E7082
:1039C8000AF086FE08BD00BFC81900207C1D002033
:1039D800254A432370B54FF46C701370BE21002341
:1039E800EF255080117182F8AD5382F8AE331E4630
:1039F8001D4A985C0133B3F56C7F86EA0006F7D15F
:103A080082F8AE6308F010FD04260025711E11F03F
:103A1800FF061BD0342008F01DFD00245CB1124ABB
:103A280004F1006505F57F30A15808F03FFD042832
:103A3800054607D0EAE70D4808F060FD042805466A
:103A4800EDD0E3E70434B4F56C7FE7D108F0FAFC75
:103A5800042D02D1FFF722FF20B90A20BDE87040EB
:103A680001F0EEBF70BD00BFC819002000FC0308BC
:103A7800034B996808420CBF00200120704700BF23
:103A8800C8190020024B9A6810439860704700BF1D
:103A9800C81900202DE9F04FAA4AAB4D10685168AB
:103AA800AA4C85B002AB03C34FF46C7200212846C0
:103AB8000AF0B0FED022002120460AF0ABFE4320D7
:103AC8000321287002206971FFF7DCFF2A232021D7
:103AD800A5F8EE304FF4FA702B2385F8F41040F275
:103AE8004C41FA22A5F8F60085F80531212001F5A8
:103AF8004873A5F8F22085F806016E2240F27E4050
:103B0800A5F816314FF47A7300274FF001094FF4E6
:103B1800167685F80421A5F8141140F2DC5200F558
:103B28002F71A5F8D00003F5CB70A5F81221A5F8E0
:103B3800F06085F8AC73A5F8FA70A5F8F870A5F8E8
:103B4800FC7085F8E27085F8E37085F8E470A5F8F4
:103B5800E670A5F8E870A5F8EA7085F8ED7085F8C4
:103B6800EC9085F8077185F8387185F83A7185F811
:103B7800397185F8107185F8187185F81A7185F80A
:103B88001B7185F81C91A5F8D210A5F8D6006C30E9
:103B9800A5F8D8004FF4C87040F2B451A5F8D43055
:103BA800A5F8DE00322305F590709B46A5F8DA10DB
:103BB800A5F8DC30A5F8E030019285F81E7185F88B
:103BC8001F71FFF79FFE1E211723552040F6AC52A8
:103BD800E17263752173A3750B211423AA81E07028
:103BE8002D2208206171A3710E21637450234FF0B8
:103BF800280862732074A2766420E171E3765A2162
:103C080078234FF00A0A22754122A37284F82020F3
:103C180021722077E177AF73277084F8018084F8E8
:103C28000280E77584F804B0A7732776E773677690
:103C380084F812A084F8098084F81E9084F8237010
:103C480084F8247084F82570019984F821B004F16F
:103C58002A00E18484F8227002F0FAF804203C4A31
:103C680084F82E003B493C48A263152384F834307D
:103C7800E163206405F584713848278584F82F802E
:103C880084F8308084F8449004F000FE4FF44873C0
:103C9800A4F87430C8224FF4966140F2D93040F647
:103CA80043033E4684F8707084F8717084F872801B
:103CB80084F8739084F8767084F8B8A084F8B920F2
:103CC800A4F8BA10A4F8BC00A4F8BE304FF47F7270
:103CD800A4F8782007F108036A464FF4FA61A1F5C1
:103CE800FA70A4F87A10995CA4F87C000137FF20D8
:103CF80084F87E1084F87F000834082FE6D1134832
:103D0800012480F8C04080F8C14080F8C240C43027
:103D1800FFF7E8FD00230C4A981810330021C02B48
:103D28000161F8D100240E4B0849E018D022D034A4
:103D38000AF0CEFCB4F51C7FF5D105B0BDE8F04F14
:103D4800FFF746BE98030108C81900207C1D002013
:103D58009A99193FF6287C3F3D0A773F4E0501089E
:103D6800041B002008B5FFF799FD18B9BDE8084005
:103D7800FFF790BE08BD0000024B9A6822EA0000D7
:103D880098607047C8190020314B9A6810B5140420
:103D980009D4D00707D4110705D4D20303D44FF4AC
:103DA8000040FFF76FFE2A48816811F4803F0446FF
:103DB80012D00B0702D50820FFF7DEFFA36818040E
:103DC80003D54FF40040FFF7D7FF214A9068C10799
:103DD80002D50120FFF7D0FF1D498B6813F0080FAB
:103DE8000C460BD01A0403D54FF40040FFF7C4FF6C
:103DF800A268D30702D50120FFF7BEFF14488168E7
:103E080048F2010348F201040B40A342044603D1DF
:103E18004FF40040FFF7B0FFA26848F2400010409E
:103E280048F24001884202D14020FFF7A5FF094827
:103E380004F0C6FB084805F005FD074805F09EFCA0
:103E480020B90548BDE81040FFF75CBD10BD00BFB4
:103E5800C8190020D01A0020E81A002010B5FFF772
:103E68001DFD10B90A2001F0EBFD0F4C0F4920464B
:103E78004FF46C720AF02CFC94F8AC33022B02D984
:103E8800002084F8AC0394F8AC130948D02202FB54
:103E9800014303F59E710AF01BFCFFF775FFBDE8AF
:103EA8001040FFF749BD00BFC819002000FC0308F7
:103EB8007C1D002008B5FFF7D1FF0F201421012237
:103EC800BDE8084007F014BB08B5054B93F8AC03F0
:103ED800FFF76EFDFFF77CFDBDE80840FFF7EABF7E
:103EE800C8190020014B9868704700BFC819002006
:103EF800884203DB8242B4BF114601460846704738
:103F08000023036170472DE9F04106690136012E4F
:103F180004460D46066105D1002361602160836077
:103F2800BDE8F081D0F8008008464146FCF770FDF6
:103F380007463046FCF722FE01463846FCF726FFC6
:103F480001464046FCF766FD064660603146284655
:103F5800FCF75EFD01463846FCF764FEA168FCF7F5
:103F680059FD2660E060A060BDE8F08110B5044608
:103F78000069012807DD0138FCF700FE0146E0680A
:103F8800FCF704FF10BD002010BD08B5FFF7EEFFD9
:103F9800BDE8084008F0FEBC08B5FCF76DFA04A3BC
:103FA800D3E90023FCF7CEFAFCF7DEFC08BD00BF1E
:103FB800399D52A246DF913F2DE9F041069C064605
:103FC8000F46002B0CBF4FF020084FF0300820465A
:103FD80010F8013B0BB9154603E0002AFBDD013A56
:103FE800F6E7002D04DD30464146B847013DF8E7C5
:103FF80014F8011B11B13046B847F9E7BDE8F08164
:10400800014B186801F0A2BB300D00202DE9F043E8
:1040180089B006460F4603921C46039A134613F8C6
:10402800011B0393002900F08A80252901D030461E
:1040380083E0002004905578911C302D039105D120
:104048009578033203924FF0010800E08046A5F10D
:104058003003D8B2092806D8284603A90A2204AB97
:1040680000F02AF905466C2D05D1039911F8015B7A
:104078000122039100E00022642D2FD010D8582D82
:104088003AD006D8002D5AD0252DC6D1304629461B
:1040980053E0632DC1D130462178251DB8474AE049
:1040A800752D0DD0782D27D0732DB6D1251D2468F8
:1040B800049A0094304639460023FFF77DFF3AE022
:1040C800251D20680A2122B1002205AB00F07EF8E8
:1040D80002E005AB00F0AAF82C4623E005AD04F198
:1040E80004092068294612B100F095F801E000F0B3
:1040F800C2F84C46009517E004F104092068102125
:1041080042B1B5F15804634253EB040205AB00F029
:104118005DF806E0B5F158035A425A4105AB00F084
:1041280085F84C4605A8009030463946049A43461F
:10413800FFF742FF71E72C466FE7B8476DE709B014
:10414800BDE8F0830FB407B5094904AB086809490D
:1041580053F8042B09680193FFF758FF064B1868BA
:1041680001F013FB0028F9D0BDE80E4004B07047F9
:104178002C0D0020280D0020300D0020034A044B90
:1041880004491A6000200860704700BF0940000811
:10419800280D00202C0D0020014B1860704700BF2F
:1041A800300D002070B50646B6FBF2F408461546F9
:1041B80014B12046FFF7F6FF05FB1464024B195DA6
:1041C80000F8011B70BD00BF57050108F0B50124B8
:1041D800B0FBF4F58D4201D34C43F9E70026C4B196
:1041E800B0FBF4F504FB1500B4FBF1F41EB9002D87
:1041F80001DC002CF4D1092DEFB204DD002A0CBF3C
:104208005725372500E03025ED1903F8015B013605
:10421800E5E71C70F0BD00280B4603DA2D2203F8F1
:10422800012B40420A210022FFF7D0BFF0B501243C
:10423800B0FBF4F58D4201D34C43F9E70026C4B135
:10424800B0FBF4F504FB1500B4FBF1F41EB9002D26
:1042580001DC002CF4D1092DEFB204DD002A0CBFDB
:104268005725372500E03025ED1903F8015B0136A5
:10427800E5E71C70F0BD00280B4603DA2D2203F891
:10428800012B40420A210022FFF7D0BFA0F13003E2
:10429800DAB2092A01D818467047A0F16101052948
:1042A80001D857387047A0F14103052B01D837389A
:1042B80070474FF0FF3070472DE9F8430D6804460A
:1042C8000F469046994600262046FFF7DFFF002854
:1042D80006DB404504DC08FB060615F8014BF3E74E
:1042E8003D602046C9F80060BDE8F883931E222B84
:1042F80088BF0A22031E10B50C4603DA2D2001F8E8
:10430800010B5842FFF74EFF00210170204610BDF7
:1043180030B587B005460C4603A800210C220AF0E8
:1043280079FA28460021FCF739FE20B128462949A8
:10433800FCF770FB03E028462649FCF769FB264991
:10434800FCF770FCFCF734FE054685EAE570A0EB47
:10435800E5700A226946FFF7C9FF002D01DB20231B
:1043680000E02D2368468DF80C300BF099F90128F0
:1043780007D130228DF80D208DF80E208DF80F20F2
:104388000CE0022805D130218DF80D108DF80E10A3
:1043980004E0032802D130208DF80D00694603A8F7
:1043A8000BF07CF803A80BF07BF9C51EEDB22A468A
:1043B80003A920460BF014FA002363552046074949
:1043C8000BF06CF803A9204649190BF067F8204652
:1043D80007B030BD6F12033A00007A44C80F0108D5
:1043E8002DE9F041027803460130202AFAD0092A43
:1043F800F8D02D2A02D10346414D04E02B2A08BFEC
:1044080003464FF07E551E460024334616F8010B2E
:10441800A0F13007F9B209290DD83A492046FCF72E
:1044280001FC04463846FCF7A9FB01462046FCF788
:10443800F1FA0446E9E72E2817D1324F334616F829
:10444800010B3038C2B2092A0FD8FCF797FB39465E
:10445800FCF79CFC01462046FCF7DCFA2949044697
:104468003846FCF7DFFB0746E8E71878652801D0EF
:10447800452839D15E782D2E02D19F1C012605E0F2
:104488002B2E01D05F1C00E09F1C00267B1E0027FE
:1044980013F8012F303AD1B2092903D80A2000FBBA
:1044A8000727F5E7B7F59A7F28BF4FF49A77B846FC
:1044B8004FF07E51B8F1070F07D908461249FCF7AB
:1044C800B1FBA8F108080146F4E707F0070737B180
:1044D80008460C49FCF7A6FB013F0146F7E72EB159
:1044E8002046FCF753FC04E04FF07E512046FCF7D1
:1044F80099FB01462846FCF795FBBDE8F08100BF13
:10450800000080BF0000204120BCBE4C014B0022AF
:104518009A807047380D0020034BB3F90400D0F19E
:10452800010038BF00207047380D0020064B074AAD
:104538001968B2F904000B7803EB83018842D4BFF1
:1045480000200120704700BF400D0020380D0020DA
:1045580010B50446FFF7EAFF002814BF20460020E4
:1045680000F0010010BD0000074B084A1968B2F9B5
:1045780004004B780A78D118052251438842D4BFE9
:1045880000200120704700BF400D0020380D00209A
:10459800024B9A88501C9880704700BF380D002045
:1045A800024B18600248002282807047400D0020AC
:1045B800380D0020034B04491860044800220160AC
:1045C800C2807047440D00207C050108380D00208A
:1045D80008B501F035FC024B00221A7008BD00BF77
:1045E800771F002010B5FFF7A1FF00281ED0104B41
:1045F8005C78201C18BF0120FFF7AAFF70B10D4896
:104608000D4B01680D484A8901681A805A809A80C2
:104618004A88DA800A4BD888411CD980FFF7A4FF62
:1046280000B91CB9BDE81040FFF7D2BF10BD00BFEC
:10463800771F0020440D0020CE1F0020400D0020D1
:10464800380D0020044B9A8811B2142901DD143A60
:1046580000E000229A807047380D002003280ED809
:104668000B4B1B689A888A4209D2DB888B4206D991
:10467800084901220B7802FA00F01843087005492E
:104688000A780F2A03D100200870FFF7DBBF7047B4
:10469800400D0020340D002030B5814C89B0FFF763
:1046A8006DFDFFF75FFBFFF7D9FBA07B003018BF5C
:1046B800012001F0CFF894F8073133B1012B01D074
:1046C800092B02D18DF80C3004E000218DF80C1074
:1046D80084F8071103A8FCF781FE0220FFF7C8F948
:1046E80010B17048FEF754FE6F48704DFEF77AFE21
:1046F800022003F0CBFE6A4AB5F92830B2F8EE1072
:1047080002F1E20092F8ED2000F08EFF10B90320CC
:1047180001F096F9664C4FF488404FF48853A06135
:104728000A252385624CA18A8AB282F48840A08235
:10473800A38A99B281F48852A282192001F07FF8E5
:10474800012001F037F8192001F079F8013D002027
:1047580001F030F815F0FF05E4D14FF488434FF429
:104768008850208523854E4C01F012FC04F110017D
:10477800607902F077F8FEF7AFF904F5907005F06C
:10478800D7F861790E2901D0082903D101228DF8C3
:10479800152001E08DF815504020FFF769F98DF8D4
:1047A80012004FF40040FFF763F98DF81000012064
:1047B800FFF75EF98DF8110002F07CFC8DF813000C
:1047C8003A4890F8C230C3F380048DF81440344C52
:1047D8004FF47A70B4F8DE10B4F8E020ADF81C009D
:1047E8004FF48040ADF81810ADF81A20FFF740F9E3
:1047F80018B1B4F8DA30ADF81C30BDF81810B1F5BE
:10480800FA7F02D90022ADF81C20B4F8120194F8FE
:104818000741ADF81E00012C04D0092C01D1072452
:1048280000E0002404A88DF81640FDF71FF9214880
:10483800214CFFF7BFFE2060FEF794FF1D4821685A
:1048480003F0F8FE4FF48070FFF712F958B11448DE
:104858001A4B90F81F1190F81E21009300F59070E4
:10486800C33302F057FE4FF40060FFF701F908B1B7
:1048780004F012FB00F0B8FF0949114B4A7918609F
:10488800052A03D14FF4C87000F0E0FC4FF47A70A9
:1048980000F0FAFD0B4B0120587309B030BD00BF82
:1048A800C8190020CC1A0020AE1A00207C1D002058
:1048B80000100048D01A0020501E00207D1D002046
:1048C800540D0020771F002008B5FFF7E5FE00F023
:1048D800E1F9FCE708B5034BB3F9D40002F0D8F8C6
:1048E800FEE700BFC819002008B500F0D3FD0B4B48
:1048F80050B19A7842B1597879B901225A70084B67
:1049080008491888088008BD587830B90220FF2166
:104918000122BDE8084006F0EBBD08BD771F002066
:104928009A1E0020601E00202DE9F04FB44BB54AB6
:10493800B3F90600D18C884285B00FDBB0F5FA6F69
:1049480092F8254007DA451A6C43A1F5FA6694FBFC
:10495800F6F4643403E0C4F1640400E06424AA4F6C
:10496800A84B97F9EC1093F82320B7F812C193F8E5
:10497800705093F8716093F8243001924F42BAB2A4
:104988000021029203930A469D4FCB5F0093CCEB24
:10499800030303F2F31E40F2E637BE4503D8002BAB
:1049A800B8BF5B4201E04FF4FA73022ADFF8648271
:1049B8002CD025B1AB42CCBFC5EB03030023642741
:1049C80093FBF7FEDFF874A26FF0630B3AF81E90C2
:1049D8000BFB0E3B0EF1010E3AF91EA00FFA89FEF1
:1049E800CEEB0A0E0EFB0BFE9EFBF7FEF14428F8F9
:1049F8000190DDF8048003FB08FE844B9EFBF3F373
:104A0800DB199BB2634393FBF7F712E026B1B3427D
:104A1800CCBFC6EB03030023029F5F43A8F80470D2
:104A2800039F002BB8BF5B427B43784F93FBF7F79C
:104A38006437744B02EB030E64239EF8019007FB66
:104A480009F898FBF3F9DFF8F88102F808909EF866
:104A58000B909EF815E007FB09F898FBF3F9DFF8CF
:104A6800E48107FB0EF702F80890DDF8008097FB59
:104A7800F3F3674FE045D35503DA664BCF5A7F42CD
:104A8800CF5201320231032A7FF47EAF5E4C4FF4DD
:104A9800FA62B4F81411FFF72BFAB4F814615D4CFC
:104AA800801B4FF47A75C6F5FA634543B5FBF3F5F9
:104AB800642195FBF1F358486FF0630630F8132032
:104AC80006FB0355013330F9130013B2C01A534BD8
:104AD800454395FBF1F1587A8A18E280002838D0CE
:104AE8004F4F504D3E882988721A10B2FFF754FA7A
:104AF800074607F04DFE0646384607F0BDFE054658
:104B0800B4F90200FCF73AF80746B4F90000FCF7DC
:104B180035F831468046FCF785F8294681463846FF
:104B2800FCF780F801464846FBF772FFFCF740FAAD
:104B3800314620803846FCF775F829460646404637
:104B4800FCF770F801463046FBF764FFFCF730FAD3
:104B580060800220FEF78CFF90B133480378591C1F
:104B6800CBB206220370B3FBF2F002FB103111F056
:104B7800FF0F05D1FEF7D4FBFEF7F4FB2B4B1870A3
:104B88002A4A1078003018BF0120FEF7F1FD00F026
:104B980063FB18B100F07EFC60B904E0022003F06A
:104BA8006BFC0028F6D0224B9A8A91B281F4885087
:104BB80098820EE0194B997819B11D4A4FF4885024
:104BC80010855B781BB11A484FF48851816104F055
:104BD8003DF9184B184A196810680B1A002B35DB79
:104BE8000E4B587B80BB9870114B988A80B280F42A
:104BF800885001F5F421988201F59073136025E03F
:104C0800CE1F00207C1D0020C81900200CFEFFFFCD
:104C1800931E00209E1F0020A61F0020771F002043
:104C28009A1E0020601E0020590D0020500D002003
:104C3800001000484C0D0020640D0020BE1F00200D
:104C4800961E0020901E00200121997004F080FE1D
:104C58000C4A107830B94FF40060FEF709FF08B12C
:104C680004F02EF9202003F007FC18B10649086863
:104C780003F0E6FB054B9A680AB10548904705B072
:104C8800BDE8F08F881400204C0D0020781E00200D
:104C9800541E002038B5954C03F016FD206803F02B
:104CA8003DFD002800F01182206803F0CFFD4FF48D
:104CB8008040FEF7DDFE20B18D4C25780DB901F05E
:104CC800BFF88C4A92F81801B0B18B4B8B4D411E3E
:104CD8004FF47A7233F911400021A4F57A70FFF786
:104CE80007F9FBF74BFF8649FCF750F88549FBF7B6
:104CF80099FFFCF783F928804FF40070FEF7B8FE9F
:104D080020B1814A106801684B699847794C0022A4
:104D1800B4F81451B4F8160113467749545E9B0849
:104D2800AC42C4BF63F07F03DBB28442B8BF43F038
:104D380040030232082AF0D1744D754A2878984207
:104D48002C4604D11578F92D03D8691C00E0002100
:104D580011704FF480402370FEF78AFE68B16548F1
:104D6800654BB0F81211B0F8DC20B3F906408D1A83
:104D7800AC4202DD8B189C420CDB4FF48040FEF7FE
:104D880077FED8B95C4C5B49B4F90600B1F8142138
:104D9800904213DA5F4D01F05FF801F065F8B5F85D
:104DA80046305BB1524C5C492078002800F01A82EA
:104DB8000A78002A00F01682FFF796FD544B1C78FB
:104DC800142C40F0C58054484478ECB1514BB3F8EA
:104DD80046502DB94D490C785F2C01D101F030F8BF
:104DE800444A92F81A01002800F0B280494BB3F8FF
:104DF8004650002D40F0AC8044490C787D2C40F0A2
:104E0800A78001F01DF8A3E0404D2978572911D15A
:104E18004FF47A7000F038FB4FF48070FEF728FEEC
:104E280008B102F0D5FA082003F026FBE0B93B4CA4
:104E3800208019E00420FEF71BFEA8B12A785A2A20
:104E480012D1374B187820B11C70364B01221A70DA
:104E58000AE0354C257885F00101217009B102205E
:104E680000E00320FEF714FD284805785D2D00F0CA
:104E7800C0815B2D00F0BF815E2D00F0BE8125480A
:104E8800B0F8465035B921490C786F2C02D1FFF79C
:104E98002BFD15E0174A1D4B92F81A0118B115B9E8
:104EA8001D787E2DF3D01978972904D14FF4C87056
:104EB80000F0CCF904E0A72902D1174A0124947321
:104EC80012480378BB2B03D11248818D8D1C04E056
:104ED800B72B04D10F48838D9D1E85852CE0BE2BF2
:104EE80024D10C4D6A8D941C25E000BF4C0D002088
:104EF800881F0020C8190020CE1F00205E1E002039
:104F080000007A4400C07F44501E0020580D002045
:104F1800690D00207C1D0020771F00209A1E0020AC
:104F2800680D00205C0D00205B0D0020BD2B0FD10B
:104F3800744D698D8C1E6C85734C94F8AC03FEF728
:104F480037FDFEF745FDFEF7B5FF704800220270F9
:104F58000420FEF78DFD00282CD06D4B1A788AB1FD
:104F68006C48457875B16C49674AB1F90640B2F8A2
:104F78001401844206DD694D2C781CB968491C70FF
:104F880032220A80654B587C50B1664B1D782DB98A
:104F9800654C227812B9624832210180012008E06C
:104FA800614D2C7834B15B4A517819B95F4B29703F
:104FB8000120187000235E4C1A4634F8020F40F2A4
:104FC800135501B2A942A0F21550CCBF0025012506
:104FD80005FA03F5B0F5C77F8CBF002001202A43EE
:104FE8005D1C00FA05F0024340F2A4608142D4BF80
:104FF80000210121981C01FA00F103330A430C2B0C
:1050080092B2DAD100233F49444C01EB4300B0F897
:1050180046100A420CBF0020012018550133152BF9
:10502800F1D1627822B1022003F026FA68B914E0BF
:105038004FF40070FEF71CFD78B13E4C21680868FB
:10504800836898470028EED107E0324CE17839B9F7
:1050580000F002FF0120E07002E02E4C0022E27016
:105068002E4B2C4C987830B121790022E27019B976
:1050780000F0F2FE01202071284B26491A780AB95F
:1050880001200870CA782C4B12B92249087918B146
:105098004FF48841996102E04FF488421A85202034
:1050A80003F0EAF908B103F06DF91C4B19481A7BB3
:1050B80002B10122144982724B79082B01D00E2BC0
:1050C80045D1144A0020507241E01C4B1A68042A4A
:1050D8003DD8DFE802F00305080B35000120186011
:1050E80019684A1C1A601868411C1960134B1A6821
:1050F800501C18604FF48070FEF7BAFC00B302F041
:105108003BFB24E07C1D0020C8190020690D00200D
:105118005B0D0020771F0020CE1F0020881F002075
:105128006A0D00205A0D0020680D00205C0D00203B
:10513800D41F0020501E002000100048480D0020F9
:10514800364B00214FF400501960FEF791FC00F037
:105158004BFB334B33499A890860334B1AB11968B2
:10516800411A002959DB84181C6001F015F9FFF772
:10517800DBFB00F039FB2D4B2A4A19681060441AF2
:1051880018602B482B4A90F87630148053B12A497E
:10519800CC780CB90A792AB12848294BC4881988CF
:1051A8000A19C280202003F067F940B12248C37968
:1051B8000BB9017A19B1047B0CB103F059F82148F5
:1051C800214A174B1468B3F8F62000F11E0100F1CC
:1051D8002903A04701F06EFC01F0EAFBBDE8384066
:1051E80001F042BC4D78002D3FF4E8AD00F028FEF8
:1051F800E4E5012102E0022100E00321CCB2084BE2
:10520800621E83F8AC23FEF7E3FBFEF727FE0220BD
:105218002821224606F06CF931E638BD480D0020F9
:10522800C81900204C0D0020600D0020540D0020EE
:105238007C1D00205E0D0020771F00209E1F00208F
:105248009C0E00207D1D002008000020014B1880C6
:10525800704700BF740D0020034B1888D0F101007F
:1052680038BF0020704700BF740D0020F8B51E4BF2
:105278000022196813461D4C2588B5F5C87F1C4DBA
:1052880001D10026EE501B4EEF5832F906C0184CDB
:105298006744EF500025043395538D5202320C2B8E
:1052A800E9D1124B1A88012A18D1236803F1C802E0
:1052B8004FF4C87392FBF3F20A806268C83292FB1B
:1052C800F3F24A80A268C83292FBF3F30A4A1288C2
:1052D8009B1A8B8000F0BCFDFEF7F6FD03480188A1
:1052E8004A1E0280F8BD00BF780D0020740D002012
:1052F800900D0020B41E002004000020F8B5354BA6
:105308000446188832280ED13349344D0A68344887
:10531800168857889388218862882E806F80AB8092
:105328000180428001E0002834D02B4D00222E68F5
:105338001346284F2B493888322801D10025CD50F3
:105348002948CD58175EED19CD500021043311526C
:10535800B15202320C2B0D46EBD11E4801880129AF
:1053680014D1224B224A1D7002201170FEF790FAC8
:105378001A4A1948118803685088928819805880F9
:105388009A80174B1988588821806080114B1A8899
:10539800511E198017480378DBB10F490B68114972
:1053A800002202700868322290FBF2F018804868E8
:1053B80090FBF2F0588089680F4891FBF2F201885F
:1053C800521A9A80204600F043FDBDE8F840FEF7E7
:1053D8007BBDF8BD6A0D0020780D00206E0D002001
:1053E8007C0D0020800D0020B41E00205A0D0020E6
:1053F800680D00205C0D002004000020064B028888
:105408001988891A198042885988891A5980808888
:1054180099880A1A9A807047B41E00200F4B10B55D
:10542800596804460E4888470D480E4A01461278C6
:10543800FEF76EF80C48038813B12046FFF716FFF5
:105448000420FEF715FB10B12046FFF757FF074968
:105458000868BDE81040FFF7D1BF00BF641E0020F8
:10546800B41E00206C0D0020740D0020780D002063
:10547800014B1860704700BF780D0020014B186081
:10548800704700BFA40D0020014B1880704700BF73
:10549800A80D0020034B1888D0F1010038BF002068
:1054A800704700BFA80D00202DE9F8433C4B3D484C
:1054B800596888473B483C4A01461278FEF728F865
:1054C8003A480388002B42D0394C256800242F78AD
:1054D8002646254635490A88B2F57A7F08D1354BE4
:1054E800354A00201421E85001FB0620FEF708FD8C
:1054F800DFF8B0802F4B38F90400E9580A18EA5051
:105508002D4B4FF0140909FB0639FBF737FB014611
:105518004846FEF7F8FC002024F80800DFF88C80E5
:105528002649B8F800206052012A2FD14846FEF7D4
:105538002CFD8146DFB13846FBF720FB0146484683
:10554800FBF72CFD98B14FF47A73A8F80030154B8F
:105558001A4A18881188401A1880518858889288E1
:10556800401A99885880881A9880BDE8F883114BAA
:10557800E858124B00F5FA714FF47A7291FBF2F089
:10558800E0520F210A20012205F0B2FF013604354E
:105598000234032E9ED105490A88501E0880D6E79A
:1055A800781E00209C1E0020F40D0020A80D00206D
:1055B800A40D0020E80D0020AC0D0020900E002066
:1055C80010B50D4B044600220C481A702146FDF711
:1055D800DDFD78B909482146FDF752FE50B9074864
:1055E8002146FDF78BFC28B904482146BDE8104048
:1055F800FBF77ABE012010BDF40D0020781E0020B4
:1056080003780BB1054A1370417809B1044B19703E
:10561800807808B1034A1070704700BFF40D00206D
:105628006C0D0020A00D00202DE9F3410646084628
:1056380014461D46FFF7C4FF002876D03C4A0023D5
:105648001370072C3BD8DFE804F0080818212A3328
:105658003A04022002F022FF31E04FF44870ADF81E
:10566800060034498DF8043001A8FDF7CBFA10B1D3
:10567800314B01211970012C21D02E48FDF734FD42
:1056880020B102222C489442027018D02948FDF714
:105698009FFB20B10321284B8C4219700FD025485D
:1056A800FDF710FB20B1042223489442027006D073
:1056B8002048FBF771FE10B11F4B052119701E4AD7
:1056C800107828B90CB10446B8E7022002F0E6FECB
:1056D8003046FFF795FF022002F0CEFE10B1154CC0
:1056E80021688847154B164C1A689047082002F025
:1056F800C3FEB8B1642795FBF7F63046FBF73EFAD0
:1057080007FB1651804608B2FBF738FA0D49FBF73C
:1057180089FA01464046FBF77DF90B49FBF782FA07
:10572800206001E0002020600120BDE8FC8100BF6E
:105738006C0D0020641E00208C0D0020781E0020B7
:10574800A00E00208988883C0000204108B5036825
:105758001A68904708BD38B505460C4614F8011B71
:1057680019B12846FFF7F2FFF8E738BD08B5036816
:105778005968884708BD08B503689968884708BD0F
:1057880008B50368DA68904708BD08B50368196961
:10579800884708BD08B503685A69904708BD0000E6
:1057A800034B4FF4085208B19A6170471A85704745
:1057B8000010004808B5024B1968884708BD00BFAB
:1057C800F80D0020024A034B00201A60FFF7F2BFD1
:1057D800A9570008F80D0020024B1A68501C1860E1
:1057E800704700BFFC0D002010B5094A094913682D
:1057F8008C6810688342F8D1074A106811684FF422
:105808007A725043001BB0FBF1F102FB031010BD8C
:10581800FC0D002010E000E0000E0020014B18688D
:10582800704700BFFC0D002038B50446FFF7DCFFC9
:105838000546FFF7D9FF401BA042FAD338BD10B583
:1058480004462CB14FF47A70FFF7EEFF013CF8E7FD
:1058580010BD000030B56B4D0FCD9DB002AC0FC42C
:1058680095E8030084E8030005F000FF4FF4D870C2
:1058780006F0D0F801216448644D06F00DF90121C5
:105888004FF4CD201CAC06F0FBF80121604806F06F
:10589800EBF806F025F941F6FF7024F86C0D0323A8
:1058A80021464FF090408DF80630FCF7B3F84FF6DC
:1058B800FF71ADF8041057482146FCF7ABF82146B4
:1058C8005548FCF7A7F821465448FCF7A3F82846A2
:1058D8002146FCF79FF8082106224FF0904005F07A
:1058E80080FE082101224B4805F07BFE0921012298
:1058F800484805F076FE06210422474805F071FE67
:1059080007210422444805F06CFE0422424808217D
:1059180005F067FE0C214148022205F062FE3F486F
:105928000D21022205F05DFE3C480E21022205F001
:1059380058FE3A480F21022205F053FE01210A467B
:105948004FF0904005F04DFE4FF0904002210122AB
:1059580005F047FE2F480021022205F042FE2D489F
:105968000121022205F03DFE02224FF09040042161
:1059780005F037FE0024FFF725FF4FF488524FF457
:1059880088432A852B8525462548264A0168914261
:1059980002AB05D118198179112901D1012282712F
:1059A80003EBC501185904310135FCF733F8083405
:1059B800032DE9D108A805F0ABFE1B48089B1B4A3C
:1059C800B3FBF0F11A48116001684FF47A73B1FB28
:1059D800F3F2501EB0F1807F09D2164B164A586078
:1059E800F02182F8231000200721986019601348DD
:1059F800FBF762FEFBF794FF6420FFF720FF1DB062
:105A080030BD00BFA0030108070042000010004895
:105A180001003E100004004800080048000C00483F
:105A280068010020001BB70040420F00000E002054
:105A38006C01002010E000E000ED00E0005800409C
:105A480010B5114B40F2DB144FF488424FF48851E3
:105A580060439A61841E19850B48838A9AB282F43E
:105A680088418182838A9AB282F488518182204651
:105A7800FFF7E5FE0120FFF79DFE1920FFF7DFFE87
:105A88000020FFF797FEE7E70010004810B1034A2F
:105A9800034B1A6003480449C8607047EFBEADDE87
:105AA800F04F00200400FA0500ED00E02DE9F04F6A
:105AB80089B0804607937C4B0592B3F90000B3F98F
:105AC80002200028B8BF4042002AB8BF5242002432
:105AD8008242B8BF024604922546A346274603944D
:105AE800029426467149CB7813B90A79002A3DD029
:105AF800022E3BD06E4B6C48DDF814C0295A585F13
:105B0800022211FB0200CCF100016246FEF7F0F917
:105B18006849DDF81C9035F901A039F9053098F885
:105B28000720DFF8AC91CAEB000000EB030A02FB88
:105B38000AF1642098F81B2091FBF0F06FF0040143
:105B4800514302EB8202FEF7D3F954F80930029070
:105B5800594942F210720AEB0300FEF7C9F998F8A6
:105B6800111044F809004843021303924F48C378C0
:105B78001BB1017909B9022E2FD14B4FDFF840A193
:105B88007F5F18F80630DFF84CB1BA0102EB071056
:105B980035F90A2090FBF3F154F80B30881AC01835
:105BA80046494FF47A52FEF7A3F935F90A104BF833
:105BB80004000029B8BF4942B1F5207F02DD002268
:105BC8004BF804205BF8040008EB06027D2390FBE9
:105BD800F3F1907A41434FEAA11B344B1979C1B1D3
:105BE800022E16D00498DDF808C0DDF81090DDF814
:105BF8000CA0C0F5FA72784302FB0C0309FB0BF00A
:105C08004FF4FA7102FB0A0293FBF1F392FBF1F2F3
:105C180008E0DA780AB1022E02D15A463B4601E082
:105C2800039A029B2649DFF8B0A0685A25490090DC
:105C3800705C25490690009835F901C068520FFA42
:105C480080F9CCEB0909DFF894C054F80A0054F83D
:105C58000C10091801EB090054F80C1044F80C90CA
:105C6800DFF87CC044F80A1016F80C104FF0200C2E
:105C780001FB00F090FBFCF1DDF800C00698521A19
:105C88001CFB00F06FF04F0190FBF1F01B180F495F
:105C9800D21801366A5204340235032E7FF422AF3B
:105CA80009B0BDE8F08F00BF9E1F0020771F0020BD
:105CB80096100020600E0020F0D8FFFF80C1FFFF83
:105CC800700E0020961E0020100E00208A1E002054
:105CD800240E0020040E0020180E00202C0E002098
:105CE800931E00202DE9F04F85B000250646894611
:105CF8009246039307462C46022CDFF8388109D1D7
:105D080099F80500B8F904B01B300BFB00FC4FEA0A
:105D18006C1E2CE03E4B38F9140033F9141052462F
:105D280001EB4000CAF10001FEF7E2F8394A039995
:105D380032F9143031F91420C01A374BD978801849
:105D480079B999F8042038F914801B791B3208FBBB
:105D580002F14FEA211E53B1727C50430EEB202E04
:105D680005E096F807B00BFB00FC4FEA2C1E2B4908
:105D7800DFF8C4C031F91430325DBCF80010C3EB51
:105D88000E08274B02FB08F001FB08F24FEAE01B64
:105D9800B97AD012EA5801FB0020E8502149029351
:105DA8004FF40012CDF804C0FEF7A2F8029BDDF80C
:105DB80004C01D4AE850BCF80030A95845F80280D4
:105DC8001B094FF6FF72B2FBF3F3C1EB080159430D
:105DD800DFF868C0154B55F80C2055F80380891179
:105DE8004244E9505218397D114B45F80C804A431A
:105DF8000BEB603000EB222223F81420013401372A
:105E08000435032C7FF478AF05B0BDE8F08F00BFF0
:105E180096100020600E0020771F0020700E0020D2
:105E2800040E00200000E0FF440E0020500E002069
:105E38008A1E00209E1F00205E0D0020380E0020C4
:105E4800024B5A780AB1002058707047771F00201B
:105E58000023038043807047024B00221A605A6077
:105E6800704700BF240E0020024B00221A605A60BF
:105E78009A607047040E00200128034B14BF034AA0
:105E8800034A1A60704700BF08000020B55A00088E
:105E9800ED5C0008000000002DE9F84F384E376827
:105EA8000446384606F074FC0546384606F0E4FC1D
:105EB80076688046304606F06BFC8346304606F02E
:105EC800DBFCD4F80490A768064629464846FAF74A
:105ED800A9FE414682463846FAF7A4FE01465046D6
:105EE800FAF796FD216882465846FAF79BFE414626
:105EF80004464846FAF796FE3146FAF793FE0146FD
:105F08002046FAF787FD314604463846FAF78AFEF6
:105F18002946FAF787FE01462046FAF77BFD014637
:105F2800504606F035FD1749FAF77CFEFAF7B6FA3F
:105F380011A3D3E90023FAF72FFC134B0446186882
:105F48000D46FAF7ABFA02460B4620462946FAF701
:105F580047F900220D4BFAF71FFCFAF705FD06F08A
:105F68004BFC81B20A0444BF00F5B47189B208B28F
:105F7800BDE8F88FAFF30080182D4454FB21094089
:105F8800680E00200000E144A00E0020000024401C
:105F980010B5194C2088FAF7F1FD1849FAF742FEB6
:105FA80006F02AFC164B18802088FAF7E7FD014610
:105FB8001448FAF7EBFE1449FAF7E8FE13490860AB
:105FC8001348B0F87400FAF7D9FD01461148FAF7FA
:105FD800DDFEFAF763FA06A3D3E90023FAF7B2FA6B
:105FE800FAF7C2FC0C4A106010BD00BFAFF3008086
:105FF8003B597E90A9E7814004000020C903683F0F
:10600800640E00200AE81C4100401C46B01E002017
:106018007C1D002000006144CC1E0020AFF30080EE
:106028002DE9F04104460068D4F80480A7680D46BD
:106038000146FAF7F7FD414606464046FAF7F2FDF3
:1060480001463046FAF7E6FC394606463846FAF77E
:10605800E9FD01463046FAF7DDFC06F09BFC00211D
:106068000646FAF773FF70B920683146FAF78EFED4
:10607800314628606068FAF789FE31466860A06892
:10608800FAF784FEA860BDE8F0812DE9F04F0C68AE
:106098008368D0F800A0D0F8048089B0064620466E
:1060A80003938B4606F074FB0746204606F0E4FB94
:1060B800DBF804408146204606F06AFB0546204688
:1060C80006F0DAFBDBF8082004461046019206F0D9
:1060D8005FFB8346019806F0CFFB3946029058468D
:1060E800FAF7A0FD394604900298FAF79BFD594645
:1060F80005904846FAF796FD029906904846FAF741
:1061080091FD294607905846FAF78CFD01465046FE
:10611800FAF788FD214683460698FAF783FD01467B
:106128000598FAF777FC01464046FAF77BFD0146E9
:106138005846FAF76FFC214683460498FAF772FD31
:1061480001460798FAF764FC01460398FAF76AFDD6
:1061580001465846FAF75EFC3060029905F10040A6
:10616800FAF760FD01465046FAF75CFD2146834682
:106178000798FAF757FD01460498FAF749FC0146D3
:106188004046FAF74FFD01465846FAF743FC2146C8
:1061980083460598FAF746FD01460698FAF73AFC51
:1061A80001460398FAF73EFD01465846FAF732FCD5
:1061B800214670605046FAF735FD2946044609F134
:1061C8000040FAF72FFD01464046FAF72BFD01463D
:1061D8002046FAF71FFC394604462846FAF722FDFE
:1061E80001460398FAF71EFD01462046FAF712FC0D
:1061F800B06009B0BDE8F08F80EAE073A3EBE0730C
:106208008B4206DB002801DD401A704702D0401897
:1062180070470020704700002DE9F041524B534C65
:106228001A685B6886B003F100430193504B02F192
:1062380000420646B3F900000092FAF79FFC00F10D
:106248000040FAF72BF946A3D3E90023FAF77AF9C5
:10625800FAF78AFB0290B4F90000FAF78FFC039072
:10626800B4F90200FAF78AFC0490B4F90400FAF7CA
:1062780085FC6946059003A8FFF707FF3D4B93F897
:106288004430012B16D13C48417869B93B4C22680F
:10629800402592FBF5F7D01BFAF770FC0599FAF741
:1062A800B9FBFAF785FE2060344B1868402190FB53
:1062B800F1F001E0324B1888FAF760FC01460598C6
:1062C800304DFAF7A5FB05903046FAF753FC2E49F6
:1062D8002C680746FAF79EFB01463846FAF756FD42
:1062E800214607460598FAF793FB01463846FAF720
:1062F80099FC01462046FAF78DFB244C28601D4D79
:10630800D4F800800746039806F076FA95F830101E
:10631800FFF772FF08EB000204982260D4F80480AB
:1063280006F06AFA95F83010FFF766FF08EB0003ED
:1063380038466360D4F8088006F05EFA95F82F10A6
:10634800FFF75AFF1249134B0A684044A0601868C7
:10635800B6180E60411C196006B0BDE8F08100BF98
:10636800399D52A246DF913F680E0020C41E0020CE
:106378009A1E00207C1D0020771F00205C0E002044
:10638800040000208C0E00203661823CA41E0020F0
:10639800880E0020980E00202DE9F04F87B0FFF7F7
:1063A80083F8022002F068F8002800F0AD81AE4CB6
:1063B800AE48FFF733F8FFF717FA2768C71B0546FB
:1063C8003846FAF7D7FBAA49C968FAF72BFC83467F
:1063D800A848256090F82E8000252C462E46A64A0F
:1063E800105FFAF7CBFB5946FAF71CFC03AB585180
:1063F800B8F1000F27D04046FAF7C0FB01464FF02E
:106408007E50FAF7C3FCDFF8B092824651464FF04F
:106418007E50FAF7FDFA55F80910FAF703FC974988
:106428000346085F0193FAF7A9FB5146FAF7FAFB0E
:1064380001460198FAF7EEFA49F80500FAF7B8FDAF
:106448008F4A105303E08D498D4A605AA0528C4BF5
:10645800E15A02340435062C11FB0166BFD1894A82
:106468001388642046435B43874803A996FBF3F6E9
:10647800FFF70BFE082001F0FFFF20B1834803A9B6
:10648800FFF703FE07E0824803A9FFF7FEFD8048F7
:106498000146FFF7C5FD493E7E49B4B23B2CB1F831
:1064A800F00007D97B4E0820B6F8F25001F0E4FF5F
:1064B80030BB4FE0FAF75EFB4FF07E518046FAF7AB
:1064C800A9FA01464FF07E50FAF760FC0024064610
:1064D8006D4D404655F81410FAF7A4FB81466848FC
:1064E800005FFAF74BFB01464846FAF793FA314644
:1064F800FAF798FB45F814000234062CE8D1D1E7E6
:10650800B6F8F200FAF736FB80462846FAF732FB6F
:106518004FF07E51FAF77EFA01464FF07E50FAF7B7
:1065280035FC00240646594D404655F81410FAF734
:1065380079FB594A8146105FFAF720FB0146484625
:10654800FAF768FA3146FAF76DFB45F81400023499
:10655800062CE8D1514B4C4DB3F90000AC68FAF762
:106568000DFB014620460126FAF718FD00B906463C
:106578004B4968684E73214606F00AFA494CD5F82B
:1065880008802060286800F1004668680146FAF72C
:1065980049FB414605464046FAF744FB0146284672
:1065A800FAF738FA06F0F6F90146304606F0F0F93F
:1065B800606020683C4DF9F771FF29A3D3E90023F7
:1065C800F9F7C0FFFAF7D0F906F016F928806068E5
:1065D800364CF9F763FF22A3D3E90023F9F7B2FF9A
:1065E800FAF7C2F906F008F96880082001F044FFBC
:1065F80008B1264800E02648FFF74EFC1D4D2080D4
:106608003846FFF709FE95F87620002A00F08080CA
:106618001D4B18689C685F680146FAF703FB39460A
:1066280006463846FAF7FEFA01463046FAF7F2F916
:10663800214606462046FAF7F5FA01463046FAF7AB
:10664800E9F906F0A7F901462046FAF79FFB184931
:106658000446FAF78FFC88B316480021018057E0FA
:106668003B597E90A9E78140B00E0020A61D00206E
:10667800781E00207C1D00209C1E0020B41E0020D7
:10668800C41E002004000020D01E0020A40E0020FC
:106698000C000020C8190020701E0020640E002085
:1066A800771F0020680E0020600E00209A1E002030
:1066B8008FC2753C9C0E0020780E0020204606F004
:1066C80017F9274B1968FAF7ADFA06F095F8B0F5FF
:1066D800617FA8BF4FF46170F9F7CEFE1EA3D3E91E
:1066E8000023FAF759F8FAF73FF906F0C5F8044617
:1066F80095F87600FAF742FA2146FAF793FA06F087
:106708007BF8184B188003E0174B18805880988046
:10671800164A5379012B164B07D0164819885A8800
:106728009B8801804280838011E01349B3F90420DB
:106738000C88022014FB0020032290FBF2F080B2A8
:106748000C4A088019885B8890801180538007B0B4
:10675800BDE8F08FAFF30080A2EB0FE5DD169640A1
:10676800CC1E00209C0E0020B41E0020C81900205A
:106778009C1E0020700E0020960E0020AFF30080B3
:1067880010B5054C00202188FBF7A8FA6188012084
:10679800BDE81040FBF7A2BA1800002010B5094C5C
:1067A800206009480160094909480A60094A0A49FC
:1067B8001360029B039A03600848049B0A60036005
:1067C80010BD00BFB40E0020900F00208C0F0020D9
:1067D800BC0E0020940F0020C40E0020880F00205B
:1067E8000A4B1A6802EBC002D379FF2B07D008497D
:1067F8000978994203D9074830F8130004E00728BC
:10680800D4BF908840F2DC5000B27047B40E00202C
:10681800CC1F0020CE1F0020054B1A6802EBC000D9
:1068280090F9063019420CBF01204FF0FF30704735
:10683800B40E002010B500244FF48040FDF718F97D
:1068480008B1054B00E0054B1868054A8188A1523C
:106858000234182CF0D110BD900F00208C0F0020AE
:10686800F41E0020F8B53A4B3A4E1870054606EB70
:10687800C0000F46384C417820202160FDF7F8F819
:1068880008B101222260162D19D10024385900219F
:10689800FAF75CFB28B14FF48040FDF7E9F850BBEC
:1068A80025E02E4A3B1916190FCB86E80F002C4815
:1068B800017810344A1CC02C0270E7D1EBE716F8B7
:1068C8003570274B06EBC5061F70D6F804E0BEF1FD
:1068D800000FE0D00024BC42DDDA20011F4E0EEB91
:1068E800000136180FC9013486E80F00F3E7082DB8
:1068F8001C4B23D124E01A4F3F78012FF7D91A4CAB
:1069080000261034BE42F2DA54F8100C4FF07C51D5
:10691800FAF788F94FF07C5144F8100C54F8140C2D
:10692800FAF780F94FF07C5144F8140C54F80C0C29
:10693800FAF778F9013644F80C0CE2E70E2D01D18C
:10694800012000E000201874BDE8F840FFF772BF8E
:10695800B80E0020AC070108980F0020C80E0020D0
:10696800C00E0020771F0020D00E0020F0B58C4606
:10697800461C002300224CF803201033C02BF9D109
:106988000A4800EBC6014F6807B9F0BD0024074B61
:1069980013F83620944208DA200139180CEB000568
:1069A8000FC9013485E80F00F1E7F0BDAC07010815
:1069B800284B186810B500284AD027490A78531E72
:1069C800142B3DD8DFE803F00B3C3C24403C3C1C36
:1069D8003C3C3C3C3C2C3C3C3C3C3C242C001F4874
:1069E80001684A7832B11E4949890020BDE8104043
:1069F800FBF774B91B4B58780028F4D10146F5E72A
:106A0800174C0020E188FBF769F901202189EDE79F
:106A1800134C00202189FBF761F901206189E5E722
:106A28000F4C0020E188FBF759F901202189FBF779
:106A380055F902206189FBF751F90320A189D5E7AF
:106A48002020FDF715F818B1BDE81040FFF798BEF3
:106A580010BD00BF980F0020B80E0020940F002032
:106A680018000020771F002010B50024064B187866
:106A7800A04208D90549204631F814100134FBF723
:106A880021F9E4B2F2E710BDC00E0020DC1E0020A0
:106A9800064B1A780023D9B2914204D2044921F84E
:106AA80013000133F7E7FFF7DFBF00BFC00E002078
:106AB800DC1E00202DE9F74FA44B187803280FD9C6
:106AC800A349A44CB1F90420B4F90400002AB8BFC2
:106AD80052426FF06305A91A6432FDF709FAA080E3
:106AE8009A4A1678012E1DD89B4E9C4A3478651E0A
:106AF800142D00F2CB81DFE815F0A400C901C9010B
:106B08007B00B300C901C9015C01C901C901C90100
:106B1800C901C901D300C901C901C901C901C90114
:106B28005F00A3018E488B4B894F0168B7F806B008
:106B3800B3F800805F88B3F904A08A4C019100255E
:106B48001034B542D0D20FFA8BF0FAF717F854F890
:106B5800101CFAF767F8814638B2FAF70FF854F8BC
:106B6800081CFAF75FF801464846F9F753FF8146D3
:106B78000FFA88F0FAF702F854F80C1CFAF752F8F2
:106B880001464846F9F746FF019A814692F9000006
:106B980041420AFB01F0F9F7F1FF54F8041CFAF737
:106BA80041F801464846F9F735FFFAF701FA6E4B06
:106BB80023F815000135C3E70121664D674C042011
:106BC800FFF72AFE6E88704387B204202781FFF7FB
:106BD80007FE3818208101210520FFF71DFE2B88AC
:106BE800584385B205206581FFF7FAFD2B1826E08A
:106BF800584C02210420FFF70FFEA688704387B285
:106C080001210420FFF708FE6588544C00FB05703D
:106C180087B20420FFF7E4FD02213A1805202281FB
:106C2800FFF7FAFD704386B201210520FFF7F4FD56
:106C380000FB056105208DB2FFF7D2FD2B1863819B
:106C480024E101210520434FFFF7E6FDBC8860439E
:106C580086B20520FFF7C4FD404A3018508115E17F
:106C6800424A434E1768758897F806803B4C0020C7
:106C7800FFF7B6FD4FFA88F111FB05F3322593FBB8
:106C8800F5F840442080BF7B36880120FFF7A8FD37
:106C98007AB212FB06F191FBF5F3C5186580F5E0B1
:106CA800344C354E6178376811B9B888D08108E01E
:106CB800274A3988B2F906007A88FDF719F9274B6F
:106CC800D881264D2D4FEC8927493E680C803278B3
:106CD8004AB3264D2A4C0220FFF782FD2B68B3F9F0
:106CE8001010B3F91220FDF703F92168254B4C89E0
:106CF8001A88201A16B201B28E4203DA3E68317839
:106D08008A1803E003DD3F683878121A1A802D6864
:106D1800B3F9003095F91670104E7B43642093FB4D
:106D2800F0F2A418B48013490C4F8D7A65B1084B62
:106D380018880E4EF88038819A88084D7A815C88C8
:106D4800BC81376803241FE0024BF1E7C00E002026
:106D58009E1F00208A1E0020B80E00201800002068
:106D6800940F0020C80E0020DC1E0020B40E002066
:106D7800600E0020771F00208C0F0020BC0E002022
:106D8800C40E0020BA0E002007EBC401B5F90600B6
:106D980091F906306422584390FBF2F6EE802046C3
:106DA800FFF71EFD01343118E9800235072CEBD1BD
:106DB8006CE0A54FA54B78781E6810B9B488D481CB
:106DC80008E0A34A3188B2F906007288FDF790F806
:106DD800A049C8819C489F4C9F4FE589837A3D8094
:106DE800032001211BB1FFF717FD994D02E0FFF7C2
:106DF80013FD9A4D6E88704387B202210320FFF776
:106E08000BFD2D88012100FB05720420E280FFF7AD
:106E180003FD704386B202210420FFF7FDFC00FB4E
:106E28000561218103208B4CFFF7DAFCE388C01849
:106E3800E0800420FFF7D4FC2789C519258125E0C7
:106E4800864FBF88032402212046FFF7E5FC7843DC
:106E580086B201212046FFF7DFFCC4F1060359087A
:106E68007E4D35F811207B4D00FB026086B225F877
:106E780014602046FFF7B4FC331825F814300134A9
:106E8800072CE0D1724F744AF98811802020FCF752
:106E9800EFFD002845D00020FFF7A2FC6D4F054606
:106EA80038800120FFF79CFC6D4978800B7A002B15
:106EB80037D06C4C6C4B266832786C4E02F002016D
:106EC800CCB2D4B13668B3F9001096F90E2096F911
:106ED8000660B3F902304A433224714292FBF4F25D
:106EE8004B436FF0310692B293FBF6F156187519C1
:106EF80093FBF4F43D80141911E03168B3F90240B2
:106F080091F90620B3F900305443322294FBF2F68B
:106F1800AD193D8091F90E104B4393FBF2F4001923
:106F280078800026514F4B4D3B68A85F33F92610F7
:106F380003EB8602B2F90220FCF7DAFFA853023607
:106F4800102EEFD147490C68207800F00407FBB2F7
:106F58002BB9414A464916880C7801231CE0454D57
:106F68002E780E2E0AD0082E08D0434A02EBC6010E
:106F78004C78002C14BF0225002500E004250026CB
:106F88003E4F07EB46037019C0B219890136FAF76C
:106F9800A5FE042EF4D1DCE7A34209D22E4F37F91F
:106FA800131036B2B142A8BF0E46B6B20133F3E7AA
:106FB800002427462E4803789F4272D2234D2A6820
:106FC800518830B2884204DD234BE25A8D1BA91840
:106FD800E1524FF48040FCF74BFD1F4DC0B1284AE9
:106FE800264B1168B3F906004B8926499842174881
:106FF80005DD02680968285F4988528804E002684C
:107008000B68285F91881A88FCF772FF28533EE0C6
:10701800DFF83880285FD8F8003019885A88FCF7DC
:1070280067FF174928530B681448B0F90620988958
:10703800824205EB04092ADA1020FCF719FDD8F87A
:10704800002008BB118820E0771F00208C0F00204B
:107058009E1F002018000020DC1E00208A1E002031
:10706800881F0020880F0020600E0020B40E00202A
:10707800C00E0020B80E0020AC070108CE1F00206B
:10708800C40E0020900F00209188A9F8001006482F
:1070980043781BB905490648625A2252013702341F
:1070A80088E7BDE8FE8F00BF771F0020F41E002090
:1070B800DC1E0020024B1868003018BF0120704702
:1070C800980F002044F25063984203DDA0F50C406D
:1070D800A038704703498842BCBF00F50C40A03077
:1070E800704700BFB0B9FFFF10B5F9F747FD0021A1
:1070F8000446F9F753FF08B1204601E004F10040C7
:107108000549F9F743FE0549F9F78CFD05F040FB01
:10711800034B186010BD00BF8096184B35FA8E3CA3
:107128002800002010B5044C002320702361FEF7CE
:1071380075FB606110BD00BF08110020F8B51D4641
:1071480014460E46F9F71AFD6968F9F76BFD3146E2
:10715800F9F768FD2168F9F75DFC2060F9F728FF69
:10716800ED68074605F10040F9F722FF0646284674
:10717800F9F71EFF314602463846FCF7B9FEF9F723
:10718800FDFC2060F9F714FFF8BD0000F8B5101AEF
:107198000C461F46F9F7F2FC0546381BF9F7EEFCDA
:1071A800174B079E1968F9F73DFD294604462846FE
:1071B800F9F738FD214607462046F9F733FD014621
:1071C8003846F9F727FC05F0E5FB0E49F9F72AFDE3
:1071D800F9F714FF06990860214605F1004005F00B
:1071E800D7FB0949F9F71EFD0849F9F713FCF9F728
:1071F800DFFE0028BCBF00F50C40A0303060F8BDB1
:10720800280000202C7D8E3FA00CB34500A00C4622
:1072180010B50446002003460D49CA5CA2B12E2AC7
:1072280004D1013394B1C91800220A55084AD25C26
:107238000A214843A2F13001092901D830388018C1
:107248000E2B02D80133E7E710BD002010BD00BFA8
:107258007C100020000000002DE9F843224B07466F
:1072680048681D68381A0C469146F9F787FC294684
:10727800F9F78CFD1D4920610A68A6688046907858
:10728800F9F778FCF9F70AF915A3D3E90023F9F718
:1072980059F902460B4600201549F9F77DFAF9F726
:1072A80063FB2946F9F7B6FB01462846F9F76EFD58
:1072B800314605464046F9F7ABFB01462846F9F743
:1072C800B1FC01463046F9F7A5FBD9F80810206152
:1072D8006760A060F9F7A6FCF9F76AFEBDE8F883D5
:1072E800182D4454FB211940AC10002064100020D4
:1072F8000000F03FAFF30080014B1860704700BFFB
:1073080064100020F8B52D4B187810B1012850D121
:107318000AE02B4B2B4A58782B4B02EB00111868CC
:107328004968FEF72DFA41E0274D2868FEF72DFA47
:1073380000283ED0224C2178012926461ED1FEF78E
:107348006DFA06466069321A632A35D9216904291B
:1073580012D81C4F286807EB01135968FEF710FA7A
:10736800607807EB00172868B968FEF7F4F9226916
:107378006661511C21611CE0022018E022693AB9BB
:107388006478104B286803EB04114968FEF7F8F994
:1073980033690B4C8B2B09D80C4A0B48D15C00681D
:1073A800FEF7D4F921694B1C236102E00320FFF7A3
:1073B800B9FE034A00205060F8BD00BF94100020B9
:1073C800081100202C0C0108601000209E0B0108F9
:1073D80010B50B4CE37A8BB10A48017804290DD912
:1073E800094A0A4B1068516818605960FFF77CFE1B
:1073F8000748084B028801211A80217310BD00BF7D
:10740800771F0020641F00204C1F0020301F002021
:107418009A1E00206C100020002370B51C460F48EF
:107428000F4A104E104D00211952142060439952F2
:1074380000223250595335180C4E6960AA603250F8
:1074480035180B4E6960AA60013435180233022CD6
:1074580032506960AA60E2D170BD00BFA810002058
:10746800961000202010002028110020C80F0020AE
:10747800C410002070B5044600791F4D1F4EF9F75F
:1074880079FB1F49F9F782FC2860A07BF9F772FBAA
:107498001B49F9F77BFCEE6068606079194DF9F7D4
:1074A80069FB1949F9F772FC2860E07BF9F762FB80
:1074B8001349F9F76BFC6860607EF9F75BFB1349C9
:1074C800F9F764FCEE60A860A079114DF9F752FB5A
:1074D8000D49F9F75BFC2860207CF9F74BFB08495C
:1074E800F9F754FC6860A07EF9F744FB0749F9F7FF
:1074F8004DFCEE60A86070BD481000200000FA4402
:107508000000C842001000200000204100007A441A
:10751800101000202DE9F3411A4F1B4D3A700E460A
:107528001A491B4A086000201360DDF82080FFF725
:10753800F9FD6E70FEF772F9A860387800246C6067
:10754800A0420CBF012503254046FFF793FF114BCE
:10755800009403EB06162146102072682B4602F0B1
:107568009BF90D49086030B94FF4807002B0BDE84E
:10757800F041FCF701BC012002B0BDE8F041FFF783
:10758800D1BD00BF94100020081100203411002044
:10759800641000202C0C010860100020F7B5264B61
:1075A8001D78032D44D1202002F068F8234E0446AC
:1075B80038B102F0D7F931682046C968FEF7E0F81B
:1075C8000AE03268009021462020D2682B4602F05B
:1075D80063F9044600282DD019484FF488554FF414
:1075E800884605850685174F3868FEF7BFF858B1F5
:1075F800134D38684FF48856AE61FEF7BCF8014663
:107608002046FEF7A3F82E852046FEF7AFF800289F
:10761800E9D00B4D0B4B4FF48846AE6120461F68EE
:10762800FEF7A9F801463846FEF790F82E85DAE706
:10763800022000E02846FEBD081100203411002079
:107648000010004860100020F7B50368164C174D6D
:1076580023600968164E61600068164FFFF744FD05
:107668001548019694E80C00009095E80300FFF790
:107678008DFD6B68114A61683668C81A1660F9F79B
:107688007DFA0F4A1168F9F7CDFAF9F791FC2968E4
:10769800786020680B4A431A0B483B600168166003
:1076A8000A4BCA881A80FEBD741000204C1F0020A7
:1076B800F0100020381100209C10002070100020CD
:1076C8002800002000110020641000203011002044
:1076D800264BF0B51D68024600F110011678AB196B
:1076E80014465B7803F00403DBB2013263B18A42CB
:1076F800F4D10020F0BD13B10A225343DBB210F8D5
:10770800011B30395B18DBB2211A0229F3DC002196
:10771800844209D911B10A225143C9B210F8012B88
:10772800303A8918C9B2F3E72E2E11D1013404205A
:1077380000220A2672432678AF197F7807F00407DB
:10774800FFB217B1303A921901340138F1D100E093
:107758000022074C6420614300FB021106240548FF
:10776800B1FBF4F200FB0320F0BD00BFA401002030
:1077780040420F00809698002DE9F04F9A4B186808
:107788008BB0B8B9994C21784A1E032A00F2658556
:10779800DFE812F0F704F70442052C052068FDF72E
:1077A800EAFF93490B78012B044600F0DF8008D3E9
:1077B800022B06D08C4C2068FDF7D8FF0028EDD1AD
:1077C800E0E7242C07D18B4B8B4A8C4C0021197095
:1077D80011702170C5E02C2C02D02A2C40F0828038
:1077E800854D844A2978864B1578864A0020585456
:1077F800B5B918781570472868D15978502965D1D6
:107808009878472840F01785D978472940F013859C
:107818001B79412B40F00F850120107000F00BBD43
:10782800117801293AD1022D05D11846FFF750FFEA
:10783800754908604AE0032D07D11978532945D1C5
:10784800714802685342036040E0042D05D1184690
:10785800FFF73EFF6C4B586038E0052D07D11B78C9
:10786800572B33D168494A68504248602EE0062DAC
:1078780007D119786548302994BF00210121C172C8
:1078880024E0072D04D1FFF7C3FC614A10701DE006
:10789800092D1BD1FFF7BCFC5E4B16E0022915D160
:1078A800072D0CD10120FFF7B3FC41F218425043D9
:1078B8004FF47A71584BB0FBF1F0188006E0082DB0
:1078C80004D10120FFF7A4FC544B1880494B4A49C6
:1078D800013500202A2C1D70087039D15048012428
:1078E80004703EE00D2C4E4A01D00A2C26D11478A3
:1078F800FCB1434C21786478A1F13000C3B2092B64
:1079080084BFA1F13703DBB2A4F1300003F00F020A
:10791800C3B21101092B84BFA4F13703DBB2374C82
:1079280003F00F0289182078CBB2C21A514251EBEA
:1079380002043B4B002018707CB912E02E490B78EA
:107948000E2B03D82E48C45401330B70127842B959
:107958002A4B1A7854401C7003E02A4A10780128F0
:1079680000D00020C00700F1338123E72D4B1978A0
:10797800002208293FF61EAFDFE801F00A051119B9
:1079880027607C96A000622801D1022105E01A70C8
:10799800B52C7FF40FAF1C78611C19700AE72249D7
:1079A800224A087003261E701070214B0BE01F4EF0
:1079B8000421197032781E4BA1181878CAB2101811
:1079C80018701C4B32701C70F4E605211970174BA7
:1079D800174E1A783078A118CAB210183070164E9F
:1079E8001A703480E6E600BF6010002008110020FD
:1079F8009410002069100020FC0F0020FD0F0020CB
:107A08007C100020C40F00204C1F0020771F00208E
:107A1800641F00201E1F0020221F0020FC100020D1
:107A2800061100206A100020041100205C100020BC
:107A38006B100020C50F0020FE0F00206C490626A1
:107A48001E700A786B4BA6181878F2B210181870C6
:107A5800694B0A70198801EB0424A6B2B6F5007FB9
:107A680001D81E8003E000221A80644B1A7000249B
:107A7800634983E35E495F4E0A783078A318DAB227
:107A8800101830705E4E0A7033885B4AC72B98BF57
:107A98005C49108898BFCC545C1CA1B288423180E4
:107AA8007FF488AE072107E0514808261E70037846
:107AB800A3423FF47FAE0021504B6EE74D4E1A7043
:107AC800337883427FF476AE4F4C207806283BD03B
:107AD80005D8022813D003287FF46CAE23E01228BF
:107AE80047D030287FF466AE464A484C1679454A56
:107AF800102E88BF102626702178002347E0414CBD
:107B0800434E6368A06821697360424B30604FF44C
:107B18007A7291FBF2F6404C404918782680C87278
:107B280001223F4923E037494A7912F0010004D085
:107B38000E79F41E634253EB04003649087000289E
:107B480039D1364AD07236E02E4EF47A14F001015B
:107B580004D0B07AC21E534253EB02012D4E31704D
:107B680009B92E4CE17227482E4990F82F200A7047
:107B780021E024482C49866942692C4B0A8042F24C
:107B8800107496FBF4F0188001222949EFE70C32B3
:107B98008B4210DA12F8046C264812F8034C1E5473
:107BA800254E26489C5512F8014C16781C54244C36
:107BB8001E550133EBE71A490A78002A3FF4FAAD5B
:107BC8001B4B1E78002E3FF4F5AD00240C701C7082
:107BD8001C4CA068E060FDF721FEA060202000F0AA
:107BE80055FC19490A78012A30D100232FE000BF3B
:107BF8005C1000206B100020FE0F00206A1000208F
:107C08000C12002044110020C50F0020651F002021
:107C18004C1F00202E1100201E1F0020771F00205F
:107C280068100020641F0020221F0020FC10002084
:107C3800051100200C1F00203A1F0020541F0020AF
:107C4800661F0020081100203211002001230B704C
:107C58000C787E497E48CA7AC480002A3FF4AAADCF
:107C68007C4B1C78042C7FF6A5AD4F7807B90F73B1
:107C78000D7B15B90FB1FFF7ABFB774E774F307817
:107C880097F800C0764D421C052192FBF1F301FBE9
:107C980013243470734E002306EB84027248734930
:107CA8001C58DFF814E2724E5C50724FDFF80C92E9
:107CB80094FBFEF103EB000A06FB014042F210744C
:107CC800D95190FBF4F716681060BCB253F80970EC
:107CD80025F8024FC6EB07084044052643F809007B
:107CE80090FBF6F00EFB01016348BCF1010F19503F
:107CF80005D1023CB4F5797F98BFCAF80010043367
:107D08001432082BCAD15D4D5D4CFDF787FD2A68FA
:107D1800801AF8F72FFF5B49F9F738F82060FDF76C
:107D28007DFD286025684FF07E512846F9F718F93F
:107D380008B94FF07E55256006A907AC4A48524B52
:107D48000194009103C80CCBFFF720FA069A4F491B
:107D58004F4C6423B2FBF3F00880079A3B4892FB30
:107D6800F3F3027B23800AB90A80228049490C7800
:107D7800002C36D0424F3C4E3968474D4FF07E506C
:107D8800F9F704F82B6804463068C01AF8F7F6FECD
:107D98002146F8F747FFF9F70BF972686968074653
:107DA800501AF8F7EBFE3D4B1968F8F73BFF2146F0
:107DB800F8F738FFF9F7FCF8394B3A49B3F90240BC
:107DC80004FA80F0022490FBF4F2B3F9000000FA00
:107DD80087F090FBF4F492B2A0B24A8008805A80EF
:107DE80018802C4B204C01221A70184B61682A4AC3
:107DF80020681C7A516010601CB9DA79002A3FF4B7
:107E0800D9AC294E294D2A4C01960095164F294E7A
:107E180094E80C00FFF7BAF961687868081AF8F76F
:107E2800ADFE1E4B1968F8F7FDFEF9F7C1F8706052
:107E38000A48226890F900303C68012BC4EB020123
:107E480031603DD0022B7FF4B5ACA0E0771F002055
:107E5800561E0020641F002040110020BC10002086
:107E68009E1000209C0F00204C1F00202011002095
:107E7800806967FFB0100020F40F0020B8100020C0
:107E8800AC10002000007A44301F00202C1F002076
:107E9800381F0020EC1000208C1000202800002043
:107EA80058100020BE100020F01000209C10002068
:107EB800741000203811002080969800F4100020DB
:107EC800002634463546DFF818C3AF4F5CF825B0B6
:107ED800CDF80CC05846F8F751FE3968DFF8E4923F
:107EE800DFF8E882F8F79EFEF9F762F834F809201F
:107EF800A649801A83B21FB2635238460497A44F2A
:107F0800F8F73CFE3968F8F78DFEF9F751F84FF0AD
:107F1800140A82B29F4B0498196805920AFB058AD5
:107F28003B4658445246FFF709F90599DFF8B4B2C1
:107F3800DDF80CC00A1824F80B205CF8250051461F
:107F48003A46FFF789F994494FF4FA62FBF7D0FFF4
:107F580034F809303BF80420313399B2622998BFCC
:107F68000020801883B22BF804308C4940F6B832D0
:107F780018B2FBF7BDFF58F80610894A2BF8040021
:107F88000135B15002341436022D9CD112E4854FCC
:107F98002D683E68B6F908206C08A24228BF224620
:107FA800814C268897B239B230B2814209DD794BCB
:107FB8007E491868F8F736FEF8F7FAFF8719BFB256
:107FC80027807B4A7B4E14683168661A3046FFF773
:107FD80079F80028D8BF404241F293139842CCBFA9
:107FE8000020012050B33046F8F7C8FD7249F8F771
:107FF80019FE04F041FC06462846F8F7BBFD014689
:108008003046F8F70FFEF8F7D3FF6C4A6349108043
:1080180000B240F6B832FBF76BFF201848F6A044D0
:10802800A04203DDA0F50C40A03804E00028BCBF46
:1080380000F50C40A0306249086001E0604D2C60FA
:108048005F4B1D68C5F50C502830F8F797FD5A4965
:10805800F8F7E8FD064604F09BFB0990304604F06B
:108068000BFC002508902C462E4638B2F8F786FD02
:1080780008AADFF8189152F82610DFF824A1F8F7BB
:10808800D1FD80464F48005FF8F778FD014640462D
:10809800F8F7BEFCF8F78CFF4FF47A7224F8090061
:1080A8004949DFF8448100B2FBF722FF81B20BB2E5
:1080B80024F8091018460493F8F760FDD8F8001062
:1080C800F8F7B0FDF8F774FF4FF0140B049A314934
:1080D8000BFB06AB1FFA80FC0968CDF80CC04346C1
:1080E80010465A46FFF72AF842460346594639F9D8
:1080F80004000493FFF7B0F8049ADDF80C808018A8
:1081080008EB000CDFF8DC801FFA8CF124F808106B
:1081180008B240F6B8322149FBF7EAFE55F80A20C2
:108128002A4B28F804000136EA5002341435022E8E
:108138009BD11C480368197931B1214A1468244A33
:10814800642094FBF0F11180224C1B88206898422F
:108158000ED91749174B0A681C68101BFEF7B2FFA7
:1081680042F210710028B8BF404288427FF722AB24
:10817800194B1A4A1C881649012010700C80FFF709
:1081880019BBFFF7BFF868E048100020F00F002087
:1081980000100020AC10002030F8FFFF48F4FFFF6B
:1081A800C410002064100020301100200000C842D4
:1081B800F010002000110020D30237392C110020C4
:1081C80070100020BE10002018FCFFFFC80F002010
:1081D800881E00209C1000206C100020BC1000207D
:1081E80038110020281100201010002062686078E3
:1081F800531C411CCAB263600523B2FBF3F003FBB6
:1082080010216170FDF70AFB154AA060154800238C
:10821800C372137001200BE0FDF700FBA36840F662
:10822800C411C01A884218D9202000F037F9042058
:10823800FEF778FF11E00C498A78522A7FF446ABA2
:10824800CB784D2B7FF442AB087943287FF43EABC3
:10825800064A02211170FFF739BB0BB0BDE8F08F59
:10826800641F0020771F00207C100020C40F00200E
:108278003D4B2DE9F047B3F90000DFF804913B4F7F
:10828800F8F77CFC3A49F8F7CDFC044604F0F4FA18
:108298000646204604F07CFA0546D9F8000090F816
:1082A8000380B8F1000F2BD0324CB7F90210B4F8A4
:1082B80002A00FFA8AF2881AFEF704FFC8F100013B
:1082C8004246FBF715FEB4F8008000EB0A03B7F945
:1082D800000063800FFA88F7C01BFEF7F3FED9F899
:1082E8000010CA785142FBF703FE00EB080297B270
:1082F8002780B4F90200F8F741FC804638B206E05E
:10830800B7F90200F8F73AFC8046B7F90000F8F729
:1083180035FC294607464046F8F784FC3146814635
:108328003846F8F77FFC01464846F8F771FB1249D2
:10833800124CF8F72BFDF8F73BFE314620804046FB
:10834800F8F770FC294606463846F8F76BFC0146F4
:108358003046F8F75FFB0849F8F718FDF8F728FEEC
:108368006080BDE8F08700BF9A1E00202811002019
:1083780035FA8E3CA81000200000204196100020FD
:108388006410002038B5254CE37A2246002B3ED0F5
:108398002348017804293AD92248817A79B1E179C8
:1083A800002939D12048214B217201221970011D61
:1083B800E271FFF749F91E490220087038BDC37AF7
:1083C800E171C3B11B4A1068408900F075F890B19B
:1083D800237A002B20D115481749037017480A68DB
:1083E8004B6802600125011D43602572FFF72CF9D7
:1083F8000F48057038BD0D48084B027800211972E6
:1084080052B901210170BDE83840FFF705B80023D3
:10841800D3711372064A137038BD00BF771F00204E
:10842800641F0020881F0020301F00202C0000201F
:10843800BC100020641000204C1F0020241F0020C6
:108448000A4B1A68811A00290EDB094A1178042997
:108458000AD900F5123000F5F8721A60054B998AAE
:1084680088B280F488429A82704700BFA410002026
:10847800641F002000100048034B196808420CBF15
:1084880000200120704700BF10120020024B1A681C
:1084980010431860704700BF10120020024B1A6882
:1084A80022EA00001860704710120020014B18687B
:1084B800704700BF10120020094BB3F90020002AB2
:1084C800B8BF5242824209DAB3F902100029B8BF94
:1084D80049428142ACBF002001207047002070470C
:1084E8009E1F002010B544780078002303FB03F199
:1084F8001939614301F6C4115943414340F6C41286
:1085080091FBF2F1034A22F813100133072BEDD146
:1085180010BD00BFBE1F00202DE9F0478478C77842
:108528001D48C4F164084FF00A0C5FFA88F80CFB88
:1085380004FCC7F1640900231D1BADB22EB2002E46
:1085480004DCB8BF224602DB012200E0424615FBEC
:1085580005F57D4312FB02F295FBF2F509EB0502E6
:1085680072434FF00A0A92FBFAF60CEB0605ADB21D
:1085780045800A884E882DB2B61A754353444FF485
:108588007A7695FBF6F59BB25219782B20F8022FD4
:10859800D2D1BDE8F08700BFA41F002008B54FF472
:1085A8000040FBF765FA30B90120FBF761FA80F06B
:1085B8000101C8B200E0002000F0010008BD000081
:1085C800014B1860704700BF9C120020074B1968C8
:1085D8000B7A032B09D8DFE803F00202040600F047
:1085E80091BB00F0D7B900F0BBBA70479C120020CD
:1085F80008B5037A032B12D8DFE803F00202070C50
:108608000A490B4A00F086FB08E00849084A00F0CE
:10861800C9F903E00549064A00F0AAFA28B9082072
:10862800FBF7AAFB02480022026008BDCC1F00200D
:1086380094120020174B10B5186004460023608977
:10864800154A98520233242BF9D1144801600820A6
:10865800FBF70EFA10B12046FFF7CAFF4FF480303F
:10866800FBF706FA20B120460D490E4A00F038F90A
:108678000120FBF7FDF928B109480A49BDE8104077
:1086880000F03CB94FF40040FBF7F2F90028F3D1B1
:1086980010BD00BF9C120020CE1F002090120020A9
:1086A800CC1F002094120020037A032B09D8DFE89E
:1086B80003F00202040600F065BB00F09FB900F069
:1086C80075BA00207047000010B5114C002308202F
:1086D8002370FBF7CDF920B10E480068FFF7E4FFDF
:1086E80020704FF48030FBF7C3F9094C10B100F04B
:1086F800EDF82070217849B14FF40070FBF7B8F914
:1087080020B1054A136818680168884710BD00BF82
:10871800981200209C12002090120020054B197816
:1087280029B9054A1368C01AC143C80F7047012008
:10873800704700BF98120020A01200200E4A0F4B6D
:10874800127802F0030202EB800223F8121003EB06
:10875800C00233F830105388CB189188D2885B1840
:1087680012FA83F1064A8BB222F81030042118B2AB
:1087780090FBF1F398B270478C120020141200207D
:108788007412002070B500241E4B1878A04238D906
:108798001D491E4A0B682BB912681D49508921F8DA
:1087A80014002BE015681748072C94BF2E5D264649
:1087B8003146984705464FF40070FBF759F930B138
:1087C800144801680B683046DA6929469047A5F2D3
:1087D800EE26B0B240F2DC51884202D90B4D2B682C
:1087E8005D89FFF7DBFE0A4E10B126F8145005E04C
:1087F80020462946FFF7A2FF26F814000134E4B208
:10880800C2E770BDCC1F0020941200209C120020EB
:10881800CE1F00209012002010B5064C237843B1DB
:10882800054801680A6813689847FFF7ABFF0020FE
:10883800207010BD9812002090120020024B1A7868
:10884800501C1870FFF79EBF8C12002008B500F569
:108858009C400C4B203018604FF40070FBF708F96F
:1088680020B109490A68106803699847FFF796FE1E
:1088780018B1BDE80840FFF7CFBFBDE80840FFF7D3
:10888800DDBF00BFA012002090120020F8B50546F9
:108898000F46441E14F8011F49B1054E304606F034
:1088A80023FE0028F6D0861B631BBB55F2E7F8BDF4
:1088B8007C0C0108014B33F811007047CE1F0020D3
:1088C800014B01221A707047A4120020034B18783C
:1088D80010B100221A700120704700BFA4120020B6
:1088E80008230B700AB1024810600120704700BFCE
:1088F800BD8800080846F9F7F9BA0000084B10B51A
:1089080004460B604FF40040FBF7B2F808B10820AA
:1089180020700120FBF7ACF808B10C21217010BDC4
:10892800FD880008034B53F82100410801F57772D0
:1089380090B27047B012002038B50446FCF754FFD7
:10894800104B1A6840F6C411821A8A421A460E4B16
:1089580001D9002119701B7810600BB90F2C10D1A8
:108968000A48094A002101704BB1094DED18182B2E
:1089780005F8014C03D101230370117038BD013390
:10898800137038BDA8120020AC120020AD120020D0
:10899800E0120020024B032143608360417370475B
:1089A800A0860100F7B50746002505230E461446A4
:1089B8000D490E4A0095082000F06EFF79890C4B8E
:1089C800A1F57772186051002B460A4A9950043372
:1089D800302BFAD10CB1084921600C2200303270DA
:1089E80018BF0120FEBD00BF41890008A086010014
:1089F800FC120020B01200202D890008344B1A7890
:108A080010B50AB9002010BD00201870314B997DAF
:108A18000A07F7D4587819782F4A00F0070441EA72
:108A280004211160997801F03F04640144EAD00000
:108A38005060DC78A00040EA9110197901F0010437
:108A480040EA84209060587900F00F04E40144EA79
:108A58005101D160997901F07F04240144EA101092
:108A68001061DC79600040EAD111187A00F0030443
:108A780041EA44215161597A01F01F04A40144EAF2
:108A8800900090619C7AE00040EA5111D161187B16
:108A9800D97A00F0070441EA04211162597B01F0F8
:108AA8003F04640144EAD00050629C7BA00040EA85
:108AB8009110D97B01F0010440EA842090621B7C6C
:108AC80003F00F00C30143EA5101D162012010BD38
:108AD800AD120020E0120020B0120020024B53F823
:108AE8002100C0F3CF0070473413002010B50446AE
:108AF800FCF77AFE154B1A68811AB1F57A6F1A4697
:108B0800134B01D9002119701060187820B9A82CCE
:108B18001AD1104B187006E0022802D10E4A1470C0
:108B280001E0242801D80D490C540B49084A0130AA
:108B3800C3B2087813704100481D834204D1002352
:108B48000449137001220A7010BD00BF04130020ED
:108B5800741300202D130020001300200813002098
:108B68004FF4E13301214360836041737047000093
:108B780037B5002300930D461446094908204FF4E1
:108B8800E132012300F088FE064908600CB1064A6C
:108B98002260102300302B7018BF01203EBD00BF9B
:108BA800F58A000830130020E58A0008124B1A786D
:108BB80010B50AB9002010BD1049002018704B7874
:108BC800012BF7D10E480278102A01D91021017023
:108BD80001780C4A0023D8B2023288420AD212F82D
:108BE800010C12F8024C40EA0424074840F82340DC
:108BF8000133F0E7012010BD2D13002008130020D9
:108C0800001300200B13002034130020114B012205
:108C180010B51A700446FCF7E7FD0F4A01461068C4
:108C280011600B1A0D4841F288318B4203600C4BDE
:108C380001D900221A7018780A49E4B20F280C5496
:108C480003D109490120087010BD054A431C13705F
:108C580010BD00BF8513002078130020801300206A
:108C680084130020BA1300207C1300201E4B1A78AE
:108C78002DE9F0411AB31D4C1D4D2678077895F85B
:108C880000C002231B4AD45C44FA06F404F00F0423
:108C9800E5B2BD4203F101080BD20B2D09D8D55C12
:108CA80012F8082005EA0C0502EB0525124A42F8DD
:108CB80024500233102BE5D10B4B00221A70007898
:108CC80088420ED90D4A107860B10D4B0A481A78BF
:108CD80050F8211002B1490801F5777398B2BDE840
:108CE800F0810020BDE8F0817C130020751300207E
:108CF800B9130020BA130020881300208513002020
:108D0800B81300204FF4E1330121436083604173BD
:108D18007047000013B5037A14465BB1012B13D1D9
:108D2800124A03201070124A07201070114803706D
:108D38000C2308E00D4A022010700D4A0320107021
:108D48000C48037007230B70002100914FF4E132A7
:108D580008200949012300F09FFD084A10600CB162
:108D6800074B2360003018BF01201CBD751300207D
:108D7800B9130020B8130020158C0008CC1300206C
:108D8800758C0008014B1878704700BF7C130020D1
:108D9800014B1860704700BFD4130020034B1868BC
:108DA8000178D1F1010038BF00207047D4130020AA
:108DB800034B186801784A1E534253EB0200704770
:108DC800D413002008B54FF40060FAF751FE20B123
:108DD8000420BDE8084000F017BD08BD084B18780E
:108DE80060B108490A68537813B1074A117D01E058
:108DF80006484178081C18BF0120704701207047B9
:108E0800D0130020D4130020881F0020771F0020D3
:108E180008B5FFF7C3FF18B1BDE8084000F062BA13
:108E2800FFF7C6FF18B1BDE8084000F09DBB08BDBC
:108E380008B5FFF7B3FF08B100F094F8FFF7B8FFE3
:108E480018B1BDE8084000F07FBA08BD0F4B18788C
:108E580010B5D0B1FFF7C2FF0D490A788242044627
:108E680013D070B1FFF79AFF18B10A4B186800F0D9
:108E780091F8FFF79DFF30B10648006800F07CFAD2
:108E880001E0FFF7D5FF02490C7010BDD813002090
:108E9800D1130020D413002008B50121042000F0CC
:108EA800BFFC054B1870FFF78DFF04490870BDE83B
:108EB8000840FFF7CBBF00BFD0130020D813002015
:108EC80008B5094B187870B1FFF788FF58B1FFF75C
:108ED80065FF08B100F0A0F8FFF76AFF18B1BDE818
:108EE800084000F07DBA08BDD813002038B5064CFC
:108EF80005465E212068FCF729FC20682946BDE864
:108F08003840FCF723BC00BFEC130020024B186864
:108F18005E21FCF71BBC00BFEC13002010B50A4C07
:108F28005E280146206805D15D21FCF70FFC20680A
:108F38003E2105E05D2903D1FCF708FC20683D21AE
:108F4800BDE81040FCF702BCEC13002010B5044645
:108F5800C0B2FFF7E3FFC4F30720BDE81040FFF7F6
:108F6800DDBF000010B5084B084C19782068FCF7E5
:108F780011FC074920680968FCF702FC20680421F5
:108F8800BDE8104000F0AABBE4130020EC13002059
:108F9800DC13002037B50546042000F06FFB154CA4
:108FA80001462060A0B14279134B81681A70134AB8
:108FB80011604FF41651FCF7E3FB20680221FCF71F
:108FC800E9FB2068042103B0BDE8304000F074BB21
:108FD800AB784FF4165200930420022300F05CFC97
:108FE800054942792060054B80680A70186003B013
:108FF80030BD00BFEC130020E4130020DC13002078
:1090080008B5044B1868FCF7B1FBD0F1010038BF74
:10901800002008BDEC1300202DE9F041FFF7F0FF18
:10902800002800F04181FCF7F9FBA04B1A68811A6F
:109038007C2940F2398118609D480478651C0570C8
:10904800002404F12406F0B2FFF750FF994B33F9DE
:109058001400F7F793FD984A05461088F7F78EFD38
:1090680001462846F7F792FE9449F7F7DBFDF7F734
:109078009FFF013400B2FFF769FF032CE1D13020D4
:10908800FFF734FF8E49B1F90000FFF75FFFFFF7E4
:109098003DFF8748067816F0030629D1894D102030
:1090A800FFF724FF2B68642493FBF4F210B2FFF758
:1090B8004DFF2120FFF71AFF296891FBF4F004FB0C
:1090C800101484EAE473A3EBE47318B2FFF73EFFCD
:1090D8001420FFF70BFF7C4AB2F90000FFF736FFB8
:1090E8001C20FFF703FF3046FFF730FFFFF70EFFA6
:1090F8006F490878430740F0B180744D0220FFF7AC
:10910800F5FEB5F900300A2593FBF5F0FFF71EFFD1
:109118000220FAF7ADFC002848D06D4F6D4E387824
:109128003478B4FBF0F26C4C40F634014A432188A1
:1091380091FBF0F800FB18102A23B2FBF3F24FEA78
:10914800001399B241EA022C1FFA8CFEC2F30322E3
:109158004EEA02080620FFF7C9FE0FFA88F0FFF76B
:10916800F5FE20883F783678431C9AB292FBF7F1D7
:1091780007FB112020806E2416FB04F2152392FBB6
:10918800F3F43A206427FFF7B1FEB4FBF7F6304654
:10919800FFF7DCFE3B20FFF7A9FE07FB164188B26C
:1091A800441D94FBF5F210B2FFF7D0FE2020FFF724
:1091B80063F9002850D0494C494F1320FFF796FE19
:1091C8002568002DB8BF6D4295FBF7F630B2FFF762
:1091D800BDFE1B20FFF78AFE23680A26002BB8BFB6
:1091E8005B4293FBF6F142F2107591FBF5F005FB3B
:1091F800101210B2FFF7AAFE2320FFF777FE2368AC
:10920800002BACBF4E205320FFF7A0FE1220FFF723
:109218006DFE61680029B8BF494291FBF7F000B2C2
:10922800FFF794FE1A20FFF761FE6268002AB8BFB4
:10923800524292FBF6F696FBF5F305FB136108B272
:10924800FFF784FE2220FFF751FE60680028ACBFBC
:1092580045205720FFF77AFEFFF758FE144B1A787F
:10926800282A21D100241C70FCF7D8FA4FF47A750B
:109278003C24B0FBF5F61720FFF738FEB6FBF4F5F3
:10928800B5FBF4F104FB1150030218B2FFF75EFEC0
:109298001820FFF72BFE04FB156210B2FFF756FEED
:1092A800BDE8F041FFF732BEBDE8F081E8130020C9
:1092B800E0130020C41E00200400002000007A44AF
:1092C800840E00209C0D00209A1E0020541E0020B1
:1092D80002000020C4190020E21300204C1F0020C7
:1092E800A08601004FF4165070470000154B2DE979
:1092F800F04180460F4618680221FCF74BFA00241B
:109308002646781E84420F4D0DDA18F80410286896
:109318008E190134FCF71AFA40F6B830B6B2FCF7E9
:1093280083FAE4B2EDE7F1B22868FCF70FFA40F6E9
:10933800B830FCF779FA28680121BDE8F041FCF75C
:1093480029BA00BF2014002010B5084B084C197822
:109358002068FCF71FFA074920680968FCF710FA2B
:1093680020680421BDE8104000F0B8B9521400206C
:10937800201400201C14002013B5042000F07EF9EE
:10938800144C01462060A0B14279134B81681A70D1
:10939800124A11604FF49641FCF7F2F92068012156
:1093A800FCF7F8F92068042102B0BDE8104000F08D
:1093B80083B900904FF496420123042000F06CFA20
:1093C800054B42792060054980681A70086002B030
:1093D80010BD00BF20140020521400201C140020CF
:1093E800F8B5544C2068FCF7C1F9002800F0A180BA
:1093F8002068FCF7C0F905460520FCF720FA8A2DFD
:1094080021D08E2DEDD14C4C00212E22204605F086
:1094180001FA4A4A65707C2323701378E0207D2185
:10942800E07084F82C1014204FF4FA71A377237598
:1094380048227823207660766183628484F8243019
:1094480020462E2172E02020FFF716F80028C8D009
:109458003B4C00212C22204605F0DCF9A021E170CC
:10946800384B394965707C207D22207084F82B2088
:109478001878CA7AA076002A53D0344966250F682E
:1094880084F82950324D4968FE0F97FBF5FE667245
:10949800304E5FFA8EFE06FB0E720620424342F201
:1094A8001073B2FBF3FC03FB1C2791FBF5F5EDB23F
:1094B80027733F0A6773CF0F06FB051141436422E8
:1094C800B1FBF3F003FB101302FB05F151FA80F036
:1094D800010AE07320482174018863741B0A02FBA7
:1094E8000EFEA374B1FBF2F224235A4390B21B4A36
:1094F800E0711388A773010A2172180A18492075A8
:1095080018480A880188E3745EFA8CFC4FEA1C2E1E
:10951800130A84F80AC084F80BE06275A3752177F2
:1095280002E0202384F8293005482C21FFF7DEFECD
:1095380057E7F8BD2014002024140020C419002087
:10954800F0130020641F0020771F00204C1F00200C
:10955800A08601006079FEFF221F00202C1F00203A
:109568001E1F0020381F00204FF49640704700004F
:1095780010B500230C245C430549615C8142DAB2D2
:1095880003D00133042BF5D11A46104610BD00BF95
:10959800300000202DE9F84F0C2283460D46224862
:1095A800224B042105F0CCF900260C231E4A7343F4
:1095B80002EB030898F808101BEA010F2DD0D05CC5
:1095C80000241B4F2201BA46BB5C834203D00134FE
:1095D800E4B2042CF5D14FEA041940200AEB09073C
:1095E800FAF746FA20B91AF80910881E012814D982
:1095F8006B7B13B13A7B13420FD06968786881425C
:109608000BD3AA68BB689A4207D80A4804708760D7
:10961800C0F80480C560BDE8F88F0136042EC4D1B7
:109628000020BDE8F88F00BF3000002041960008F8
:10963800900C010854140020037A002023B15A1E0C
:1096480001301340C0B2F9E70A7A22B1511E013342
:109658000A40DBB2F9E7984294BF00200120704726
:1096680000230549595C8142DAB203D00133092B42
:10967800F7D11A4610467047850C010800220D4B99
:109688000C2101FB0233197A814211D00132D2B286
:10969800042AF4D10022074B0C2101FB0233197A6A
:1096A800014005D10132D2B2042AF4D108467047EC
:1096B800586870473000002010B50023064A0C2473
:1096C80004FB03225468844203D00133042BF5D1F0
:1096D8000022517210BD00BF300000200023074A4D
:1096E8000C2101FB03225168814203D00133042B72
:1096F800F5D1002200205072704700BF30000020D2
:1097080038B500220546110119484318405CA842A3
:1097180004D00132062AF6D1002038BD0FCB154CF3
:10972800042D84E80F0016D007D8012D0DD0022D86
:109738001BD111490B6898680AE0082D11D0202D1B
:1097480013D10D490B68D86802E00B4802685068CD
:109758006060A06003E0FFF75BFB6060A0602046EC
:1097680038BD2046FEF732FFF9E7024838BD00BF92
:10977800D00C01086414002084140020214B10B57B
:1097880018600120FFF7BCFF01460120FFF702FF28
:1097980008B9002010BD0220FFF7B2FF01460220E1
:1097A800FFF7F8FE0028F4D01020FFF7A9FF0146C4
:1097B8001020FFF7EFFE04464FF48070FAF758F9CF
:1097C80008B1002CE5D00820FFF79AFF01460820D1
:1097D800FFF7E0FE04460820FAF74AF908B1002C22
:1097E800D7D00420FFF78CFF01460420FFF7D2FEF4
:1097F80004464FF40060FAF73BF908B1002CC8D0D2
:10980800012010BD8414002010B50446FFF778FF2E
:1098180001462046FFF7BEFE003018BF012010BDEC
:1098280038B505460C46FFF76BFF01462846FFF79B
:10983800B1FE28B14368187A04420CBF0020012009
:1098480038BD0000F8B505460020FFF791FE104E20
:109858002B78104C0C27E15C07FB0060017201209B
:10986800FFF786FE07FB00626878235C022013720C
:10987800FFF77EFEAA7807FB0061A05C0872032050
:10988800FFF776FEEB7807FB0061E25C0A72F8BD31
:1098980030000020850C01082DE9FF47814603921E
:1098A8000C461E469DF83070FFF72AFF01464846D1
:1098B800FFF770FE039A054600282ED0836890F8BB
:1098C80000A093F80080B8F1030F26D8DFE808F06D
:1098D80002050D0F0097134801E013480097214631
:1098E8003346F8F739FB04460AE0002000E001207F
:1098F80021463B46F8F706FE31460446FBF74AFF89
:109908005CB184F80480696808484C6040F82A40D3
:1099180049462046FFF7D0FE00E00024204604B068
:10992800BDE8F0870038014000440040741400206E
:1099380038B5064C05462060FFF784FF284600F03E
:10994800FFFF2068BDE8384000F0E0BE8414002026
:10995800034B187808B100F0E1BD01F07BB800BFF7
:109968008814002010B504462046FBF70EFF18B9EE
:109978000A20FBF764FFF7E710BD0000232801D198
:1099880000F0CCBD044B19680A7D824202D1012047
:10999800FCF77CB8704700BF8414002010B5441E43
:1099A80014F8011F21B1034B1868FBF7CFFEF7E746
:1099B80010BD00BFC01400200148FFF7EFBF00BF73
:1099C800B80E010810B50748FFF7E8FF0024064B5A
:1099D8000648E1581A190C345268FAF7B3FBC02C40
:1099E800F5D110BDF60E0108D40D01080C0F0108C1
:1099F80070B5FBF713FF244C244B4FF47A71B0FB7E
:109A0800F1F11A7822482378FAF79CFBFEF74EFD0D
:109A180005462048204902682048B2FBF1F1FAF7D0
:109A280091FB00241E4B53F8241051B1012000FA79
:109A380004F0284202D01B48FAF784FB0134E4B250
:109A4800F0E70220FEF718FD68B1174A174B1178A6
:109A5800174853F82110FAF775FB1648017A11B127
:109A68001548FAF76FFB154C1548FFF797FF248840
:109A7800F7F728FE0246134821464FF46C73BDE8F9
:109A88007040FAF75FBB00BF02000020C419002035
:109A9800140F01086C01002040420F00520F01080A
:109AA8005C1D0108700F01088C0D0020940E010840
:109AB800740F0108641E00207E0F01085E0D00204F
:109AC800E4110108820F010838B50C6805462046E4
:109AD80005F0E6FD024628682146BDE8384005F055
:109AE8000FBE000037B5037904460D46052B34D860
:109AF800DFE803F003060A0D1114816809782DE0E8
:109B0800806890F9001029E08368198826E0826847
:109B1800B2F9001022E0816809681FE08068694690
:109B28000068FAF7F5FB01461148FAF70BFBF5B1A7
:109B3800E068F7F723F86946FAF7EAFB01460D48AB
:109B4800FAF700FB2069F7F719F86946FAF7E0FB1E
:109B580001460848FAF7F6FA09E000210648FAF73C
:109B6800F1FA25B10548E1682269FAF7EBFA3EBD3A
:109B78007B0F01087A0F0108B80F0108B40F01081C
:109B880008B50648FFF70AFF054B1868FFF7EAFE15
:109B98000020BDE80840FBF779BF00BFBB0F0108F4
:109BA800C014002008B50748FFF7F8FE064B93F8E5
:109BB800AC03F9F7FDFEF9F70BFFBDE80840FFF726
:109BC800DFBF00BFCA0F0108C81900207FB50446CF
:109BD80005F066FD082825D100231F49E25C0868C6
:109BE80085186E7806F00301022908BF203AE2546E
:109BF8000133082BF1D10025665D1848314605F080
:109C080073FC28B101356019314605F06DFC18B1B7
:109C18001348FFF7C3FE1DE0082DEDD1204611497A
:109C2800FEF734FE1048FFF7B9FE00230F4A9818D4
:109C380004A990F808218818084A995C0133082B70
:109C480000F80C1CF2D100208DF80C0001A908487E
:109C5800FAF778FA7FBD00BFA40100207C0C010848
:109C6800D40F0108D01A0020F40F0108C8190020E9
:109C78000F0F010808B5FDF791FC022801D0032851
:109C880004D10348BDE80840FFF788BE08BD00BFFF
:109C9800091001082DE9F041054605F001FD0446CB
:109CA800FAF720F9064694B92A48FFF777FE2A49B9
:109CB80051F8241049B1012202FA04F2324202D0CA
:109CC8002648FAF73FFA0134F1E7254821E028460B
:109CD8002449224605F014FD58B92348234CFFF7C0
:109CE8005DFE54F8041F0029EFD01C48FAF72AFA41
:109CF800F7E72B782D2B04D10135013C4FF00108F3
:109D080001E04FF000080026134850F8267027B9E4
:109D18001748BDE8F041FFF741BE284639462246BC
:109D280005F0EEFCA0B9012000FA06F0B8F1000F2A
:109D380003D0FAF721F80F4802E0F9F7A3FE0E481E
:109D4800FFF72CFE0D483946BDE8F041FAF7FAB99D
:109D58000136D9E72F100108300D0108700F0108EE
:109D6800E4110108411B0108421001082C0D0108EB
:109D780057100108711001087B1001080F0F010826
:109D880010B504460848FFF709FE084A084809497B
:109D98000023036013700B70FCF74CFD2046BDE8F0
:109DA8001040FFF7FFBE00BF84100108891400208F
:109DB800BC1400208814002008B50448FFF7EEFD05
:109DC800F9F768FEBDE80840FFF7DABE9C10010805
:109DD8002DE9F04389B0044605F062FCC6B2002EB6
:109DE8006AD17A487A4CFFF7D9FD20690021F7F744
:109DF800ADF838BB013677483146FAF7A3F9206940
:109E080004A9FAF785FA01467348FAF79BF96069DD
:109E180004A9FAF77DFA01466F48FAF793F9A069A1
:109E280004A9FAF775FA01466B48FAF78BF9E06965
:109E380004A9FAF76DFA01466848FAF783F910346D
:109E48000C2ED2D10025664C2F46A8464FF00009AB
:109E58001034B14514DA404654F8101CF6F7DAFD10
:109E680054F80C1C80462846F6F7D4FD54F8081C14
:109E780005463846F6F7CEFD09F101090746E7E73A
:109E88005848CDF8048002950397FFF787FD002412
:109E980001A85549235823F00040F7F77FF85349A4
:109EA800534A0434002814BF10460846FFF776FDCD
:109EB8000C2CEDD14F4871E020464F49052205F0A2
:109EC8001FFC38B9424BC11810300022C0280A6163
:109ED800F8D177E020464949042205F011FC0546EF
:109EE80020460DBB202105F0FFFA00286AD0461C49
:109EF800304605F0D5FB2C460746414850F824501B
:109F08000DB940484AE030462946FAB205F0F8FB58
:109F180040B920463C49FCF729FD3C482946FAF758
:109F280011F947E00134E8E704F080FB461E0B2EE8
:109F3800074643DC2046202105F0D6FA054640B105
:109F4800451C2846FAF74CFA3F01214B0124D85109
:109F580000E004462846202105F0C6FA054640B12F
:109F6800451C2846FAF73CFA194901EB0612013458
:109F780050612846202105F0B7FA054640B1451C36
:109F88002846FAF72DFA124B03EB061101348861C3
:109F98002846202105F0A8FA18B91D48FFF7FEFC4D
:109FA80010E00130FAF71CFA094A02EB0616032CF6
:109FB800F061F2D11748FFF70BFF03E016480C21B8
:109FC800FAF7C0F809B0BDE8F08300BFBD1001087A
:109FD800C8190020E8100108EE1001080F0F010849
:109FE800DC190020F21001080AD7233CB910010837
:109FF800B5100108E4110108011101080711010851
:10A00800780D01080C110108D81900202411010845
:10A01800371101082314010871110108F8B5074622
:10A0280005F03EFB044638B91A491B4B4A791B48D0
:10A03800511E53F8211028E038461949224605F0E8
:10A048005FFB60B91748184CFFF7A8FC54F8041FC9
:10A0580019B11648FAF776F8F8E7154805E000252B
:10A068000D4B53F8256026B91248BDE8F840FFF7B4
:10A0780095BC38463146224605F042FB013500289A
:10A08800EED1044845710C483146BDE8F840FAF76E
:10A0980059B800BFC8190020780D010899110108A6
:10A0A800411B0108AD110108740D0108700F01086A
:10A0B800E41101080C110108C01101082DE9F0474D
:10A0C800064605F0EDFA054620B1012819D1337886
:10A0D8002A2B16D14748FFF761FC00241426664353
:10A0E800454F4648F159FAF72DF8B8192946FFF7B0
:10A0F800F9FC01344248FFF751FC732CEED1BDE85E
:10A10800F08730463D2105F0EFF9002857D0441C70
:10A11800204604F08BFA82462046FAF761F90027B8
:10A1280005461424DFF8D0907C4354F80980404653
:10A1380005F0B6FA41460246304605F0E1FA002835
:10A1480035D14C44E068F6F719FD01462846F6F784
:10A158001BFF002829D02069F6F710FD0146284684
:10A16800F6F708FF002820D020792279052818BFA3
:10A178005546052A0FD8DFE802F003030606090C46
:10A18800A1680D7007E0A268158004E0A06805606A
:10A1980001E0A1680D6041461A48F9F7D3FF20464F
:10A1A8000021BDE8F047FFF79DBC174803E00137E1
:10A1B800732FB6D11548BDE8F047FFF7EFBB04464B
:10A1C80014250D4F6543314655F80780404605F084
:10A1D80079FD50B109484146F9F7B4FF78190021D3
:10A1E800FFF780FC0648F9F7ADFF0134732CE7D17F
:10A1F800BDE8F087D21101087C1D0108AC130108E5
:10A20800E4110108E7110108F21101081712010809
:10A2180010B50446204605F043FA10F0FF0F07D1A9
:10A228000B490C4891F8AC13BDE81040F9F78ABF08
:10A23800204604F0FBF9022808D8054B064C83F8A1
:10A24800AC03F9F7C5FBF9F709FEE3E710BD00BF5A
:10A25800C8190020341201082314010870B50446F7
:10A2680005F01EFA08B9204830E020461F4905F0DD
:10A27800A1FE00242646254678B12CB1012C06D132
:10A2880004F0D4F9064602E004F0D0F905460020AF
:10A298001649013405F08EFEEEE70B2D05D914485A
:10A2A8000C21BDE87040F9F74DBF012C08DC114ABC
:10A2B800114832F915202946BDE87040F9F742BF28
:10A2C800A6F57A73B3F57A7F04D90C48BDE87040D7
:10A2D800F9F738BF0A4829463246F9F733FF0548E7
:10A2E80020F8156070BD00BF4A120108ED1301087F
:10A2F80084120108F41E0020AA120108C2120108E3
:10A30800E412010838B5054605F0CAF9C0B268B9C3
:10A3180004461249124801EB44022146B2F846208D
:10A328000134F9F70FFF152CF3D138BD284604F096
:10A338007DF9142804460BDC2021284605F0D4F8C2
:10A3480004F074F9054B03EB4404A4F8460038BD47
:10A3580004481521BDE83840F9F7F4BE7C1D0020FB
:10A36800FD120108091301082DE9F0435848594C1A
:10A3780085B0F9F7E7FE5848FFF7C4FF6279574BF5
:10A388005748511E53F82110F9F7DCFE20690021C7
:10A39800F6F7DCFD002858D1002526690021304653
:10A3A800F6F7D4FD00284CD101354E48D4F8149066
:10A3B800D4F81880E7692946F9F7C4FE3046002129
:10A3C800F6F7CEFD10B14848F9F7BCFE69463046AD
:10A3D800F9F79EFF01464548F9F7B4FE48460021C3
:10A3E800F6F7BEFD10B14048F9F7ACFE694648469D
:10A3F800F9F78EFF01463D48F9F7A4FE40460021D3
:10A40800F6F7AEFD10B13848F9F79CFE69464046AC
:10A41800F9F77EFF01463548F9F794FE38460021E2
:10A42800F6F79EFD10B13048F9F78CFE69463846BC
:10A43800F9F76EFF01462E48F9F784FE10340C2D0B
:10A44800ABD12C48691CF9F77DFEF9F74BFD2A4C76
:10A45800064654F8041F19B12848F9F773FEF8E7BF
:10A468000D46274850F8251049B1012202FA05F295
:10A47800324202D02348F9F765FE0135F1E7154B62
:10A48800214ACE1804A896F808418B5C05190131B9
:10A49800082905F8103CF2D100241C488DF8084022
:10A4A8006946F9F74FFE14256543194E1948A9590D
:10A4B800F9F748FE00217019FFF714FB013416481C
:10A4C800FFF76CFA732CEED105B0BDE8F08300BF3E
:10A4D8002F130108C819002023140108780D01085A
:10A4E8005F1301086A130108ED1301087B0F0108C7
:10A4F8000F0F0108721301082C0D010884130108BD
:10A50800300D0108921301087C0C01089F13010803
:10A518007C1D0108A8130108E4110108F0B56D4B72
:10A528001A7887B07AB96C4C01201870022120681B
:10A53800FFF7C2F82068F9F72FFE6848FFF72EFAF0
:10A548006748FFF72BFA644C2068FBF70FF90028DF
:10A5580000F0BD802068FBF70EF909280146614A22
:10A5680001D03F2851D1002517685F4C2E462FB1E6
:10A578005E4821683A4605F0C3F810B9254606B981
:10A5880026465B490C348C42F1D3C6B13468D5F801
:10A5980000E03B46E05C1EF8031081420DD1534AAF
:10A5A80041B92D2B06D82024D4544E4801330360DA
:10A5B800D15404E0D0540133ECE74A490B60494ACE
:10A5C80014681CB1AE4201D13C4612E04948FFF77D
:10A5D800E5F9AE4209D856F80C0BFFF7DFF93E4B08
:10A5E80009211868FBF7B2F8F3E73D48FFF7D6F9F9
:10A5F80000243C4B18688442A5D237493B4A086876
:10A60800115DFBF7A3F80134F3E713682BB90428AD
:10A6180038D13648FFF7B4FB59E00C2801D1364849
:10A628008CE70A2901D00D2948D12E4D33482F4CEB
:10A63800FFF7B4F92A6832482B4903940023A3543E
:10A6480004930090102203A80C2303F0F3FF05469F
:10A6580038B1006805F024F8411CAA6860189047D2
:10A6680002E02848FFF79AF9002130221F4804F039
:10A67800D1F818491B4B0A7800201860002A7FF48B
:10A688005FAF24E00C28CAD07F2903D15BE72F2BCA
:10A698003FF659AF1F297FF656AF7E293FF653AFD5
:10A6A80013B920293FF44FAF104C0B4AE154581C02
:10A6B8000C4B18601068FBF749F844E77F29E6D18E
:10A6C800581E0A4C1060002121540F4839E707B082
:10A6D800F0BD00BF88140020C0140020B213010888
:10A6E800EA130108BC140020D40D010889140020C5
:10A6F800940E0108EF130108F4130108E41101088E
:10A70800D19A0008FF1301082014010837B505463F
:10A718000220FEF7B3FF064C0146206030B90090D6
:10A72800AA6802200323FFF7B7F820603EBD00BFE8
:10A73800C0140020F8B5174E174C184D0746C1B283
:10A7480030682170FBF702F822782B7882EA030040
:10A75800C7F30721287030682170FAF7F7FF2178CE
:10A768002A78306881EA0203C7F307412B70217009
:10A77800FAF7ECFF2078297880EA0102390E306870
:10A7880021702A70FAF7E2FF2B78207880EA03011B
:10A798002970F8BDC8140020CE140020C41400206D
:10A7A800F8B50D4E0D4D0E4CC1B2074630682970F4
:10A7B800FAF7CCFF2A782378391282EA030020704E
:10A7C80029703068C9B2FAF7C1FF23782A7882EA7B
:10A7D80003002070F8BD00BFC8140020CD1400206D
:10A7E800C4140020054B10B5044621461868FAF732
:10A7F800ADFF034802785440047010BDC81400200F
:10A80800C4140020034B04491A78885C01321A707A
:10A81800704700BFC5140020E514002010B5FFF7ED
:10A82800F1FF0446FFF7EEFF04EB002080B210BDF5
:10A8380010B5FFF7F3FF0446FFF7F0FF04EB004005
:10A8480010BD000038B5044624200D46FFF7CAFFA6
:10A858004D20FFF7C7FF002C0CBF3E202120FFF73B
:10A86800C1FF064B002228461A70FFF7BBFF0448B9
:10A878000078BDE83840FFF7B5BF00BFC41400201A
:10A888002515002001460020FFF7DCBF0146012006
:10A89800FFF7D8BF014B1878FFF7A4BFC4140020F6
:10A8A80070B5054608460E46FFF7ECFF2C467219B0
:10A8B800D0B2E3B2984204D014F8010BFFF792FF2C
:10A8C800F5E770BD10B5441E14F8010F10B1FFF77D
:10A8D80089FFF9E710BD00002DE9F843002701249E
:10A8E8000025144B187885421CDA1349134B15F8C8
:10A8F80001800C2202FB0830406804F0D1FE81463A
:10A908000CB13F180CE026464E4509DA0B4A0C21DB
:10A9180001FB08235868805DFFF764FF0136F3E701
:10A928000135DEE724B1F8B2FFF7ACFF0024D7E722
:10A93800BDE8F883C6140020CF1400206000002072
:10A94800F7B5404DFF2115220746284603F062FF60
:10A95800002302202B70FDF78FFD012418B102207F
:10A968006C70A87003240420FDF786FD68B1354E8D
:10A9780003214FF400503155651CF9F779F818B1E7
:10A9880004227255023400E02C460220FDF774FDC3
:10A9980048B12C4B1E190520062107251855717042
:10A9A800B570033404E00820FDF766FD0028F0D1F7
:10A9B8002020F9F75DF818B1224B08221A55013406
:10A9C8004FF48070F9F754F830B11E4801190A267F
:10A9D8000B2506554D7002341B4A1A4B507908282E
:10A9E80001D00E2802D10C261E5501340D21042059
:10A9F8001955651CF9F73CF818B11248112242554F
:10AA0800A51C11490F4E91F8392113236C1C101CF9
:10AA180018BF01207355F9F72BF810B114203055E1
:10AA2800AC1C0A4B01201C70FEF728FE084C01469E
:10AA3800206030B900907A6801200323FEF72CFFCC
:10AA48002060FEBDCF140020C8190020C6140020C5
:10AA5800C8140020F8B5B54C2068FAF787FE00281E
:10AA680000F039852068FAF786FEB14A1178034666
:10AA780071B9B0F124014B4253EB01041470002C5E
:10AA8800E9D1AC4A51780029E5D1FEF777FFE2E732
:10AA9800012904D14D280CBF0223002321E00229FB
:10AAA80004D13C280CBF032300231AE003290FD14B
:10AAB80040284FF0000401D91470CCE79E489F4904
:10AAC80003709F480C7004709E4C2370042308E0A8
:10AAD800042908D19B4C9C48217803704B40237073
:10AAE80005231370B7E70529B5D19448924C01782E
:10AAF80022788A42934A07D914785C401470934AA2
:10AB0800535401310170A6E71078984240F0DE8472
:10AB18008D4B19787B2900F01B8300F2C5806E29C4
:10AB280000F06D8360D8682900F02E8325D8652948
:10AB380000F0028219D8642940F0C3840720844CAD
:10AB4800FFF7A0FEE620FFF74DFE6079FFF74AFE0B
:10AB58000020FFF747FE94F81B017E4B7E4A002831
:10AB68000CBF1046184600F05DBC662900F06282F2
:10AB7800672940F0A684794807E36B2900F01D8314
:10AB880023D8692900F005836A2940F09A841020A7
:10AB9800FFF778FE6748724CC07AFFF723FE7149C9
:10ABA8000878FFF71FFE2068FFF7C4FD6068FFF70D
:10ABB800C1FD6D4AB2F90000FFF7F2FD6B4BB3F926
:10ABC8000000FFF7EDFD6A4A16E36C2900F00783E1
:10ABD8006D2940F076840620FFF754FE6549086821
:10ABE800FFF7A8FD644A07E3732900F075833CD892
:10ABF800702900F03383C0F01383712900F041837A
:10AC0800722940F05E84524C5C4D1620FFF73AFEE4
:10AC18000020FFF7C5FDB4F9D000FFF7C1FDB4F976
:10AC2800D200FFF7BDFDB4F9D400FFF7B9FDB5F9BF
:10AC3800BA00FFF7B5FD0020FFF7B2FD0020FFF7CF
:10AC480079FDB5F928000A2390FBF3F0FFF7A8FD7A
:10AC580094F80401FFF7C6FD94F80601FFF7C2FD5A
:10AC680094F80501FFF7BEFD65E3762900F03F8300
:10AC78000DD8742900F01D83752940F022842F20F7
:10AC8800FFF700FE3E48FFF71DFE00F01DBC7729C8
:10AC980000F01283782940F01484384C3820FFF7EC
:10ACA800F1FD04F1400503E2D02900F0798300F2B8
:10ACB800C680CA2900F0018168D8A42900F0E08381
:10ACC80010D8A02940F0FD832E4C0C20FFF7DAFDA8
:10ACD8002068FFF72FFD4FF080510868FFF72AFD25
:10ACE80020689FE3C82900F0DA80C92940F0E98389
:10ACF800FFF788FD0F4A1A4CD072FFF783FD194BF6
:10AD08001870FFF795FD2060FFF792FD6060FFF770
:10AD180085FD15490880FFF781FD144A10801A48FF
:10AD2800037843F002040470D6E000BFC814002082
:10AD3800CC140020771F0020E4140020C714002042
:10AD4800C5140020C414002025150020E514002097
:10AD5800C81900201C000080140000801800002082
:10AD68004C1F0020641F00201E1F0020221F0020EF
:10AD7800FC100020BC1E0020840E00207C1D00203A
:10AD8800782601080300001032110020CD2900F0B8
:10AD9800118322D8CB2900F0A180CC2940F09183DF
:10ADA800FFF730FDCC4CE077FFF72CFD84F820004E
:10ADB800FFF728FD84F82300FFF724FD84F824001A
:10ADC800FFF720FD84F82500FFF71CFD84F821001B
:10ADD800FFF718FD84F822007EE0CE2900F0F48207
:10ADE800CF2940F06E83FFF719FDFFF717FDBB4C25
:10ADF800B94DA4F8D000FFF711FDA4F8D200FFF771
:10AE08000DFDA4F8D400FFF709FDA5F8BA00FFF777
:10AE180005FDFFF70DFDFFF701FD0A2250432885C8
:10AE2800FFF7F0FC84F80401FFF7ECFC84F8060156
:10AE3800FFF7E8FC84F80501FFF7E4FC4CE0D529AE
:10AE480000F094810FD8D22961D0C0F07882D3293C
:10AE58006DD0D42940F035839F4C0020FFF712FDB8
:10AE680004F1400556E1F02900F0CF820CD8D6292C
:10AE780044D0EF2940F02583FFF7D0FC964CA085FD
:10AE8800FFF7CCFC608527E0FA2900F0A582FE29AF
:10AE980040F017830820FFF7F5FC0024ADE20024FA
:10AEA800FFF7BCFC8E4908530234102CF8D100205F
:10AEB800FFF7E8FCFDF704FD06E38A4C04F10A05F8
:10AEC800FFF7A0FC01346070FFF79CFCE072FFF70D
:10AED80099FCAC426075F3D100208BE200248248D3
:10AEE80003789C42F8D2814D655DFFF797FC7A495B
:10AEF80001EB45050134A5F84600F0E70024FFF70B
:10AF08008DFC7B4908530234102CF8D1E4E7794CC6
:10AF18006478002CE0D1FFF775FC704B022883F8A9
:10AF2800AC0388BF83F8AC43F8F752FD3FE2FFF764
:10AF380075FC714A1080CFE7704D0B20FFF7A2FC1B
:10AF4800B5F90000FFF72CFCF6F7BCFB00B2FFF7E1
:10AF580027FC0220FDF790FA05460420FDF78CFA3D
:10AF680004460820FDF788FA820042EA4401294392
:10AF780020208CB2FDF780FA44EAC00084B2102089
:10AF8800FDF77AFA44EA001318B2FFF709FC594AA8
:10AF98001079D1785378840044EA410190791943B3
:10AFA80041EAC0045179537A44EA411040EA8314D3
:10AFB8005348C17944EAC113047A417A43EA042325
:10AFC80043EA4124D379117A927A44EA832444EA01
:10AFD800C123417B43EA0234827B44EA4133017C4A
:10AFE80043EA8234027944EA0143417C43EA021489
:10AFF800827C44EA4143C17C007D43EA824444EABE
:10B00800C142394B42EA00540020197803468B426A
:10B018000AD2364D5D5D012202FA05F525421CBFB4
:10B028009A4010430133F2E72C4CFFF783FB94F866
:10B03800AC0381E11220FFF725FC32490C88B4F5F6
:10B04800806F314CB4F9000008D8FFF7A9FBB4F9B8
:10B058000200FFF7A5FBB4F904000EE0082590FBF9
:10B06800F5F0FFF79DFBB4F9020090FBF5F0FFF750
:10B0780097FBB4F9043093FBF5F0244CFFF790FBF1
:10B08800B4F90000FFF78CFBB4F90200FFF788FB66
:10B09800B4F904001E4CFFF783FBB4F90000FFF776
:10B0A8007FFBB4F90200FFF77BFBB4F90400B6E1BB
:10B0B800B4F97800FFF774FBB4F97A00FFF770FB76
:10B0C800B4F97C00FFF76CFB94F87E000834FFF7B6
:10B0D80089FBAC42ECD1F7E17C1D0020C8190020A7
:10B0E800CE1F00207B1D0020C6140020CF14002096
:10B0F800F41E0020771F0020881E00205E0D00200F
:10B10800881F002004000020C41E0020700E0020AC
:10B11800701E0020FFF782FBA4F87800FFF77EFB83
:10B12800A4F87A00FFF77AFBA0F57A73072899B29A
:10B1380098BF84F87F00B1F57A7F98BFA4F87C00A7
:10B14800FFF760FB84F87E000834AC42E2D1BBE133
:10B158000820FFF797FB0024B4496218083492F8D6
:10B168007F00FFF73FFB402CF6D1ADE10020FFF751
:10B1780089FB0024FFF746FBAC4962180834402CD1
:10B1880082F87F00F6D19FE1A9481021FFF788FBDC
:10B198009AE1A84801784C0004F0FE00FFF772FB22
:10B1A8000024A44A13789C4280F08E81A24830F98A
:10B1B8001400FFF7F5FA0134F3E70520FFF762FB07
:10B1C8009E4BB3F90000FFF7EBFA9D48B0F9000079
:10B1D800FFF7E6FA9B490A7802F00100ACE09A4CC6
:10B1E8000620FFF74FFBB4F90000FFF7D9FAB4F9CE
:10B1F8000200FFF7D5FA954AB2F900000FE10720DF
:10B20800FFF740FB92480078FFF7ECFA0020FFF7C1
:10B21800C7FA904BB3F90000FFF7C2FA0020FEE02E
:10B22800824C0720FFF72EFBE07FFFF7DBFA94F84C
:10B238002000FFF7D7FA94F82300FFF7D3FA94F821
:10B248002400FFF7CFFA94F82500FFF7CBFA94F81B
:10B258002100FFF7C7FA94F822006DE01E207E4C0B
:10B26800FFF710FB04F10A0501346078FFF7BAFA1A
:10B27800E07AFFF7B7FA607DFFF7B4FAAC42F3D192
:10B2880022E176490A78540004F0FE00FFF7FAFA42
:10B298000024724803789C4280F016817049634804
:10B2A800625C00EB42030134B3F94600FFF778FA19
:10B2B800EFE7FFF711FB07E168490878FFF7E2FAC3
:10B2C8000024664A1078844280F0FE80644B185D42
:10B2D800FFF788FA0134F4E70820FFF7D3FA0124CE
:10B2E800E0B20134FFF77EFA092CF9D1ECE0FFF760
:10B2F80089FA06461220FFF7C5FA0EB9594902E045
:10B30800102E03D158490D684C6801E000242546E9
:10B318003046FFF767FA2846FFF70CFA2046FFF792
:10B3280009FA524A1068FFF705FA0020FFF738FAC1
:10B338000020FFF735FA0020FFF754FAC4E0FFF7C2
:10B3480061FA0546FFF774FA0746FFF771FA0646F1
:10B35800FFF76EFA0446FFF761FAFFF75FFAFFF7A7
:10B3680051FA65B93F48424B076001214660DD71DB
:10B378001973002C3FF4B0AD3C4A1460ACE5102DB5
:10B388007FF4AAAD3848076046600CB1374B1C60A3
:10B39800384A354802211170011DFCF755F99BE523
:10B3A80033484378002B7FF497ADF8F773FBF8F731
:10B3B80055FD91E52E4C6278002A7FF48DAD4FF44F
:10B3C800C870F9F743FF87E529484378002B7FF4D5
:10B3D80083AD012181737FE5254A5478002C70D113
:10B3E800254B93F8AC03F8F7E3FAF8F7F1FAF8F716
:10B3F80035FD2046FFF746FA66E02048005F023434
:10B40800FFF7CEF9082CF8D15EE0084C0420FFF7CE
:10B4180039FAB4F92C00FFF7C3F9B4F92A00FFF799
:10B42800BFF951E0FFF786F94EE000BF7C1D002010
:10B43800DC1E0020CC1F0020CE1F00202C1F002067
:10B44800381F002032110020600E00209A1E0020B4
:10B45800C41900205E1E00207B1D0020C614002099
:10B46800CF140020301F0020241F0020C01E002001
:10B47800771F0020BC100020C8190020561E00208D
:10B48800154C22789000431CD8B2FFF7FBF92078BE
:10B49800FFF7A8F9002410490A78944214D20F48FB
:10B4A800005DFFF79FF90E4B185DFFF79BF90D49FB
:10B4B800085DFFF797F90C4A105DFFF793F901341F
:10B4C800E9E70020FFF7E2F9FFF7E4F9074B00206E
:10B4D8001870FFF7C0BAF8BD651F00200C1F0020C8
:10B4E8003A1F0020541F0020661F0020CC140020A3
:10B4F8002DE9F0410746884616460024B4421AD082
:10B508000025BD4211D00D4B9A8A90B280F4885123
:10B5180099820120FAF74EF94046FAF790F9013579
:10B528000020FAF747F9EDB2EBE73C200134FAF7CF
:10B5380086F9E4B2E2E7BDE8F08100BF00100048F8
:10B54800F0B500230E681A46012505FA02F505EA4A
:10B558000604AC4232D10D796F1E012F1BD88768C3
:10B568004FF0030C0CFA03FC27EA0C07876091F8EC
:10B5780005C087680CFA03FC4CEA070787608788D0
:10B58800BFB227EA040484808C79878804FA02F41D
:10B598003C43A7B287800324076804FA03F4E44312
:10B5A80027400760076805FA03F53D430560C5684D
:10B5B8002C40CD7905FA03F52C43C46001320233DF
:10B5C800102AC1D1F0BD00214FF6FF73022203609B
:10B5D800017142718171C171704781617047018544
:10B5E800704701F00703C908083130B59B0050F8CF
:10B5F80021500F2404FA03F425EA040440F82140FA
:10B6080050F8214002FA03F2144340F8214030BDBB
:10B61800124B1A6842F0010018605968104A0A4033
:10B628005A60186820F0847121F480321A60186812
:10B6380020F4802119605A6822F4FE005860D96A03
:10B6480021F00F02DA62186B0649002201401963E3
:10B658009A60054B4FF000609860704700100240F8
:10B668000CC07FF8CCFC00FF00ED00E082B00023A6
:10B67800254800930193026842F480310160224B0F
:10B68800186800F4003201920099481C0090019A51
:10B698001AB90099B1F5A04FF1D11B6813F4003025
:10B6A80018BF01200190019A012A2AD1174B1221B3
:10B6B800A3F5805019604268426041684160436860
:10B6C80043F480624260416821F47C13436042681D
:10B6D80042F4E8114160036843F080720260016837
:10B6E800094A8901FBD5506820F00303536051686B
:10B6F80041F002005060044A536803F00C01082925
:10B70800F9D102B0704700BF00100240002002408B
:10B71800A44B5A6802F00C02042A2DE9F04305D024
:10B72800082A06D0A0490160B2B916E09E4C046010
:10B7380012E05D685C68C5F38346B71CE20301D478
:10B748009A4A06E0DB6A984D03F00F02511CB5FBDC
:10B75800F1F27A43026000E00022924F944D7E6835
:10B76800C6F30313EC5C036823FA04F141607E68B6
:10B77800C6F30226AE5D21FA06F68660D7F804C045
:10B78800CCF3C228DFF82CC215F8085021FA05F1CD
:10B79800C160D7F82C90C9F3041808F00F0918F005
:10B7A800100F3CF819C01FFA8CFC07D0BCF1000F31
:10B7B80004D0B2FBFCF8C0F8108000E00361FF6A17
:10B7C800C7F3442C0CF00F087A4F37F818701CF0A8
:10B7D800100FBFB204D01FB1B2FBF7F7476100E00A
:10B7E8004361704FD7F830C01CF0100F0ABFDFF864
:10B7F800B8C18361C0F818C03F6BBF0656BF6A4F17
:10B80800C361C761674FD7F830C01CF0400F0ABF4B
:10B81800DFF894C10362C0F820C03F6BFF0506D56E
:10B82800934204D1A54202D15F00476200E0416221
:10B838005C4FD7F830C01CF4805F08D0934206D123
:10B84800A54204D14FEA430CC0F828C000E0816249
:10B858003F6BBF0506D5934204D1A54202D15F00D4
:10B86800C76200E0C1624F4FD7F830C01CF4806F48
:10B8780008D0934206D1A54204D14FEA430CC0F840
:10B8880044C000E041643F6B3F0506D5934204D1B4
:10B89800A54202D15F00876400E08164414FD7F878
:10B8A80030C01CF4005F06D0934204D1A54202D1F7
:10B8B8005A00C26400E081643C6B3A4A14F0030FFA
:10B8C80001D1016315E0116B01F00301012901D1D8
:10B8D80003630EE0116B01F00301022902D14FF45A
:10B8E800004205E0126B02F00301032901D12E4A40
:10B8F80002632C4A116B11F4403F01D1466318E0F2
:10B90800116B01F44031B1F5803F01D1436310E080
:10B91800116B01F44031B1F5003F02D14FF4004101
:10B9280006E0116B01F44031B1F5403F01D11E49E9
:10B938004163126B1B4912F4402F01D1866318E052
:10B948000A6B02F44022B2F5802F01D1836310E024
:10B958000A6B02F44022B2F5002F02D14FF40041E5
:10B9680006E0096B01F44022B2F5402F01D10E49DF
:10B9780081630C4A116B11F4401F01D1C66323E0A7
:10B98800116B01F44011B1F5801F01D1C3631BE0B5
:10B99800116B01F44011B1F5001F0DD14FF40041B6
:10B9A80011E000BF0010024000127A0000093D00BB
:10B9B8009001002070010020116B01F44011B1F5D5
:10B9C800401F01D11149C163126B114912F4400F94
:10B9D80002D10664BDE8F0830A6B02F44002B2F5B6
:10B9E800800F0FD00B6B03F44002B2F5000F02D1A9
:10B9F8004FF4004306E0096B01F44003B3F5400F30
:10BA080001D1024B0364BDE8F08300BF00127A0045
:10BA180000100240030F064BDA6A14BF22F4785272
:10BA280022F4F872DA62D96A0843D862704700BF14
:10BA380000100240020F012A0A4B0AD005D3022A3D
:10BA48000BD1196B21F0400206E0196B21F01002AE
:10BA580002E01A6B22F020021A63196B084318637C
:10BA6800704700BF00100240044B5A6909B11043E7
:10BA780001E022EA00005861704700BF0010024050
:10BA8800044B9A6909B1104301E022EA0000986169
:10BA9800704700BF00100240044BDA6909B1104337
:10BAA80001E022EA0000D861704700BF00100240A0
:10BAB800044BDA6809B1104301E022EA0000D860BB
:10BAC800704700BF00100240044B1A6909B11043C7
:10BAD80001E022EA00001861704700BF0010024030
:10BAE800024B5A6A42F08070586270470010024058
:10BAF80008B5154B98420BD101214FF48050FFF740
:10BB0800D7FF4FF480500021BDE80840FFF7D0BFB1
:10BB18000E49884207D14FF480400121FFF7D4FF36
:10BB28004FF4804009E00A4A90420BD14FF400409C
:10BB38000121FFF7C9FF4FF400400021BDE808408C
:10BB4800FFF7C2BF08BD00BF003001400038004009
:10BB5800003C00404A88B2F5827F30B51BD104888A
:10BB6800CB8804F441520C881C4344F482730C893A
:10BB780023434C8923438C892343CC8923431A4389
:10BB880093B20380828822F470631A04130C8A88A3
:10BB98001343838019E0838823F4706425048C8818
:10BBA8002B0C234383800B8805881343CA8805F42C
:10BBB80041540D8913434A892B438D891343CA89FC
:10BBC8002B43134323439AB20280838B098A23F4BD
:10BBD800006213041A0C8283018230BD038819B1F4
:10BBE80099B241F0400303E023F040010A04130C2A
:10BBF80003807047838823F4805213041A0C8280D0
:10BC080083889AB21143818070470173704781819C
:10BC18007047007B7047808980B27047038919425A
:10BC28000CBF002001207047C2680D4B10B51340AF
:10BC380091E8140014438A681443CA6814430A69D3
:10BC480014434A6914438A6922431343C360026B4D
:10BC5800097F22F00F024B1E1343036310BD00BF80
:10BC680007C0FFFD00230121036043608360C360B8
:10BC7800036143618361017770470000B0F1A04F11
:10BC880010B502D0104B984201D1104A00E0104A7A
:10BC98009468104B234091E8140014438A681443B5
:10BCA800CA68097C44EA023242EA0122B0F1A04F94
:10BCB80042EA030302D00449884201D1034800E064
:10BCC8000348836010BD00BF00010050000300500E
:10BCD80000070050E010FCFF00230360436083600E
:10BCE800C36003747047836811B143F0010101E038
:10BCF80043F0020181607047836843F0004181602E
:10BD08007047836823F080428260836819438160AA
:10BD180070478068C00F7047836823F04052826084
:10BD2800836811B143F0805101E043F00051816014
:10BD38007047042A30B514B20DD86200E400A41A82
:10BD4800056B1F2202FA04F225EA020201FA04F442
:10BD5800224302632FE0092A0ED86200E400A41AE5
:10BD6800456B1E3C1F2202FA04F225EA020201FA80
:10BD780004F4224342631EE00E2A0ED86200E40057
:10BD8800A41A856B3C3C1F2202FA04F225EA02023F
:10BD980001FA04F4224382630DE06200E400A41A6D
:10BDA800C56B5A3C1F2202FA04F225EA020201FA84
:10BDB80004F42243C263092910D901EB41018269C5
:10BDC80084691E39072202FA01F224EA020282611A
:10BDD800826903FA01F31343836130BD4269446900
:10BDE8004A1E03256A43382505FA02F224EA0202AC
:10BDF8004261426901EB410103FA01F313434361D4
:10BE080030BD836843F0040181607047C36811B195
:10BE180043F0010101E023F00101C1607047C368EC
:10BE280023F00202C260C3681943C1607047036807
:10BE380019420CBF00200120704730B5046A24F075
:10BE4800010505628569046A25F0F3052A4342EA7B
:10BE5800031341F0010124F00A0241EA020483615C
:10BE6800046230BD30B5056A4FF6EF742C400462A9
:10BE78008469056A24F4734444EA0222090142EA07
:10BE880003334FF65F7441F010022C4091B20C431B
:10BE98008361046230BD0000204A038890429BB24F
:10BEA8000ED002F5006290420AD0B0F1804F07D060
:10BEB800A2F59832904203D002F58062904203D1F5
:10BEC8004A8823F070031343154A904208D002F5BC
:10BED8008062904204D023F440730A899BB21343D2
:10BEE80003804B680A88C3620C4B028598420FD0C6
:10BEF80003F5006290420BD002F54063984207D0E8
:10BF080003F58062904203D002F58063984201D124
:10BF18004989018601224261704700BF002C014017
:10BF28000010004000214FF0FF3343600180018181
:10BF380041804181704741627047038819B199B2C5
:10BF480041F0010303E023F001010A04130C03800C
:10BF580070470000036A23F001020262036A426824
:10BF680030B5856925F4803424F073050C682C43BA
:10BF78008D8923F002032B438D882B43134DA84250
:10BF88000FD005F50065A8420BD005F54065A8421D
:10BF980007D005F58065A84203D005F58065A8425D
:10BFA8000DD1CD8923F008032B43CD8823F004035A
:10BFB8002B430D8A22F440722A434D8A2A4389680A
:10BFC800426084614163036230BD00BF002C0140C0
:10BFD800036A23F01002026270B5056A4268846938
:10BFE80024F080760C6826F4E64343EA04248E891C
:10BFF8008B8825F02005334345EA03130E4DA842EC
:10C0080003D005F50065A84210D123F08006CB893E
:10C0180046EA0315CB8825F0400646EA03134D8A05
:10C028000E8A22F44062354342EA850289684260FA
:10C0380084618163036270BD002C0140036A23F4AC
:10C048008072026270B5056A4268C4690B6824F0A0
:10C05800730646EA03048E898B8825F400753343FA
:10C0680045EA03230E4DA84203D005F50065A84212
:10C0780010D123F40066CB8946EA0325CB8825F442
:10C08800806646EA03234D8A0E8A22F440523543DD
:10C0980042EA051289684260C461C163036270BDE7
:10C0A800002C0140036A23F48052026270B5056ACD
:10C0B8004368C4690A6824F4E64646EA02228C8882
:10C0C8008E8925F40055344345EA0434084DA842C6
:10C0D80003D005F50065A84204D10D8A23F48043F6
:10C0E80043EA851389684360C2610164046270BDD4
:10C0F800002C0140002303608380C3808360838118
:10C10800C381038243827047836923F00802114385
:10C1180081617047836923F4006242EA01218161E9
:10C128007047C36923F008021143C1617047C369AE
:10C1380023F4006242EA0121C16170470023012211
:10C14800038043808280C38003817047406B7047BF
:10C15800806B7047C06B7047006C7047836923F031
:10C168000C0282618369194381617047836923F4F2
:10C1780040628261836943EA012181617047C26933
:10C188004FF6F3731340C361C2691143C16170472D
:10C19800C2694FF2FF331340C361C26909028BB20F
:10C1A8001A43C2617047F8B50D460B88AA884988BA
:10C1B800044643B92B89FFF740FEE9882046BDE8CD
:10C1C800F840FFF7CBBF042B08D12B89FFF74AFEB5
:10C1D800E9882046BDE8F840FFF7C8BF082BB5F846
:10C1E80008C0066A1BD14FF6FF6737400762C3696C
:10C1F800066A4FF60C771F404FF2FF53334042EA6E
:10C208000C1243EA012141F480731743E988BFB255
:10C218009AB2C7610262BDE8F840FFF7B0BF4EF6B8
:10C22800FF7737400762C369076A40F6FF46120284
:10C238001E4045F6FF733B4042EA0C3C1FFA8CF265
:10C2480043EA0131164341F48052E988C66193B24A
:10C258000362BDE8F840FFF79BBF436C11B143F49C
:10C26800004201E059044A0C42647047C3680AB1AD
:10C27800194302E0C94389B21940C1607047036994
:10C28800C26811EA030003D011420CBF002001204C
:10C298007047C9438AB2026170470000C37810B57D
:10C2A80003B3164CE168CB43C3F302244178037807
:10C2B800C4F1040201FA02F10F2222FA04F284788E
:10C2C80022400A43110103F16043CAB203F56141F8
:10C2D80081F800230078012200F01F03410902FAC7
:10C2E80003F007E000780122410900F01F0302FA79
:10C2F80003F02031024B43F8210010BD00ED00E0AF
:10C3080000E100E0036830B5044623F00100206036
:10C318000D466268AB6822F4405141EA0300606050
:10C328002268EB6822F4B0516A6821F00C0043EAF5
:10C3380002012B6941EA030202432260A0686B698B
:10C3480020F4407195B041EA03026846A260FFF705
:10C35800DFF91848844201D10C9A0EE016498C4244
:10C3680001D10D9A09E0154B9C4201D10E9A04E0C7
:10C37800134884420CBF0F9A109A2168286811F458
:10C38800004F18BF5200B2FBF0F300FB13212A68DC
:10C398002068B1EB520F28BF0133020406D54FF6CF
:10C3A800F072C3F342011A4041EA020398B2A08135
:10C3B80015B030BD0038014000440040004800403E
:10C3C800004C0040036811B143F0010101E023F083
:10C3D800010101607047C905CA0D0285704783686D
:10C3E8000AB1194301E023EA010181607047C1F3F2
:10C3F800072310B5C9B20124022B04FA01F101D1B7
:10C40800043002E0032B08BF0830036812B143EA86
:10C41800010201E023EA0102026010BD090C0123B8
:10C4280003FA01F202627047044B1A69120604D536
:10C43800034800F188315860596070470020024075
:10C4480023016745024B1A6942F080001861704762
:10C4580000200240014BD860704700BF0020024016
:10C46800084BDA68D20709D4D868C00608D4D96856
:10C4780011F0040F0CBF04200320704701207047FF
:10C48800022070470020024010B50446FFF7E8FF7D
:10C49800012806D11CB1FFF7E3FF013CF8E70520AE
:10C4A80010BD002C08BF052010BD000073B5002387
:10C4B80006464FF430200D460193FFF7E5FF0428A8
:10C4C80019D10D4C2069AAB240F0010121614FF445
:10C4D80030203280FFF7D8FF042808D102360196B1
:10C4E800019B2D0C1D804FF43020FFF7CDFF2169F3
:10C4F80021F0010222617CBD0020024038B50546CA
:10C508004FF43020FFF7C0FF042811D1094C2369EC
:10C5180043F0020020616561216941F04002226117
:10C528004FF43020FFF7B0FF236923F002012161A7
:10C5380038BD00BF00200240036823F001020260FA
:10C548000268144B13408A6843EA02234A6813437B
:10C558000A68036022F070630361026842F0010315
:10C568000022036082608B69C2600A691A43826094
:10C57800836843F400428260CB68026849691A43C1
:10C588000260436823F0784222F400430B4343607F
:10C59800704700BFFFE0CF0000234FF40042036064
:10C5A80043608360C36003614261836170470368CD
:10C5B80011B143F0010101E023F00101016070476E
:10C5C80030B54568064C890543EA91532C400399D8
:10C5D8001C4344EA010343EA0242426030BD00BF03
:10C5E800009800FC81627047406AC0B27047836956
:10C5F80019420CBF002001207047C161704700003C
:10C6080002684FF6FE73134003602D4B00219842D9
:10C61800016041608160C16022D02A49884229D0E6
:10C62800294B984230D02949884237D0284B984224
:10C638003ED0284B984206D153F8681C41F470004C
:10C6480043F8680C70472449884206D151F87C0C9D
:10C6580040F0706241F87C2C7047204B984206D11C
:10C6680053F8042C42F00F0143F8041C70471C498E
:10C67800884206D151F8183C43F0F00041F8180CF4
:10C688007047184B984206D153F82C2C42F470612D
:10C6980043F82C1C70471449884206D151F8403C95
:10C6A80043F4704041F8400C7047104B984205D154
:10C6B80053F8542C42F4702143F8541C704700BFBF
:10C6C800080002401C0002403000024044000240C2
:10C6D800580002406C0002408000024008040240FA
:10C6E8001C04024030040240440402405804024042
:10C6F80070B506688C680D6A26F4FF4222F0700651
:10C708000A6945EA04034C6913438A692343CC69DF
:10C7180013431C434B6A44EA03028B6A1A433243AD
:10C7280002608B890A68496843608260C16070BD95
:10C7380000230360436083608381036143618361F5
:10C74800C361036243628362704719B1016841F0B3
:10C75800010303E002684FF6FE731340036070475D
:10C7680041607047406880B2704703680AB1194356
:10C7780001E023EA0101016070470000C3004CBFDB
:10C78800014B024B58607047000402400000024011
:10C7980000B540F6D87320F00042C3F649739A42B8
:10C7A80083B0014615DDB2F1FF4F03DBF4F730F932
:10C7B80003B000BD694600F095FB00F00302012AB2
:10C7C800009801990ED0022A07D082B900F0A0FD86
:10C7D800EEE7002100F09CFDEAE700F099FD00F18A
:10C7E8000040E5E701F038FC00F10040E0E70122F5
:10C7F80001F032FCDCE700BF30B5C0F3C754A4F148
:10C808007F031E2B83B0014621DC581C1DDBCD0F96
:10C81800162B0CDD21F07F4323F4000040F40000C8
:10C82800963C00FA04F005B1404203B030BD11480F
:10C8380050F825402046F4F7EDF80190214601987C
:10C84800F4F7E6F820F0004121B90020EDE7F4F70D
:10C85800AFFBEAE720F07F4222F40003C0F3C750A1
:10C8680043F40001C0F1960221FA02F0002DDCD059
:10C87800DAE700BF5827010800B540F6D87320F062
:10C888000042C3F649739A4283B0014616DDB2F1FD
:10C89800FF4F03DBF4F7BCF803B000BD694600F0B6
:10C8A80021FB00F00300012815D002280BD0B8B9ED
:10C8B80000980199012201F0CFFBEDE70021002249
:10C8C80001F0CAFBE8E700980199012201F0C4FBD6
:10C8D80000F10040E0E70098019900F019FDDBE75E
:10C8E8000098019900F014FD00F10040D4E700BF62
:10C8F80070B5244C8AB0064600F09AF894F90030D6
:10C908000133054603D0304601F0A8FD10B928468A
:10C918000AB070BD304601F053FD4FF07E51F4F778
:10C928003DFB0028F3D0184A01210025304601922A
:10C9380000910895F3F7B2FD02460B461348CDE97E
:10C948000423CDE9022301F009FC94F90030022BFD
:10C95800CDE906010BD0684601F0FEFB38B1089816
:10C9680050B9DDE90601F3F7FFFF0546CFE701F00F
:10C9780081FE21210160F2E701F07CFE089A026045
:10C98800EFE700BFA0010020602701086827010821
:10C9980000F002BA70B5244C8AB0054600F04EFC8F
:10C9A80094F900300133064608D0284601F056FDB8
:10C9B80020B128460021F4F7D3FA10B930460AB05E
:10C9C80070BD1A4A01212846002600910192089656
:10C9D800F3F764FD2478CDE90401CDE902017CB9BF
:10C9E80000220023CDE90623684601F0B5FB88B193
:10C9F8000898A0B9DDE90601F3F7B6FF0646DDE7BA
:10CA08000020002102460B46F3F7C6FE022CCDE9B2
:10CA18000601E9D101F02EFE21230360E8E701F0C9
:10CA280029FE08990160E5E7A00100206C270108AC
:10CA3800F8B520F00043B3F17E5F044613D00BDC59
:10CA4800B3F17C5F14DAB3F10C5F00F3A48040F615
:10CA5800DB70C3F6C970F8BD0146F3F7D9FF01468C
:10CA6800F4F794F9F8BD002840F30E810020F8BDD2
:10CA78000028C0F20E8101464FF07E50F3F7C8FF40
:10CA88004FF07C51F4F7CEF8044600F0D7FB4EF691
:10CA98000871064620F47F65C3F611012046F4F7B5
:10CAA800C1F847F60471C3F64F21F3F7B3FF2146E7
:10CAB800F4F7B8F841F24611C3F62451F3F7A8FF8A
:10CAC8002146F4F7AFF840F6A821C3F64E61F3F714
:10CAD800A1FF2146F4F7A6F84BF29001C3F6A66130
:10CAE800F3F796FF2146F4F79DF84AF6AB21C3F613
:10CAF8002A61F3F78FFF2146F4F794F84CF22E6180
:10CB08000746C3F69D512046F4F78CF843F261318D
:10CB1800C3F63071F3F77CFF2146F4F783F845F24A
:10CB28002D71C4F20101F3F775FF2146F4F77AF885
:10CB38004DF23911C4F21901F3F76AFF2146F4F7EF
:10CB480071F84FF07E51F3F765FF01463846F4F768
:10CB58001DF93146F4F766F825F00F050746294612
:10CB68002846F4F75FF801462046F3F751FF2946B7
:10CB780004463046F3F74EFF01462046F4F706F91F
:10CB880001463846F3F746FF2946F3F743FF0146C7
:10CB9800F3F740FFF8BD0146F4F744F84EF6087184
:10CBA800C3F611010546F4F73DF847F60471C3F6DC
:10CBB8004F21F3F72FFF2946F4F734F841F24611D5
:10CBC800C3F62451F3F724FF2946F4F72BF840F66F
:10CBD800A821C3F64E61F3F71DFF2946F4F722F8A2
:10CBE8004BF29001C3F6A661F3F712FF2946F4F75A
:10CBF80019F84AF6AB21C3F62A61F3F70BFF294669
:10CC0800F4F710F84CF22E610646C3F69D512846FB
:10CC1800F4F708F843F26131C3F63071F3F7F8FE20
:10CC28002946F3F7FFFF45F22D71C4F20101F3F72E
:10CC3800F1FE2946F3F7F6FF4DF23911C4F2190156
:10CC4800F3F7E6FE2946F3F7EDFF4FF07E51F3F7D1
:10CC5800E1FE01463046F4F799F801462046F3F71D
:10CC6800E1FF014642F26810C3F2A230F3F7D0FEAA
:10CC780001462046F3F7CCFE014640F6DA70C3F6CB
:10CC8800C970F3F7C5FEF8BD40F6DB70C4F2490081
:10CC9800F8BD4FF07E51F3F7BDFE4FF07C51F3F72E
:10CCA800C1FF4EF60871C3F611010446F3F7BAFF47
:10CCB80047F60471C3F64F21F3F7ACFE2146F3F7AC
:10CCC800B1FF41F24611C3F62451F3F7A1FE214604
:10CCD800F3F7A8FF40F6A821C3F64E61F3F79AFED2
:10CCE8002146F3F79FFF4BF29001C3F6A661F3F7D5
:10CCF8008FFE2146F3F796FF4AF6AB21C3F62A6169
:10CD0800F3F788FE2146F3F78DFF0646204600F02C
:10CD180095FA4CF22E610546C3F69D512046F3F76D
:10CD280081FF43F26131C3F63071F3F771FE21469A
:10CD3800F3F778FF45F22D71C4F20101F3F76AFEAB
:10CD48002146F3F76FFF4DF23911C4F21901F3F7D9
:10CD58005FFE2146F3F766FF4FF07E51F3F75AFE68
:10CD680001463046F4F712F82946F3F75BFF42F222
:10CD78006811C3F2A231F3F74BFE01462846F3F7D8
:10CD880049FE0146F3F746FE014640F6DA70C4F262
:10CD98004900F3F73DFEF8BDF8B521F00044B4F1C1
:10CDA800FF4F034617DC20F00045B5F1FF4F06465C
:10CDB80011DCB1F17E5F42D08F1707F0020040EA24
:10CDC800D37775B9022F35D0032F08D140F6DB731E
:10CDD800CCF2490303E01846F3F71CFE0346184655
:10CDE800F8BDD4B1B4F1FF4F2DD0B5F1FF4F14D039
:10CDF8002C1BE4153C2C18DC002952DB1846F3F7F1
:10CE0800C5FF01F0DDFA01F0AFF9012F46D0022F7E
:10CE180035D0002F25D10346E1E7002E40F6DB731D
:10CE28001CDBC3F6C9731846F8BD40F6DB70C3F6C1
:10CE3800C970EAE740F6DB73C4F24903CFE7BDE8FF
:10CE4800F84001F091B9B5F1FF4F2FD0022FF1D082
:10CE5800032FBBD0012F34D00023C0E7CBF6C97312
:10CE6800BDE74BF62E51C3F2BB31F3F7D3FD40F6C5
:10CE7800DB71C4F24901F3F7CBFD0346AFE74BF68C
:10CE88002E51C3F2BB31F3F7C5FD014640F6DB7006
:10CE9800C4F24900F3F7BCFD0346A0E700F10043E4
:10CEA8009DE714F13C0FA9DA0020AEE7022F13D05A
:10CEB800032F0CD0012F40F6DB7305D0C3F649735E
:10CEC8008DE74FF000438AE7CBF6497387E74CF6C6
:10CED800E433CCF2160382E74CF6E433C4F21603CB
:10CEE8007DE700BF2DE9F04F40F6D87320F00044ED
:10CEF800C3F649739C4289B006460D4640F38B80C1
:10CF08004CF6E331C4F216018C4226DC4FF478610A
:10CF18000028C3F6C97140F32C81F3F779FD4FF46B
:10CF28007D6124F00F04C3F6C9718C42064600F0F7
:10CF3800818044F24341C3F23571F3F769FD01463C
:10CF480028603046F3F764FD44F24341C3F235717B
:10CF5800F3F75EFD0127686061E04FF47867C4F27B
:10CF68004937BC4240F38180B4F1FF4F5BDA4FEAA6
:10CF7800E459A9F18609A4EBC9542046F4F718F836
:10CF8800F3F7FCFD0246014620460592F3F740FD03
:10CF98004FF08741F3F746FE0746F4F709F8F3F731
:10CFA800EDFD0146044638460694F3F731FD4FF08F
:10CFB8008741F3F737FE00210790F3F7C7FF0028F2
:10CFC80000F0F7800327204600210DF11808013FE3
:10CFD800F3F7BCFF40B158F8044D00212046013F4B
:10CFE800F3F7B4FF0028F6D1924B0220009001938A
:10CFF80005A83B4629464A4600F066FA002E074631
:10D008000DDA95E80C0002F1004103F100422960B5
:10D018006A60474203E00023286000274B603846D7
:10D0280009B0BDE8F08F0146F3F7F2FC002768600D
:10D038002860F4E74FF48841C3F23571F3F7E8FC50
:10D048004AF20831C2F685610446F3F7E1FC01466D
:10D0580028602046F3F7DCFC4AF20831C2F6856105
:10D06800F3F7D6FC01276860D9E701F0A9F94FF674
:10D078008411C3F622718046F3F7D4FD4FF07C513A
:10D08800F3F7C8FCF3F794FF0746F3F777FD4FF47F
:10D098007861C3F6C9718346F3F7C4FD014640467B
:10D0A800F3F7B6FC44F243418146C3F23571584662
:10D0B800F3F7B8FD1F2F8246484620DC791E5E4BE9
:10D0C80053F8211024F0FF028A4218D05146F3F792
:10D0D8009FFC8046C5F8008041464846F3F798FC17
:10D0E8005146F3F795FC002E686098DA08F100487D
:10D0F80000F10042C5F800806A607F428FE7514620
:10D10800F3F786FCE3158046C0F3C7501A1A082ABD
:10D11800E0DD4FF48841C3F2357158460393F3F7C5
:10D1280081FD824651464846F3F772FC0446214683
:10D138004846F3F76DFC5146F3F76AFC4AF20831AA
:10D148008146C2F685615846F3F76CFD4946F3F708
:10D158005FFC824651462046F3F75AFC039BC0F316
:10D16800C7518046581A192841DCC5F80080A146E5
:10D17800B2E7F3F74FFC4FF47D6724F00F04C3F6D2
:10D18800C977BC42064616D044F24341C3F2357112
:10D19800F3F740FC014628603046F3F739FC44F2C7
:10D1A8004341C3F23571F3F735FC4FF0FF37686040
:10D1B80035E7032718E74FF48841C3F23571F3F7D1
:10D1C80029FC4AF20831C2F685610446F3F722FCCD
:10D1D800014628602046F3F71BFC4AF20831C2F6E4
:10D1E8008561F3F717FC4FF0FF37686017E74FF4D6
:10D1F8002341C2F685615846F3F714FD804641463F
:10D208002046F3F705FC814649462046F3F700FC23
:10D218004146F3F7FDFB43F232110446C2F28D4159
:10D228005846F3F7FFFC2146F3F7F2FB82464846DF
:10D238004CE700BFF42701087427010820F00042DA
:10D24800B2F1FF4FF8B50446034646D2002A42D051
:10D25800002852DBC415B2F5000F09D210F40005FE
:10D2680053D15B0001351902FBD5C5F10100241823
:10D2780023F07F417F3C21F40006E20746F40000DA
:10D2880048BF400043004FF08072002760109A4268
:10D298003C462CDD5B004FF400021825A618510807
:10D2A8009E4205F1FF3502DCB4189B1BBF185B00DA
:10D2B80062189A4202DC9B1A54187F185B004A08CD
:10D2C800013DEBD113B107F001017F187C1004F187
:10D2D8007C5303EBC0542046F8BD0146F3F7A2FC8B
:10D2E80001462046F3F796FB04462046F8BD4FF06A
:10D2F800007403F17F431746CCE70146F3F788FB38
:10D308000146F3F743FD0446E5E70120AFE700BF18
:10D318002DE9F84320F00046B6F1485F05460F4670
:10D328005BDAF3F745FE002800F0CA802946284654
:10D33800F3F778FC4DF24E71CAF647510446F3F7FD
:10D3480071FC47F2F641C3F20F11F3F763FB214674
:10D35800F3F768FC4FF27C21C3F29341F3F758FBD3
:10D368002146F3F75FFC40F60151C3F2D071F3F7A1
:10D3780051FB2146F3F756FC40F66131C3F6B6215E
:10D38800F3F746FB2146F3F74DFC4AF6AB21C3F60B
:10D398002A51F3F73FFB2146F3F744FC8046204629
:10D3A8004FF07C51F3F73EFC414606462046F3F722
:10D3B80039FC394604462846F3F734FC0146204632
:10D3C800F3F726FB01463046F3F722FB01464FF000
:10D3D8007E50F3F71DFBBDE8F8830146F3F722FC06
:10D3E8004DF24E71CAF647510446F3F71BFC47F25B
:10D3F800F641C3F20F11F3F70DFB2146F3F712FCC8
:10D408004FF27C21C3F29341F3F702FB2146F3F775
:10D4180009FC40F60151C3F2D071F3F7FBFA21463B
:10D42800F3F700FC40F66131C3F6B621F3F7F0FAE2
:10D438002146F3F7F7FB4AF6AB21C3F62A51F3F777
:10D44800E9FA2146F3F7EEFB49F69913C3F6996317
:10D458009E428046A3DD0020C3F64870864227DC42
:10D4680006F17F464FF07E503146F3F7D1FA8146F8
:10D4780020464FF07C51F3F7D5FB3146F3F7C8FA55
:10D48800414606462046F3F7CDFB39460446284672
:10D49800F3F7C8FB01462046F3F7BAFA01463046CF
:10D4A800F3F7B6FA01464846F3F7B2FABDE8F8834F
:10D4B8004FF000090026C3F63879C3F69066D7E71F
:10D4C8004FF07E50BDE8F8832DE9F04FDFB08B4C6C
:10D4D800689D0C9303F1FF3CD31E54F825600A9114
:10D4E80048BF131D8346D81020EAE0710896CDF88E
:10D4F80010C0049D0D91089E0D9CCF4302EBC702FE
:10D50800AB190792C5EB04074DD4F8186999C7EB16
:10D518000009461C002F01EB870522AC09F0010A1F
:10D52800C0F27D852868F3F729FB0137B7422060F0
:10D538004FF0040837D0BAF1000F23D0002FC0F203
:10D54800718555F80800F3F719FB0137B74244F81D
:10D55800080008F1040815D125E055F80800F3F78C
:10D568000DFB013708F1040944F8080013D455F8F5
:10D578000900F3F703FB0137B74244F8090009F142
:10D58800040810D0002FE8DA0020013708F1040958
:10D5980044F80800EBD501370020B74244F80900E9
:10D5A80009F10408EED1089A002AC0F23E850898CD
:10D5B8000C9E81004AAD6C18029149AF03944FEA62
:10D5C800860A049A002AC0F24C8322AB03EB860435
:10D5D800DBF8000054F8041CF3F724FB0146002094
:10D5E800F3F718FAA4F104090424AAF10405544530
:10D5F800C5F3800580462AD06DB159F8041DDBF8C3
:10D608000400F3F70FFB01464046F3F703FA08243A
:10D61800544580461BD059F8041C5BF80400F3F706
:10D6280001FB01464046F3F7F5F9251D804659F8F8
:10D63800081C5BF80500F3F7F5FA01464046F3F7D6
:10D64800E9F92C1D54458046A9F10809E3D147F8AA
:10D65800048F039801368742B3D1DDF808C0089ECD
:10D668000EA901EB0C070997B2005EAB9C18002EBF
:10D67800029254F8509C7BDD0DF5947E0EEB02056A
:10D68800029A4FF06E5148460DAFBF18F3F7CAFA29
:10D69800F3F78EFCF3F772FA4FF087410190F3F736
:10D6A800C1FA01464846F3F7B3F9F3F781FC0EAC2B
:10D6B80020600198014655F8040DF3F7ABF9BC4218
:10D6C8008146C7F3800153D0D1B14FF06E51F3F7C3
:10D6D800A9FAF3F76DFCF3F751FA4FF0874101907F
:10D6E800F3F7A0FA01464846F3F792F9F3F760FC1E
:10D6F8000FAC019A2060114633E000BF0C2B0108E3
:10D708004FF06E514846F3F78DFAF3F751FCF3F7F3
:10D7180035FA4FF087418046F3F784FA01464846C8
:10D72800F3F776F9F3F744FC4146606055F8040DC9
:10D73800F3F770F94FF06E518146F3F773FAF3F788
:10D7480037FCF3F71BFA4FF087418046F3F76AFA84
:10D7580001464846F3F75CF9F3F72AFC4146A06016
:10D76800083455F8040DF3F755F9BC428146C7D182
:10D778000799484600F09EFE4FF078510546F3F7AA
:10D7880051FA00F021FE4FF08241F3F74BFA0146BF
:10D798002846F3F73DF90746F3F70AFC8146F3F705
:10D7A800EDF901463846F3F733F9079B002B074696
:10D7B80040F33181721E0EACC3F1080554F82230D3
:10D7C80043FA05F101FA05F00DF1380E079D1B1A11
:10D7D800C5F107044EF82230894443FA04F4002CBA
:10D7E80052DD002E09F1010940F34B82029ADDF85F
:10D7F80008C00EAB101F53F8042B0EA90025614476
:10D80800C0F3800022B1C2F5807543F8045C01259D
:10D818008B4225D058B10F9A0433002D00F0F280C6
:10D82800C2F1FF0043F8040C01258B4218D053F8CD
:10D83800042BC2F1FF0015B9C2F5807012B143F88C
:10D84800040C012553F8042BC2F1FF001DB9C2F5E1
:10D858008070002AE9D001258B4243F8040CE6D1F8
:10D86800079B002B0DDD012B00F0DE80022B08D179
:10D87800711E0DF1380E5EF8212002F03F004EF8BF
:10D888002100022C00F0DC8038460021F3F75EFB13
:10D89800002800F0EF800898751EA84224DC029B3F
:10D8A800DDF824E00EAAD1180B46CEEB010053F8A0
:10D8B800042D011F7345C1F3800012D038B153F80D
:10D8C800041DDDF824C0634542EA010209D0099F1E
:10D8D80053F8040D53F8041D0243BB4242EA010207
:10D8E800F6D1002A40F08683089F0EAD781E55F8C1
:10D8F8002020002A40F0C78105EB8004012354F85A
:10D90800041D01330029FAD0F018771C87420B90C8
:10D9180073DC049DDDF834900B9B0C9CDDF808C08B
:10D92800EA19699F06EB0901981B07EB8108A619FC
:10D938004AA922AB01EB0C05571C820003EB8600B9
:10D94800CDF80C800295069205900026039C54F8A9
:10D95800040F0394F3F712F9049D0599002D8851DB
:10D968004DDB0DF1880E0EEB8702AAF1040352F885
:10D97800041CDBF80000C3F38004A2F10409F3F7E8
:10D9880051F901460020F3F745F80425554580462E
:10D998002AD06CB159F8041DDBF80400F3F742F9FA
:10D9A80001464046F3F736F80825554580461BD012
:10D9B80059F8041C5BF80500F3F734F901464046B2
:10D9C800F3F728F82C1D804659F8081C5BF804006A
:10D9D800F3F728F901464046F3F71CF8251D55458D
:10D9E8008046A9F10809E3D10298069940F8048F06
:10D9F800043601378E420290A8D10B9E34E64FF0D0
:10DA08000008F1E7002A3FF410AFC2F5807543F82B
:10DA1800045C012509E740F01D81701E0DF1380CEA
:10DA28005CF820100C12DAE6731E0DF1380C022C8B
:10DA38005CF8231001F07F024CF823207FF424AF18
:10DA480039464FF07E50F2F7E3FF0746002D3FF4CA
:10DA58001BAF07994FF07E5000F02CFD0146384669
:10DA6800F2F7D6FF074638460021F3F76FFA002889
:10DA78007FF411AF0394079CCDF8109061423846AB
:10DA880000F018FD4FF087410546F3F77DFA0028AE
:10DA980000F0D4824FF06E512846F3F7C3F8F3F73D
:10DAA80087FAF3F76BF84FF087410746F3F7BAF8B0
:10DAB80001462846F2F7ACFFF3F77AFA0EAB43F8C3
:10DAC80026003846F3F774FA013607990DF1380C39
:10DAD80008314CF8260007914FF07E50079900F066
:10DAE800E9FC002E0446C0F2AC804FEA860A0EAF6D
:10DAF8005744C6EB867B4FEA8B09C9F100034AA954
:10DB0800386801EB0A08C3F3800BF3F737F82146AE
:10DB1800F3F788F84FF06E51C8F800002046F3F785
:10DB280081F8A9F104096FF0030ACA45054631D006
:10DB3800BBF1000F0BD057F8040CF3F71FF8294678
:10DB4800F3F770F86FF0070A48F8040C1AE057F872
:10DB58000A00F3F713F82946F3F764F84FF06E510B
:10DB680048F80A002846F3F75DF8AAF104040546C8
:10DB78003859F3F703F82946F3F754F848F804003E
:10DB8800AAF1080A28464FF06E51F3F74BF8CA4538
:10DB98000546DCD1701CDFF8BC94DDF820A00290AB
:10DBA80000270596BAF1000FC0F22082002FC0F2BC
:10DBB8001D82002600241AF0010F354620D0D8F81F
:10DBC8000010D9F80000F3F72DF801462046F2F7C7
:10DBD80021FF0125AA45044626DB0426BD420FDDA8
:10DBE80022E0BB4520DC58F8021059F80200F3F790
:10DBF80019F801462046F2F70DFFBD42044613DC32
:10DC080058F8061059F80600F3F70CF801462046B4
:10DC1800F2F700FF05F1010B06F104020235DA45BF
:10DC2800044602F10406DCDA5EABDDF808E003EB3B
:10DC380087010137774541F8A04CA8F10408B1D114
:10DC4800059E689C032C31D8DFE814F0A0013A0146
:10DC58003A0136004FF07C51F3F796F958B9002491
:10DC680012E64FF0000847F8048F03980136874200
:10DC78007FF4A7ACF1E40224002E09F101093FF773
:10DC8800B5AD0025ECE501233EE600230399002904
:10DC980000F00B81379C369804F100420A9C00F191
:10DCA800004503F1004325606260A360049D05F010
:10DCB80007005FB0BDE8F08F002EE6DD06F1FF3803
:10DCC80036AF07EB88094D460DF1D40A55F80429FB
:10DCD800D5F808B0019210465946F2F79BFE8046E7
:10DCE80041460198F2F794FE01465846F2F792FE33
:10DCF8005545C9F38003A860C5F8048044D0BBB17A
:10DD080055F80429D5F808B0019210465946F2F79B
:10DD180081FE0199804608464146F2F779FE0146A0
:10DD28005846F2F777FE5545C5F80480A8602BD011
:10DD38002C4654F80439D4F808B0019318465946CB
:10DD4800F2F768FE804641460198F2F761FE014607
:10DD58005846F2F75FFEC4F80480A06055F804BC8A
:10DD6800251F5846D5F808804146F2F753FE044669
:10DD780021465846F2F74CFE01464046F2F74AFE65
:10DD880055456C60A860D3D1012E7FF77EAF4D4614
:10DD9800C7EB090C55F804B9D5F808A05846514600
:10DDA800ACF10409F2F736FE804641465846F2F7D0
:10DDB8002FFE01465046F2F72DFEBD42C9F38009F9
:10DDC800C5F80480A86043D0B9F1000F15D055F804
:10DDD80004A9D5F8089050464946F2F71BFE80463C
:10DDE80041465046F2F714FE01464846F2F712FE45
:10DDF800BD42C5F80480A8602AD02C4654F804A96E
:10DE0800D4F8089050464946F2F704FE8046414649
:10DE18005046F2F7FDFD01464846F2F7FBFDC4F80F
:10DE28000480A06055F8049C251F4846D5F8088052
:10DE38004146F2F7EFFD044621464846F2F7E8FD71
:10DE480001464046F2F7E6FDBD426C60A860D4D1B9
:10DE5800013607EB86073E4608357A1B131F56F82E
:10DE6800041D0020C3F38007F2F7D4FDAE42034639
:10DE78003FF40CAF3FB156F8041DF2F7CBFDAE42AC
:10DE880003463FF403AF1846341F56F8041CF2F754
:10DE9800C1FD083E54F8041CF2F7BCFDAE42F3D1B4
:10DEA8000399034600297FF4F5AEDDF828E036999A
:10DEB8003798CEF80010CEF80400CEF80830F5E612
:10DEC8000023002E29DB36AF751C07EB8504254699
:10DED800E21B55F8041D0020A2F1040CCCF38008C5
:10DEE800F2F798FDBD42034617D0B8F1000F06D0EF
:10DEF80055F8041DF2F78EFDBD4203460DD01846B5
:10DF08002C1F55F8041CF2F785FD083D54F8041C35
:10DF1800F2F780FDBD42F3D103460399002967D08B
:10DF280003F10040DDF828E01946CEF800003698E5
:10DF3800F2F76EFD002E034621DD36AF07EB8606AD
:10DF4800F51B2A1F3799C2F38007F2F763FD37AC38
:10DF5800B442034613D037B16168F2F75BFD38ACC1
:10DF6800B44203460BD0184654F8041FF2F752FD8A
:10DF780054F8041FF2F74EFDB442F5D10346039955
:10DF880009B103F100430A9C63608FE6002E5FDB52
:10DF980036AF013607EB86000546C21B55F8041D4F
:10DFA8000020141FF2F736FDBD42C4F38006034675
:10DFB80015D036B155F8041DF2F72CFDBD420346C5
:10DFC8000DD018462C1F55F8041CF2F723FD083D08
:10DFD80054F8041CF2F71EFDBD42F3D10346039921
:10DFE80009B103F100430A9C23605FE600241BE6A5
:10DFF800184697E70EAE079A56F82530CDF81090D8
:10E00800083A039407920BBB06EB85042E4654F896
:10E01800045D013E083A002DF9D007925CE5002026
:10E02800FFF783BA0020FFF790BA0C9B4FEA820EE5
:10E03800CDF808E04FEA830AFFF70FBB2846F2F74E
:10E04800B7FF0DF1380E4EF8260045E52E4643E59C
:10E058000023C4E7182B01082DE9F84320F00043FA
:10E06800B3F1485F04460F46904603DAF2F7A0FF83
:10E07800002859D021462046F2F7D4FD214605460E
:10E08800F2F7D0FD4CF6D311C2F62E71064628469B
:10E09800F2F7C8FD42F63471C3F2D721F2F7B8FCA3
:10E0A8002946F2F7BFFD4EF61B71C3F23861F2F74D
:10E0B800B1FC2946F2F7B6FD40F60151C3F65011FE
:10E0C800F2F7A6FC2946F2F7ADFD48F68901C3F63A
:10E0D8000841F2F79FFC8146B8F1000F27D04FF0B6
:10E0E8007C513846F2F79EFD494680463046F2F7A5
:10E0F80099FD01464046F2F78BFC2946F2F792FD5E
:10E108003946F2F785FC4AF6AB210546C3F62A6183
:10E118003046F2F787FD01462846F2F77BFC0146B8
:10E128002046F2F775FC04462046BDE8F883014610
:10E138002846F2F777FD4AF6AB21C3F62A61F2F7D3
:10E1480067FC3146F2F76EFD01462046F2F762FCA5
:10E1580004462046BDE8F8830020704700210020CF
:10E16800C7F6F871704700BF2DE9F04120F000456F
:10E17800B5F1A14F044606460DDBB5F1FF4F00F39C
:10E188009C80002840F6DB7440F3D480C3F6C97441
:10E198002046BDE8F0814FF6FF73C3F6DF639D426A
:10E1A80000F3A280B5F1445FC0F28E804FF0FF37D4
:10E1B80021462046F2F736FD01468046F2F732FD49
:10E1C80046F6D711C3F685410546F2F72BFD4DF605
:10E1D8005921C3F64B51F2F71DFC2946F2F722FDEF
:10E1E80046F63531C3F68851F2F714FC2946F2F7A2
:10E1F80019FD42F66E61C3F6BA51F2F70BFC2946D7
:10E20800F2F710FD44F62511C3F61261F2F702FC8D
:10E218002946F2F707FD4AF6AB21C3F6AA61F2F7E1
:10E22800F9FB4146F2F7FEFC4AF221218046CBF683
:10E2380015512846F2F7F6FC4FF26B11C3F66E51F2
:10E24800F2F7E6FB2946F2F7EDFC48F29571C3F6C2
:10E258009D51F2F7DDFB2946F2F7E4FC48F63861F8
:10E26800C3F6E351F2F7D4FB2946F2F7DBFC4CF690
:10E27800CD41C3F64C61F2F7CBFB2946F2F7D2FC4D
:10E288007B1C0146404658D0F2F7C4FB2146F2F702
:10E29800C9FC494B53F82710F2F7BAFB2146F2F7AD
:10E2A800B7FB0146454850F82700F2F7B1FB002EAE
:10E2B8003DDB04462046BDE8F0810146F2F7AAFBA3
:10E2C80004462046BDE8F0814FF2CA21C7F2491141
:10E2D800F2F7A0FB4FF07E51F2F760FE00283FF402
:10E2E80065AF2046BDE8F08100F06AF84FF6FF718F
:10E2F800C3F697718D4204464FF6FF7228DCC3F6C9
:10E308002F72954246DC0146F2F784FB4FF07E51AE
:10E31800F2F77EFB4FF0804105462046F2F77AFB84
:10E3280001462846F2F732FD0027044640E700F18F
:10E3380000442DE7CBF6C9742AE7F2F76BFB2146B8
:10E34800F2F770FC01462046F2F762FB04461FE72D
:10E35800C4F21B02954214DC4FF07F51F2F758FBD0
:10E368004FF07F5105462046F2F75CFC4FF07E5196
:10E37800F2F750FB01462846F2F708FD022704464B
:10E3880016E700202146CBF68070F2F7FFFC032742
:10E3980004460DE74FF07E51F2F73AFB4FF07E51FD
:10E3A80007462046F2F736FB01463846F2F7EEFC00
:10E3B80001270446FCE600BF442B0108542B010842
:10E3C80020F00040704700BFF8B520F00046F50D7A
:10E3D8007F3D162D014604461BDC002D074620DB39
:10E3E8004FF6FF73C0F27F0343FA05F606420ED0DC
:10E3F8004FF2CA21C7F24911F2F70CFB0021F2F7DC
:10E40800CDFD18B1002C1BDB27EA0604214608467F
:10E41800F8BDB6F1FF4FFAD3F2F7FCFA0146084609
:10E42800F8BD4FF2CA21C7F24911F2F7F3FA0021F9
:10E43800F2F7B4FD0028E9D0002C07DB0024E5E75B
:10E448004FF4000040FA05F56719DDE70021CBF627
:10E458008071002E18BF0C46D8E700BF08B902200B
:10E468007047B0F1004FFAD0A0F500026FF00143F9
:10E478009A4201D80420704700F1FF419942F9D926
:10E488004FF6FE73421EC0F27F039A4201D8032062
:10E49800704700F100414A1E9A42F8D9B0F1FF4F87
:10E4A80005D010F5000F14BF00200120704701208F
:10E4B800704700BF38B530F00044034602460D46A9
:10E4C8000FD0B4F1FF4F0ED2B4F5000F11D3E40D05
:10E4D8006419FE2C33DC002C1BDD22F0FF4141EADD
:10E4E800C453184638BD0146F2F794FA0346184655
:10E4F80038BD4FF09841F2F795FB43F6B041CFF69F
:10E50800FF718D42034612DBC0F3C7540246193C23
:10E51800DEE714F1160F21DA4CF250329542194613
:10E528000EDC44F26020C0F6A25000F023F844F25A
:10E538006021C0F6A251F2F775FB0346D1E71946F0
:10E548004FF2CA20C7F2491000F014F84FF2CA215E
:10E55800C7F24911F2F766FB0346C2E722F0FF4310
:10E5680004F1190043EAC0504FF04C51F2F75AFB3E
:10E578000346B6E701F0004120F000400843704729
:10E588002DE9F041274C2568D5F8484184B0074665
:10E59800002C41D066681F2E1CDD234810B94FF0AF
:10E5A800FF301FE04FF4C870039102920193AFF35C
:10E5B80000800399029A019B04460028EFD0D5F801
:10E5C8004861002060602660C5F84841C4F88801A9
:10E5D800C4F88C01656847B9A81C013544F82010B7
:10E5E8006560002004B0BDE8F081D4F8886101209E
:10E5F80004EB850800FA05F00643022FC8F88820C6
:10E60800C4F88861C8F80831E6D1D4F88C3143EAF7
:10E618000002C4F88C21DFE705F5A674C5F8484167
:10E62800B8E700BF6C2C01080000000000210A2296
:10E6380001F094BD2DE9F84FDDF828B081468A46EF
:10E6480098469AB193B11646002503E00FD0651C91
:10E65800AE420BD97419640808FB04A7484639462A
:10E66800D8470028F2DA2646AE42F3D800273846C3
:10E67800BDE8F88F40F2D053C2F200031868704723
:10E6880070B5114B114C181B811018D004EB810484
:10E698004E1E354654F8042D06F00106904775B114
:10E6A80026B154F8043D9847013D08D054F8040DAC
:10E6B8008047013D54F8041D8847013DF6D1BDE867
:10E6C800704004F0D7BA00BF942C0108902C0108C0
:10E6D8000F2A2DE9F00340F2958041EA00039B07D9
:10E6E80040F092800C6804604D6845608E68A2F125
:10E6F80010038660CC681D460F2DC460C3F3001656
:10E7080001F1100400F1100322D966B126681E60D9
:10E7180066685E60A6689E60E668103DDE6010343C
:10E7280010330F2D14D926681E6066685E60A668CF
:10E738009E60E668DE6026691E6166695E61A6699C
:10E748009E61E669203DDE61203420330F2DEAD832
:10E75800A2F1100323F00F0402F00F031034032B6F
:10E7680000EB0408214451D9A3F104090B464FEAF0
:10E77800990901EB890C53F8046BC1EB0C0544466D
:10E788000CF1040C634544F8046BC5F3800512D002
:10E798002DB153F8045B634544F8045B0BD01E4667
:10E7A800254656F8047B45F8047B5F68331D67608F
:10E7B8002C1D6345F3D109F101039C00091902F0EE
:10E7C80003024444DAB123460D7803F8015BA2182A
:10E7D800E4431419934204F0010410D02CB111F849
:10E7E800014F03F8014B934209D04D781C4604F8B9
:10E7F800015B8D785D70631C02319342F5D1BDE8F1
:10E80800F00370470446DDE70446DCE744461A4651
:10E81800D8E700BFF0B48407034600F08E80541E8A
:10E82800002A00F08880E507CEB211D41A46671E88
:10E8380002F8016B1346154692070FD0002C7AD0C8
:10E8480003F8016B9A073C461D4607D0013CEDE7EB
:10E85800034603F8016B9A071D46F7D1032C52D9DA
:10E86800CEB246EA06270F2C47EA07432DD9A4F172
:10E87800100217460F2FC2F300162B606B60AB60B7
:10E88800EB6005F1100216D93EB1103F13605360DA
:10E898009360D36010320F2F0DD9203F02F110067C
:10E8A800136053609360D360136153619361D361C4
:10E8B80020320F2FF1D8A4F1100222F00F0204F039
:10E8C8000F041032032C15441DD9271F3E462A4633
:10E8D800032E42F8043BC7F380070DD927B1043E45
:10E8E800032E42F8043B07D91746083E47F8043B75
:10E8F80053603A1D032EF7D8231F23F00302131D7C
:10E9080004F00304ED18B4B12B46C9B203F8011B97
:10E918002C19ED436219A34202F001050BD01DB179
:10E9280003F8011BA34206D01A4602F8011B5970CE
:10E93800531CA342F8D1F0BC7047054614468DE736
:10E948002DE9F04F8BB014468046029202EB42024A
:10E95800A508500004F0030418F0030F0491994629
:10E9680005950894099040F0D3800899002940F053
:10E978005882029A151F18BF01250195049D062D7E
:10E9880040F2CC80DDF810C0029F64464FEA5C0676
:10E99800072C07FB068A40F0E081DDF824C008EB6D
:10E9A8000C06019B002B40F0F981D8F80010DAF82A
:10E9B8000030C8F80030CAF80010029DDDF808A041
:10E9C80008EB0500494600220790344607460690A2
:10E9D800CAF1000A91460D46A74240F211812B4622
:10E9E8004D469946002D00F0C283DDF818A0049A20
:10E9F8000298CAEB070BC8EB0A015945A8BF59464C
:10EA0800002900FB028A36DD019B022BC1EB0705BA
:10EA1800424640F0CF82287812F801CB2B4602F804
:10EA2800010C03F801CB6818E94309180132834245
:10EA380001F001011FD049B112F8011C6D7802F8EC
:10EA4800015C03F8011B0132834214D012F8015C07
:10EA580093F800C0194602F801CC01F8015B12F8DE
:10EA6800015B93F801C00B4602F801CC03F8015B87
:10EA780001328342EAD1DDF808C0C6EB0A03341B31
:10EA8800CCEB0302A24228BF2246002A2FDD0198C0
:10EA98000228C2EB0A0140F054820E7838783B46CF
:10EAA800BD1803F8016B0A46FE437619AB4202F81B
:10EAB800010B06F001061AD03EB14878197803F820
:10EAC800010BAB4202F8011B11D01E7817781846CB
:10EAD800114600F8017B01F8016B5E785778034610
:10EAE8000A4603F8017BAB4202F8016BEDD1029DA7
:10EAF8005D45C0F08D81DDF808C0A4457DD2C4EB2A
:10EB08000A0818F0030FB4FBFCF404943FF42DAF8B
:10EB1800049D0223062D01933FF634AFDDF808A0CB
:10EB280008EB0A000AFB058A504566D2029FDDF809
:10EB380008B0019ECDF810A03C1D7D4203940190C1
:10EB48004F46DDF80490C14509D84DE0D9F80000DA
:10EB58002168C9F8001020604445A14644D909EB52
:10EB6800050420464946B84700283DDD002EEDD073
:10EB7800012E00F0B3830BEB04001BF804E094F8BB
:10EB880000C00BF1FF310246234601F001090029BC
:10EB980002F801CB03F801EBDEDDB9F1000F09D073
:10EBA800407894F801E00139002902F801EB03F8F4
:10EBB800010BD1DD93F800A092F800909446184616
:10EBC8000CF801AB00F8019B023992F801E093F8C8
:10EBD80001A062460346002902F801AB03F801EBE5
:10EBE800E8DC4445A146BAD8DDF80490DDF810C049
:10EBF800D944E145CDF80490A3D30BB0BDE8F08F1C
:10EC080038464146A84700280BDC8EE0206831686A
:10EC18002160306056444FF001095444A7423FF642
:10EC2800DEAE20464146A8470028C0F2AC83F4D1A6
:10EC3800019B002BEAD0019A012A35D0DDF808E0C3
:10EC4800207896F800C00EF1FF312246334601F0D5
:10EC58000109002902F801CB03F8010BDADDB9F14B
:10EC6800000F09D0107893F800C00139002902F884
:10EC780001CB03F8010BCDDD93F800B092F800E06A
:10EC8800944618460CF801BB00F801EB023992F8DB
:10EC9800019093F801B062460346002902F801BBCF
:10ECA80003F8019BE8DCB5E722463346DDF814E0BB
:10ECB80053F8041B52F8040B0EF1FF3C42F8041CF5
:10ECC8000CF0010143F8040C04320433BCF1000FCA
:10ECD800A0DD71B152F8040C53F8041C0CF1FF3C90
:10ECE80042F8041C43F8040C04320433BCF1000F4E
:10ECF80090DDA34652F8049C53F8044C104619467C
:10ED080042F8044C43F8049C50F8043B51F8042B97
:10ED1800ACF1020C40F8042C021D41F8043C0B1D18
:10ED2800BCF1000FE6DC5C4674E712D1019B002BB6
:10ED38007AD106993B680868DDF818C0CCF800302D
:10ED48003860069ADDF808E002EB0E0106914FF0F4
:10ED58000109DDF808C067443EE604980299431E9D
:10ED6800282801FB038600F2AB803446454651460D
:10ED78002846C847002821465046C0F29580C84713
:10ED880000283FF70EAE28462146C847019B34EAC3
:10ED9800200A28BFAA46002B3FF407AE0199012993
:10EDA800424600F04881DDF808C012F8014B9AF895
:10EDB80000500CF1FF31574602F8015C01F00100E8
:10EDC8000132002907F8014B7FF7F7AD58B13D78BC
:10EDD80012F8013C02F8015C01390132002907F8F8
:10EDE800013B7FF7EAAD12F8014C3B78384602F850
:10EDF800013C00F8014B12F8014B7D7802390746B7
:10EE080002F8015C0132002907F8014BEBDCD4E57C
:10EE1800029D4046BBFBF5F12A464B46FFF790FDA5
:10EE280069E602240194A9E5019A012A00F03C81CF
:10EE3800DDF818B0DDF808E039789BF800005A468C
:10EE48003B460EF1FF3B02F8011B0BF00101BBF141
:10EE5800000F03F8010B7FF774AF59B111781878D8
:10EE68000BF1FF3BBBF1000F02F8010B03F8011B8C
:10EE78007FF767AF92F800C093F8009010461946E4
:10EE880000F8019B01F801CBABF1020B92F801E00D
:10EE980093F801C002460B46BBF1000F02F801CB04
:10EEA80003F801EBE6DC4CE7C8470028FFF679AD2C
:10EEB80028462146C84735EA200A28BFA24670E5F9
:10EEC800029AC40802FB04F408EB04054FEA440B59
:10EED80029464046CDF80CB0C84708EB0B07002878
:10EEE80039462846C0F23781C847002840F3438294
:10EEF800C4F1000B0AEB0B0751463846C847544487
:10EF0800002821465046C0F21A81C847002840F31D
:10EF18002A82039806EB0B04371A21463846C8475D
:10EF2800002831462046C0F2FE80C84700283FF737
:10EF38001EAF38463146C84736EA200428BF3C464B
:10EF480015E70B4657F8045B53F8040B9208511E5B
:10EF580047F8040C3A1D01F0010043F8045C04333F
:10EF680000297FF7C4AD68B152F8045C53F8040C6B
:10EF7800013942F8040C43F8045C043204330029D4
:10EF88007FF7B5AD53F8046C52F8047C42F8046C72
:10EF98001546184643F8047C50F8042B55F8046BC2
:10EFA800023945F8042C031D2A1D002940F8046C79
:10EFB800E8DC9CE52B4652F8040B53F8045B8908FF
:10EFC80001F1FF3C42F8045C0CF0010543F8040C25
:10EFD80004320433BCF1000F7FF74DAD7DB152F818
:10EFE800041C53F8040C0CF1FF3C42F8040C43F8E1
:10EFF800041C04320433BCF1000F7FF73CAD0394CA
:10F0080052F8045C53F8044C1046194642F8044C74
:10F0180043F8045C51F8042B50F8045BACF1020C83
:10F0280040F8042C0B1D021DBCF1000F41F8045CD4
:10F03800E6DC039C1FE55746059952F8043B57F850
:10F04800040B013942F8040C01F0010447F8043CB0
:10F0580004323B1D00297FF7B0AC6CB152F8045C58
:10F0680053F8047C013942F8047C43F8045C043208
:10F07800043300297FF7A1AC52F8047C53F8045CF0
:10F088001446184642F8045C43F8047C50F8042BF4
:10F0980054F8047B023944F8042C031D221D00296E
:10F0A80040F8047CE8DC88E4069ADDF8149052F80D
:10F0B80004EB3B4609F1FF3153F8040B42F8040C0A
:10F0C80001F0010043F804EC0432043300297FF70F
:10F0D80038AE68B152F804CC53F8040C013942F840
:10F0E800040C43F804CC0432043300297FF729AE1A
:10F0F800A34652F804EC53F8044C9146184642F8DB
:10F10800044C43F804EC59F8043B50F8042B02393A
:10F1180049F8042C40F8043C031D002909F10402B5
:10F12800E7DC5C460DE6C8470028FFF620AE384607
:10F138003146C84737EA200428BF344617E6C8478F
:10F148000028FFF6E6AE38462146C84737EA200AC7
:10F1580028BFA246DDE6C8470028FFF6C9AE4046EC
:10F168003946C84738EA200528BF3D46C0E6049915
:10F17800029C079D04FB018A5545BFF43EADDDF8AE
:10F188001CB0029C019ECDF804B06542DDF808B0C1
:10F19800CDF80CA0043404941F46DDF80490C8454B
:10F1A80009D34CE0D9F800002168C9F800102060A4
:10F1B8004445A14643D909EB050420464946B847CA
:10F1C80000283CDD002EEDD0012E43D00BEB0400CF
:10F1D8001BF804E094F800C00BF1FF310246234607
:10F1E80001F00109002902F801CB03F801EBDFDD8A
:10F1F800B9F1000F09D0407894F801E001390029ED
:10F2080002F801EB03F8010BD2DD93F800A092F8A5
:10F218000090944618460CF801AB00F8019B02399F
:10F2280092F801E093F801A062460346002902F82B
:10F2380001AB03F801EBE8DC4445A146BBD8DDF897
:10F2480004C00CEB0B09DDF80CC0CDF80490E145C7
:10F25800A3D3D2E4DDF81090DDF814C009EB040262
:10F26800234652F8040C53F8041B0CF1FF3E42F8F5
:10F27800041C0EF0010143F8040C04320433BEF1FF
:10F28800000F95DD71B152F8040C53F8041C0EF10F
:10F29800FF3E42F8041C43F8040C04320433BEF168
:10F2A800000F85DDA24652F8049C53F8044C104622
:10F2B800194642F8044C43F8049C50F8043B51F8B2
:10F2C800042BAEF1020E40F8042C021D41F8043C58
:10F2D8000B1DBEF1000FE6DC544669E7039ADDF822
:10F2E80014901219234652F8040C53F8041B09F120
:10F2F800FF3C42F8041C0CF0010143F8040C0432F2
:10F308000433BCF1000F7FF727AC79B152F8040C35
:10F3180053F8041C0CF1FF3C42F8041C43F8040C9D
:10F3280004320433BCF1000F7FF716ACA24652F842
:10F3380004EC53F8044C1046194642F8044C43F8C0
:10F3480004EC50F8043B51F8042BACF1020C40F8E3
:10F35800042C021D41F8043C0B1DBCF1000FE6DC37
:10F368005446FFF7F9BB38462146C84734EA200A15
:10F3780028BFBA46CDE540463946C84737EA200592
:10F3880028BF4546B4E5A7423FF629AB019B63B9C0
:10F398003868216839602060DDF808E04FF001091D
:10F3A8007744CEEB0404FFF717BB0198012833D04C
:10F3B800DDF80890207897F800E03A4609F1FF3127
:10F3C800234602F8010B01F00100002903F801EBC4
:10F3D800E2DD48B1107893F800C00139002902F83D
:10F3E80001CB03F8010BD7DD93F800B092F800E0E9
:10F3F800944618460CF801BB00F801EB023992F864
:10F40800019093F801B062460346002902F801BB57
:10F4180003F8019BE8DCBFE73A462346DDF814E031
:10F4280053F8041B52F8040B0EF1FF3C42F8041C7D
:10F438000CF0010143F8040C04320433BCF1000F52
:10F44800AADD71B152F8040C53F8041C0CF1FF3C0E
:10F4580042F8041C43F8040C04320433BCF1000FD6
:10F468009ADDA34652F8049C53F8044C10461946FA
:10F4780042F8044C43F8049C50F8043B51F8042B20
:10F48800ACF1020C40F8042C021D41F8043C0B1DA1
:10F49800BCF1000FE6DC5C467EE700BF830770B571
:10F4A800064614D10368A3F1013222EA030010F0E2
:10F4B800803F0CD1331D1A4653F8044BA4F1013593
:10F4C80025EA040414F0803FF5D0104600E03046E9
:10F4D80003782BB1421C104601320478002CFAD173
:10F4E80000F080F8304670BDC9B2F0B400294BD0A6
:10F4F80082070FD00278002A71D0914242D0431C73
:10F5080005E013F8012B002A3BD091423AD09A0724
:10F518001846F6D10368A3F1013222EA030241EA50
:10F52800012712F0803F47EA07471CD17B40A3F12F
:10F53800013222EA030313F0803F14D1021D02E0D6
:10F5480014F0803F0FD1104652F8043BA3F1013666
:10F5580087EA030426EA0303A4F1013513F0803F88
:10F5680025EA0404ECD00278002A38D0914209D068
:10F57800431C01E0914205D0184613F8012B002ADC
:10F58800F8D11046F0BC704783070BD00278002AE8
:10F59800F8D0431C03E0017801330029F2D0990721
:10F5A8001846F8D10168A1F1013323EA010212F0EB
:10F5B800803F0AD1031D184653F8041BA1F10134FA
:10F5C80024EA010212F0803FF5D00378002BD9D04D
:10F5D800411C084601310278002AFAD1D2E71046C8
:10F5E800D0E700BF80EA0102844612F0030F4FD132
:10F5F80011F0030F32D14DF8044D11F0040F51F8FA
:10F60800043B0BD0A3F101329A4312F0803F04BFB0
:10F618004CF8043B51F8043B16D100BF51F8044B99
:10F62800A3F101329A4312F0803FA4F101320BD1C9
:10F638004CF8043BA24312F0803F04BF51F8043B4E
:10F648004CF8044BEAD023460CF8013B13F0FF0FAB
:10F658004FEA3323F8D15DF8044B704711F0010FDE
:10F6680006D011F8012B0CF8012B002A08BF7047AF
:10F6780011F0020FBFD031F8022B12F0FF0F16BFA6
:10F688002CF8022B8CF8002012F47F4FB3D170476E
:10F6980011F8012B0CF8012B002AF9D1704700BF93
:10F6A80020F0030110F00300C0F1000051F8043B02
:10F6B80000F1040C4FEACC0C6FF000021CBF22FAD8
:10F6C8000CF213434FF0010C4CEA0C2C4CEA0C4C96
:10F6D800A3EB0C0222EA030212EACC1204BF51F88F
:10F6E800043B0430F4D013F0FF0F1FBF013013F4B4
:10F6F8007F4F013013F47F0F18BF0130704700BFF0
:10F70800F0B4002A65D00446344B14F8010B1B688A
:10F718001D18571E6E7806F00305012D07F0010726
:10F728005AD011F8015B5E19767806F00306012EAF
:10F7380008BF2035401B4DD1002D4BD0013A49D090
:10F7480037B314F8010B1D186E7806F00305012D68
:10F7580011F8015B03EB050608BF2030767806F048
:10F768000306012E08BF2035401B33D195B3013A5B
:10F778000ED12FE011F8012B9E18767806F00306BB
:10F78800012E08BF2032801A24D11AB36A1E21D054
:10F7980014F8010B1D186E7806F00305012D11F8F9
:10F7A800015B03EB050608BF2030767806F00306F8
:10F7B800012E08BF2035401B0CD15DB114F8010B98
:10F7C800551E1A18567806F00302012AD2D12030A5
:10F7D800D0E71046F0BC70472030A2E7A401002013
:10F7E80041EA00039B07F0B475D1032A73D90B468D
:10F7F800161F53F8045BA5F1013727EA050717F030
:10F80800803F0446C6F3800C31D10446032E3246AD
:10F8180044F8045B2AD9BCF1000F0AD0194653F802
:10F82800045BA5F1013626EA050616F0803F18D0DC
:10F838001DE01E46194656F8045BA5F1013727EA74
:10F84800050717F0803F12D144F8045B5D68A5F105
:10F858000133314623EA0506043A0B1D16F0803FB2
:10F8680005D1043A032A44F8045BE2D8194682B366
:10F878000D78013A04F8015B9DB112F0010F23469F
:10F888002BD11C462AB311F8015F013A04F8015B39
:10F898003DB111F8015F5D70631C013A1C46002DF3
:10F8A800EFD1B2B12346002103F8011BA518E443A8
:10F8B8002A19AB4202F001040BD01CB103F8011B5A
:10F8C800AB4206D01A4602F8011B5970531CAB42D2
:10F8D800F8D1F0BC70470446C9E7234611F8015F28
:10F8E80003F8015B013A1C46002DCAD1D9E700BFD5
:10F8F8002DE9F00701273C4600254FF0FF36631934
:10F908008B4200EB060C0DD21CF804A010F8038003
:10F91800D0452ED201241D469F1B63198B4200EB54
:10F92800060CF1D34FF0010A1760544600254FF03A
:10F93800FF3C6319994200EB0C080ED918F80480B3
:10F9480010F80390C1451AD901241D46CCEB030ACF
:10F958006319994200EB0C08F0D80CF1010001364C
:10F96800B0423CBFBA463046C2F800A0BDE8F00736
:10F9780070470BD001272E463C46ED19BFE709D04A
:10F988004FF0010AAC4654465544D2E7BC4205D074
:10F998000134B4E7544505D00134CAE727461D466B
:10F9A8000124ACE7A2461D460124C2E72DE9F04F29
:10F9B800ADF2244D164607460C461046194607AACE
:10F9C8001D46FFF795FF07AB01900DF21C411A1D6C
:10F9D8005D6008338B425560F9D11DB3327801233D
:10F9E80008A8691EAB4240F8221001EA030219D0A8
:10F9F8003AB17278022301F1FF3EAB4240F822E0AF
:10FA080010D0A146A8465C1C16F803C0325DCD1A7A
:10FA180002330C1B434540F82C5040F82240F2D1E9
:10FA28004C4645460799019A3046711800F054FC37
:10FA3800002840F0BE80DDF80490DDF804E002956F
:10FA480009F1FF3B06EB0B0CCDF80CB0CEF1010B26
:10FA58002246824605F1FF39CDF810C0CDF814B022
:10FA6800044608E024B1079CA34201D202990B1B6B
:10FA78009A4400242A46029D5544B8180021AA1A1F
:10FA880000F08AFB002840F08E80002D00F08B806B
:10FA9800791908A811F8013C50F82330002BE1D15E
:10FAA800019B9C4228BF23464B452AD207EB0A01FB
:10FAB80016F803B0CA5C934506EB03006FD16FEAF2
:10FAC800030C0CEB090E1EF0010F024616D0013391
:10FAD8004B4516D2407811F803B0013283450DD05A
:10FAE8005DE012F8010F11F803C0844557D10133C6
:10FAF80012F8010F11F803E0864550D101334B4548
:10FB0800EFD3DDF804B0039B5C4528BF5B463DD2CC
:10FB1800DDF80CB007EB0A0C16F80B101CF80B00FC
:10FB2800814240F0CA80DDF810B006EB0408C8EB4B
:10FB38000B01C8075A4624D5049ADDF80CE012F8E0
:10FB4800010CDDF810B000900EF1FF310BF1FF321F
:10FB58001CF80100DDF800B0834517D10B4610E012
:10FB680012F801BC1CF80020934501F1FF320DD1B9
:10FB78000346013811F801BC1CF800108B4505D16B
:10FB88000346581E424502F1FF31E9D101349C4237
:10FB980000F29580079C029AA244141B6AE7DDF8DC
:10FBA80014B0DA4464E7002009B00DF5806DBDE8B3
:10FBB800F08FDDF804B0019ADDF80480CBEB050086
:10FBC800584538BF5846431C01980793B118C0F1EF
:10FBD800010305F1FF3B029301954FF0000A02F182
:10FBE800FF3923460D46019C5444F8180021E21AB7
:10FBF80000F0D2FA0028D6D1002CD4D03A1908A99E
:10FC080012F8010C51F8200000284FD1D84507EB15
:10FC18000A002AD210F808302A789A4218BF4346B8
:10FC280047D16FEA080303EB0B01C9072A4643468D
:10FC380018D508F101035B4517D22A4610F803E0EE
:10FC480012F8011F8E450DD033E012F8011F10F88D
:10FC580003C08C452DD1013312F8011F10F803E0C1
:10FC68008E4526D101335B45EFD3B9F1FF3F4B46B3
:10FC78009AD016F8091010F80920914215D119F0F8
:10FC8800010F0AD009F1FF33F15CC25C914204D044
:10FC98000BE0F15CC25C914207D15A1E002B83D065
:10FCA800B15C825C023B9142F3D0079882442346C0
:10FCB80099E7029A92449A44F9E7019B66E707EBB1
:10FCC8000A0071E72DE9F04F037889B005460F4621
:10FCD800002B00F067810A789AB18446013101242B
:10FCE80002E011F8012B5AB1934214BF002404F02A
:10FCF80001041CF8013F0E46002BF2D1307820B9E0
:10FD08002CB1284609B0BDE8F08F0025F9E7681C3A
:10FD18003978FFF7E9FBF61B80460028F5D0012E5D
:10FD280000F0BE80AD19A84294BFC0EB05040124C1
:10FD38001F2E06D921463A463346FFF737FE0546B9
:10FD4800DFE7314607AA3846FFF7D2FD0799814613
:10FD5800791838464A4600F0BFFA002840F0A280D9
:10FD680009F1FF3B07EB0B0ECDF808B0C9F1010B09
:10FD7800CDF810900546CDF80CE0CDF814B0224629
:10FD88008146AC1908EB02000021A21A00F004FA1F
:10FD98000028BAD1002CB8D0049B994528BF4B46FF
:10FDA8009E422BD908EB0300F95C425D914207EBB8
:10FDB80003006ED16FEA030C0CEB060E1EF0010F68
:10FDC800024608EB050116D001339E4216D9407849
:10FDD80011F803C0013284450DD05AE012F8010F22
:10FDE80011F803E0864554D1013312F8010F11F8D8
:10FDF80003C084454DD101339E42EFD8049B029A3B
:10FE08004B4540F2D28008EB050EB95C1EF80200A3
:10FE1800814240F0CA80DDF80CB007EB090ACAEB52
:10FE28000B01C9075B4624D5039BDDF808B013F81E
:10FE3800010CDDF80CC001900BF1FF31DDF804B0C6
:10FE48001EF8010083450CF1FF3317D10A4610E074
:10FE580013F801BC1EF800309B4501F1FF330DD1AA
:10FE68000246013811F801BC1EF800108B4505D177
:10FE78000246501E534503F1FF31E9D109F101094A
:10FE8800914500F29480079AAD18C2EB0609224604
:10FE980077E7DDF814B05D44ED184FF00009F6E798
:10FEA80005462EE7C9EB06034B4538BF4B46581CA1
:10FEB800C9F1010B07EB090E08EB090209F1FF353F
:10FEC800CDF80CB0234607904FF0000A0292744612
:10FED800AB460AEB060508EB03000021EA1A00F01E
:10FEE8005BF900287FF411AF002D3FF40EAF4E45AB
:10FEF80098BF08EB0A002AD9029B217813F80A0058
:10FF080081424AD16FEA09029319DB0721464A4622
:10FF180008EB0A0018D509F10102964217D92146C3
:10FF280010F802C011F8013F9C450DD036E011F8D9
:10FF3800013F10F802E09E4530D1013211F8013F2F
:10FF480010F802C09C4529D101329642EFD8BBF186
:10FF5800FF3F5B463FF4F3AE17F80B1010F80B2089
:10FF6800914216D11BF0010F0AD00BF1FF33F95C57
:10FF7800C25C914204D00CE0F95CC25C914208D1A9
:10FF88005A1E002B3FF4DBAEB95C825C023B914207
:10FF9800F2D0079882442B469BE74A46039882444E
:10FFA8009244F8E70E460124A8E6049A66E7454419
:10FFB800A7E600BF40F2D052C2F200020123126845
:10FFC8005C3200F001B800BFF0B4002825D0074625
:10FFD80038460D460678013715F8014B3CB1A64264
:10FFE800FAD1002BF4D1176007F8013C11E0C6B133
:08FFF8003D4600E01BB915F8BD
:020000040801F1
:10000000016B0C46284614F8013B9E42F6D136B1EE
:10001000002105F8011C1060781EF0BC70473046C6
:10002000F9E710680028D6D1F7E716603046F4E704
:100030002DE9F00F4A4C82B0D4F800C00190084678
:10004000044614F8015B0CEB05062046777807F0B0
:100050000806F7B2002FF3D12D2D62D02B2D03BF50
:100060002446BB4614F8015BBB46002B41D1302D22
:1000700043D00A239A46BBF1000F0CBF6FF0004635
:100080004FF00046B6FBFAF900200AFB196700970B
:1000900080460CE0303DAB421BDD461C05D0C84518
:1000A00039D835D00AFB0858012014F8015B0CEB55
:1000B0000506767806F00407FFB2002FEAD116F0A5
:1000C000030606D0012E14BF57263726AD1BAB42C0
:1000D000E3DC431C2AD0BBF1000F01D0C8F10008BB
:1000E000002A31D0D0B94046116002B0BDE8F00F0F
:1000F0007047102BBED1302DBCD12578782D25D05E
:10010000582D23D043BB4FF0080A30255346B2E7A1
:1001100000988542C6DD4FF0FF30C6E74046611EBD
:10012000E2E714F8015B4FF0010B9EE7BBF1000F13
:1001300001990CBF6FF000404FF0004022230B608C
:10014000002AD2D0611ECFE74046CEE74FF0100A1A
:100150006578534602348EE79A4630258BE700BF18
:10016000A401002070B440F2D054C2F2000406464C
:100170000D462068134631462A4670BCFFF758BF2B
:10018000024B13B1024800F005B8704700000000B0
:1001900089E600080146002002460346FEF7F4B94E
:1001A0008307F0B4C9B200F09680531E002A00F015
:1001B000948002788A420BD0421CD8071AD512F0DC
:1001C000030F10461CD01478013B01328C4211D130
:1001D000F0BC7047002B7CD01278013B8A42F7D0EC
:1001E00014F0030F204604F1010209D02478013BEA
:1001F0008C42EDD012F0030F104602F10104E9D158
:10020000032B3FD9046841EA012545EA054585EA03
:100210000407A7F1013222EA07021E1F041D12F093
:10022000803FC6F380072DD1032E334629D967B10D
:1002300020460434066885EA0602A2F1013626EA61
:10024000020212F0803F19D01CE0261D20462468CF
:1002500085EA0402A2F1013424EA020212F0803F8E
:1002600010D1346885EA0402A2F1013424EA0202C2
:10027000043B341D12F0803F304603D1043B032B76
:10028000E3D820465D1E23B303788B42A0D0431CE5
:100290000022E80714D518460122047801338C4265
:1002A00096D09542184603F1010402F102020ED0E5
:1002B0001B788B428CD0631C204624788C4287D0DC
:1002C0009542184603F1010402F10202F0D1002028
:1002D0007EE718467CE7134692E7104678E700BFB2
:1002E000032AF0B431D941EA00039C072ED10668F5
:1002F0000F68151F031D0C1DBE42C5F3800C24D1D1
:10030000032D2A461FD9BCF1000F08D025681E68AE
:100310002146184604340433AE4211D015E0184685
:10032000214623680468051D0E1D9C420DD12846F8
:10033000314635680668043A031D0C1DAE4204D1EF
:10034000043A032AEBD8214618461AB303780C78EE
:10035000A3420AD1551E0022EB0714D510F8013F25
:1003600011F8014F0122A3420DD0181B10E010F824
:10037000013F11F8014FA342F7D110F8013F11F8E6
:10038000014FA342F1D1AA4202F10202EFD10020B3
:10039000F0BC70471046FBE71E1E6464646464642E
:1003A0000010004800110102001000480044010242
:1003B000001000480022110202031048494A4B4C29
:1003C0004D44454647FF1048498A8B8C8D8485866D
:1003D00087FF0000E4030108BA030108F3030108E2
:1003E000C6030108202122232425262748494A4BF9
:1003F0004C4DFF202122232425262748498A8B8C17
:100400008DFF000041210008011F00082F1F000878
:10041000F9200008171F0008E1200008AD2400089B
:100420005B2400087F240008292600081D240008FA
:1004300019240008002C01400000004800010000C1
:10044000001B010A004401400004004800010000B4
:100450000019000A004801400004004800020000A2
:10046000001A000A00340140000800484000000063
:10047000002E010A003401400008004880000000FE
:10048000042E010A00340140000800480001000069
:10049000082E010A00040040000400480200000089
:1004A0000C1D000A0004004000000048100000007D
:1004B000041D000A00080040000C00480010000065
:1004C000001E000200080040000C00480020000050
:1004D000041E000200080040000C0048004000001C
:1004E000081E000200080040000C004800800000C8
:1004F0000C1E000200000040000000480200000046
:10050000041C00020000004000000048040000003D
:10051000081C0002002C01400000004000040040C4
:100520000008004000340140004401400048014000
:100530000000040008000C00D00732003200320036
:100540003200320032003200C80064000000414531
:100550005452313233340030313233343536373857
:10056000394142434445464748494A4B4C4D4E4F1A
:10057000505152535455565758595A001545000872
:10058000594500083545000871450008994500089F
:10059000ED45000821450008654600080000803F41
:1005A000F704353FF70435BF0000803F0000803F6F
:1005B000F70435BFF70435BF0000803F0000803FDF
:1005C000F70435BFF704353F0000803F0000803F4F
:1005D000F704353FF704353F0000803F0000803FBF
:1005E00000000000000080BF000080BF0000803FCE
:1005F000000080BF00000000000080BF0000803FBE
:10060000000000000000803F000080BF0000803F2D
:100610000000803F00000000000080BF0000803F1D
:100620000000803F000000BF0000803F0000803FCE
:10063000000000BF000080BF0000803F0000803F3E
:10064000000080BF0000003F0000803F0000803FAE
:100650000000003F0000803F0000803F0000803F1E
:100660000000003F000080BF000080BF0000803F0E
:10067000000080BF000000BF000080BF0000803F7E
:10068000000000BF0000803F000080BF0000803FEE
:100690000000803F0000003F000080BF0000803F5E
:1006A000000000BFD0B35D3F0000803F0000803FEE
:1006B000000000BFD0B35DBF0000803F0000803F5E
:1006C0000000003FD0B35D3F000080BF0000803FCE
:1006D0000000003FD0B35DBF000080BF0000803F3E
:1006E000000080BF00000000000080BF0000803FCD
:1006F0000000803F000000000000803F0000803FBD
:10070000000000000000803F0000803F0000803FAC
:10071000000080BF000080BF000000000000803F9C
:10072000000000000000803F000080BF0000803F0C
:100730000000803F000080BF000000800000803F7C
:1007400000000000A8AAAA3F000000000000803FAF
:10075000000080BFB0AA2ABF000000000000803F58
:100760000000803FB0AA2ABF000000000000803FC8
:100770000000803F00000000000000000000803FFB
:10078000000080BF00000000000000000000803F6B
:100790000000000000000000000080BF0000803F5B
:1007A00000000000000000000000803F000000008A
:1007B00000000000030100003C07010804000000E5
:1007C000E4090108040000004409010802010000D6
:1007D0006C07010800010000000000000600000096
:1007E000640A0108060000008409010801010000F4
:1007F0000000000004000000240A010806000000B8
:100800009C06010808000000C40801080800000058
:100810009C050108080000001C06010801010000F9
:1008200000000000000100000000000000010000C6
:100830000000000004000000FC06010806000000A3
:10084000640801080001000000000000020100002F
:100850008C070108010100000000000000000000FA
:10086000000000000000803F000080BF0000803FCB
:10087000000080BF0000803F000080BF000080BFFC
:100880000000803F0000803F0000803F0000803F6C
:100890000000803F0000803F0000803F000080BFDC
:1008A000000080BF0000803F00000000000000004A
:1008B000000000000000803F000000000000000079
:1008C000000000000000803F000080BF0000803F6B
:1008D000000080BF0000803F000080BF000080BF9C
:1008E0000000803F0000803F0000803F0000803F0C
:1008F0000000803F0000803F0000803F000080BF7C
:10090000000080BF0000803F000080BF0000803FEB
:100910000000803F0000803F000080BF000080BFDB
:10092000000080BF0000803F0000803F0000803F4B
:10093000000080BF0000803F0000803F000080BFBB
:100940000000803F0000803F000080BF0000803F2B
:10095000000080BF0000803F000080BF000080BF1B
:100960000000803F0000803F0000803F0000803F8B
:100970000000803F0000803F0000803F000080BFFB
:10098000000080BF0000803FD0B35DBF0000003F8B
:100990000000803F0000803FD0B35DBF000000BF7B
:1009A000000080BF0000803FD0B35D3F0000003FEB
:1009B0000000803F0000803FD0B35D3F000000BFDB
:1009C000000080BF0000803F00000000000080BFEA
:1009D0000000803F0000803F000000000000803FDA
:1009E000000080BF0000803F000000000000803F4A
:1009F000000080BF0000803F000080BF00000000BA
:100A00000000803F0000803F0000803F00000000A9
:100A10000000803F0000803F00000000000080BF19
:100A2000000080BF0000803F000000000000803F09
:100A3000000080BF0000803F000080BF000080BF3A
:100A4000000000000000803F000000000000803F28
:100A50000000803F0000803F0000803F000080BF1A
:100A6000000000000000803F00000000A8AAAA3F8C
:100A70000000803F0000803F000080BFB0AA2ABF76
:100A8000000080BF0000803F0000803FB0AA2ABF66
:100A9000000080BF0000803F00000000A8AAAA3F1D
:100AA000000080BF0000803F000080BFB0AA2ABFC6
:100AB0000000803F0000803F0000803FB0AA2ABFB6
:100AC0000000803F24505542582C34312C312C30BA
:100AD0003030332C303030312C3131353230302C15
:100AE000302A31450D0A0024504D544B3235312CFB
:100AF0003131353230302A31460D0A00245055420A
:100B0000582C34312C312C303030332C30303031C3
:100B10002C35373630302C302A32440D0A00245020
:100B20004D544B3235312C35373630302A32430D67
:100B30000A0024505542582C34312C312C3030309E
:100B4000332C303030312C33383430302C302A32A2
:100B5000360D0A0024504D544B3235312C33383485
:100B600030302A32370D0A0024505542582C343187
:100B70002C312C303030332C303030312C31393274
:100B800030302C302A32330D0A0024504D544B3271
:100B900035312C31393230302A32320D0A00B5620B
:100BA00006010300F00500FF19B56206010300F01D
:100BB0000300FD15B56206010300F00100FB11B54D
:100BC0006206010300F00000FA0FB562060103009F
:100BD000F00200FC13B56206010300F00400FE17EA
:100BE000B562060103000102010E47B5620601036A
:100BF000000103010F49B56206010300010601125D
:100C00004FB562060103000112011E67B5620616A8
:100C10000800030703000000000031E5B562060884
:100C20000600C80001000100DE6A000000000000AC
:100C300000C20100C40A0108E70A0108010000001F
:100C400000E10000FC0A01081E0B01080200000080
:100C500000960000320B0108540B0108030000004D
:100C6000004B0000680B01088A0B0108040000001B
:100C70008025000023140108231401084145525423
:100C80003132333400002710080423022001000011
:100C9000000000008025000000C2010002000000EA
:100CA000010000008025000000C2010003000000D8
:100CB0000200000080250000004B0000050000003D
:100CC0000300000080250000004B0000050000002C
:100CD000020000008025000000C2010000000000AA
:100CE000100000008025000000C20100010000008B
:100CF000200000008025000000C20100000000006C
:100D0000010000008025000000C20100000000007A
:100D1000080000008025000000C201000003000060
:100D20000400000080250000004B000000000000CF
:100D3000CA1C0108D11C0108D61C0108E71C0108C7
:100D4000F11C0108FC1C0108071D0108121D010807
:100D5000DC1B01081B1D0108D61B0108241D01080E
:100D60002E1D0108391D01083F1D0108421D010803
:100D7000521D0108000000001C1C0108201C010875
:100D8000261C01082C1C01082F1C0108361C010818
:100D9000391C01083E1C01084A1C01084D1C0108B1
:100DA000531C01085A1C0108641C01086E1C010830
:100DB000771C0108851C0108911C0108981C01087A
:100DC0009E1C0108AB1C0108B61C0108C31C0108CD
:100DD00000000000261A01082A1A01080DA30008C5
:100DE000511A0108561A0108D99D00086A1A01080B
:100DF000731A0108C19D0008901A0108951A01088C
:100E000071A30008C41A010823140108899D000871
:100E1000C91A0108D11A01089D9C0008E51A0108A9
:100E2000F41A01087D9C00080E1B01082314010818
:100E3000CD990008131B0108171B0108D59B00085A
:100E4000641A0108331B010825A00008461B01088D
:100E50004C1B010865A20008671B01086F1B0108F5
:100E600019A200087E1B0108831B0108AD9B000826
:100E700003110108931B0108C5A00008C11B01084C
:100E8000B51B0108F999000813160108231401087D
:100E9000C199000823140108E81B0108F01B010890
:100EA000F81B0108001C0108071C0108121C01089E
:100EB000171C0108000000004166726F33322043A6
:100EC0004C492076657273696F6E20322E32204D48
:100ED00061792032312032303134202F2031343AC0
:100EE00034363A3231202D2028636C65616E666C91
:100EF000696768742900417661696C61626C65207C
:100F0000636F6D6D616E64733A0D0A002573092578
:100F1000730D0A0053797374656D20557074696D93
:100F2000653A202564207365636F6E64732C2056C8
:100F30006F6C746167653A202564202A20302E3159
:100F40005620282564532062617474657279290DD6
:100F50000A004350552025644D487A2C206465745E
:100F600065637465642073656E736F72733A2000F5
:100F70002573200041434348573A202573002E250E
:100F800063004379636C652054696D653A2025647C
:100F90002C20493243204572726F72733A202564C7
:100FA0002C20636F6E6669672073697A653A202525
:100FB000640D0A00202564202564000D0A52656234
:100FC0006F6F74696E672E2E2E00536176696E679F
:100FD0002E2E2E004D75737420626520616E79206F
:100FE0006F72646572206F6620414554523132330E
:100FF000340D0A0043757272656E742061737369F3
:10100000676E6D656E743A20004572726F723A2099
:10101000456E61626C6520616E6420706C7567203E
:10102000696E204750532066697273740D0A00453B
:101030006E61626C65642066656174757265733A91
:101040002000417661696C61626C6520666561743F
:10105000757265733A2000496E76616C696420662A
:10106000656174757265206E616D652E2E2E0D0A98
:101070000044697361626C65642000456E61626C56
:10108000656420000D0A4C656176696E6720434CEB
:1010900049206D6F64652E2E2E0D0A005265736512
:1010A0007474696E6720746F2064656661756C7412
:1010B000732E2E2E004E4709004F4B0900437573C7
:1010C000746F6D206D697865723A200D0A4D6F74EA
:1010D0006F720954687209526F6C6C0950697463BD
:1010E00068095961770D0A002325643A09002573C0
:1010F000090053616E69747920636865636B3A090E
:10110000007265736574006C6F616400496E76618E
:101110006C6964206D6978657220747970652E2E13
:101120002E0D0A004C6F61646564202573206D6983
:10113000782E2E2E0D0A0057726F6E67206E756D19
:10114000626572206F6620617267756D656E74737B
:101150002C206E6565647320696478207468722041
:10116000726F6C6C207069746368207961770D0A06
:10117000004D6F746F72206E756D626572206D75B3
:101180007374206265206265747765656E20312016
:10119000616E642025640D0A0043757272656E7479
:1011A000206D697865723A2025730D0A00417661D9
:1011B000696C61626C65206D69786572733A2000B4
:1011C0004D697865722073657420746F2025730DE6
:1011D0000A0043757272656E742073657474696E6B
:1011E00067733A200D0A0025732073657420746FAD
:1011F00020004552523A2056616C75652061737328
:1012000069676E6D656E74206F7574206F662072ED
:10121000616E67650D0A004552523A20556E6B6E3D
:101220006F776E207661726961626C65206E616DA8
:10123000650D0A0043757272656E742070726F6678
:10124000696C653A2025640D0A0055736167653A3B
:101250000D0A6D6F746F7220696E646578205B761D
:10126000616C75655D202D2073686F77205B6F72F0
:10127000207365745D206D6F746F722076616C757C
:10128000650D0A004E6F2073756368206D6F746F73
:10129000722C207573652061206E756D62657220F9
:1012A0005B302C2025645D0D0A004D6F746F722039
:1012B0002564206973207365742061742025640D92
:1012C0000A00496E76616C6964206D6F746F7220DC
:1012D00076616C75652C20313030302E2E323030F6
:1012E000300D0A0053657474696E67206D6F746FFA
:1012F0007220256420746F2025640D0A00617578C2
:101300002025752025750D0A00496E76616C69648B
:10131000204665617475726520696E6465783A204F
:101320006D757374206265203C2025750D0A00439D
:10133000757272656E7420436F6E6669673A2043FA
:101340006F70792065766572797468696E6720625E
:10135000656C6F7720686572652E2E2E0D0A006D04
:10136000697865722025730D0A00636D6978202500
:101370006400636D6978202564203020302030209F
:10138000300D0A0066656174757265202D25730D38
:101390000A00666561747572652025730D0A006D1B
:1013A00061702025730D0A00736574202573203D3C
:1013B00020000D0A456E746572696E6720434C49C2
:1013C000204D6F64652C20747970652027657869DD
:1013D000742720746F2072657475726E2C206F7282
:1013E000202768656C70270D0A000D0A2320000D68
:1013F0001B5B4B001B5B324A1B5B313B314800459A
:1014000052523A20556E6B6E6F776E20636F6D6D22
:10141000616E642C20747279202768656C702700D7
:10142000082008006C6F6F7074696D6500656D66EB
:101430005F61766F6964616E6365006D6964726394
:10144000006D696E636865636B006D6178636865E4
:10145000636B00727373695F6368616E6E656C00C5
:101460006D696E7468726F74746C65006D61787408
:1014700068726F74746C65006D696E636F6D6D6119
:101480006E64006465616462616E6433645F6C6F96
:1014900077006465616462616E6433645F68696784
:1014A00068006E65757472616C33640064656164B4
:1014B00062616E6433645F7468726F74746C65002B
:1014C0006D6F746F725F70776D5F726174650073BA
:1014D0006572766F5F70776D5F72617465007265BB
:1014E0007461726465645F61726D00666C617073D3
:1014F0005F737065656400666978656477696E67B7
:101500005F616C74686F6C645F64697200736572AC
:1015100069616C5F706F72745F315F7363656E6178
:1015200072696F0073657269616C5F706F72745F6E
:10153000325F7363656E6172696F007365726961B2
:101540006C5F706F72745F335F7363656E61726935
:101550006F0073657269616C5F706F72745F345F86
:101560007363656E6172696F007265626F6F745F3D
:10157000636861726163746572006D73705F62614C
:1015800075647261746500636C695F626175647231
:10159000617465006770735F706173737468726FF4
:1015A0007567685F62617564726174650067707306
:1015B0005F70726F7669646572006770735F696EE1
:1015C000697469616C5F62617564726174655F6999
:1015D0006E6465780073657269616C72785F7072B1
:1015E0006F76696465720074656C656D6574727997
:1015F0005F70726F76696465720074656C656D65A5
:101600007472795F737769746368006672736B795B
:101610005F696E76657273696F6E0076626174736E
:1016200063616C6500766261746D617863656C6C92
:10163000766F6C7461676500766261746D696E6364
:10164000656C6C766F6C7461676500706F7765723E
:101650005F6164635F6368616E6E656C00616C6995
:10166000676E5F6779726F00616C69676E5F616357
:101670006300616C69676E5F6D616700616C6967CB
:101680006E5F626F6172645F726F6C6C00616C6937
:10169000676E5F626F6172645F7069746368006136
:1016A0006C69676E5F626F6172645F796177006D0C
:1016B00061785F616E676C655F696E636C696E61AE
:1016C00074696F6E006779726F5F6C7066006D6F22
:1016D000726F6E5F7468726573686F6C64006779AF
:1016E000726F5F636D70665F666163746F720067CF
:1016F00079726F5F636D70666D5F666163746F7240
:1017000000616C745F686F6C645F7468726F74748E
:101710006C655F6E65757472616C00616C745F6896
:101720006F6C645F666173745F6368616E676500A8
:101730007468726F74746C655F636F7272656374E2
:10174000696F6E5F76616C7565007468726F747432
:101750006C655F636F7272656374696F6E5F616EF3
:10176000676C65007961776465616462616E6400CD
:101770007961775F636F6E74726F6C5F64697265B5
:101780006374696F6E007961775F64697265637411
:10179000696F6E007472695F756E61726D65645F0A
:1017A000736572766F0072635F7261746500726355
:1017B0005F6578706F007468725F6D69640074684B
:1017C000725F6578706F00726F6C6C5F70697463C4
:1017D000685F72617465007961775F72617465003A
:1017E0007470615F72617465007470615F627265CC
:1017F000616B706F696E74006661696C73616665B8
:101800005F64656C6179006661696C736166655FD0
:101810006F66665F64656C6179006661696C7361AF
:1018200066655F7468726F74746C65006661696C7C
:10183000736166655F6D696E5F7573656300666190
:10184000696C736166655F6D61785F757365630070
:1018500067696D62616C5F666C6167730061636389
:101860005F6861726477617265006163635F6C7069
:10187000665F666163746F720061636378795F6449
:1018800065616462616E64006163637A5F6465616F
:101890006462616E64006163635F756E61726D6541
:1018A0006463616C006163635F7472696D5F70692A
:1018B000746368006163635F7472696D5F726F6CFB
:1018C0006C006261726F5F7461625F73697A650058
:1018D0006261726F5F6E6F6973655F6C70660062E4
:1018E00061726F5F63665F76656C006261726F5FE5
:1018F00063665F616C74006D61675F6465636C69EA
:101900006E6174696F6E006770735F706F735F7084
:10191000006770735F706F735F69006770735F70EB
:101920006F735F64006770735F706F73725F7000D6
:101930006770735F706F73725F69006770735F7059
:101940006F73725F64006770735F6E61765F7000C3
:101950006770735F6E61765F69006770735F6E6159
:10196000765F64006770735F77705F72616469753A
:1019700073006E61765F636F6E74726F6C735F6815
:10198000656164696E67006E61765F73706565643A
:101990005F6D696E006E61765F73706565645F6D23
:1019A0006178006E61765F736C65775F72617465F4
:1019B000007069645F636F6E74726F6C6C65720047
:1019C000705F706974636800695F70697463680050
:1019D000705F726F6C6C00695F726F6C6C00705F2F
:1019E00079617700695F79617700705F616C74007D
:1019F000695F616C7400645F616C7400705F6C653A
:101A000076656C00695F6C6576656C00645F6C651B
:101A100076656C00705F76656C00695F76656C005A
:101A2000645F76656C0061757800666561747572D7
:101A3000655F6E616D6520617578666C6167206FAA
:101A40007220626C616E6B20666F72206C697374B9
:101A500000636D69780064657369676E20637573F0
:101A6000746F6D206D697865720064656661756C70
:101A7000747300726573657420746F2064656661A9
:101A8000756C747320616E64207265626F6F740090
:101A900064756D70007072696E7420636F6E666934
:101AA00067757261626C652073657474696E6773C3
:101AB00020696E2061207061737461626C652066BC
:101AC0006F726D0065786974006665617475726522
:101AD000006C697374206F72202D76616C206F72B8
:101AE0002076616C00677073706173737468726FD5
:101AF00075676800706173737468726F75676820CA
:101B000067707320746F2073657269616C0068651B
:101B10006C70006D6170006D617070696E67206F30
:101B200066207263206368616E6E656C206F7264FC
:101B30006572006D69786572206E616D65206F72E7
:101B4000206C697374006D6F746F72006765742F19
:101B5000736574206D6F746F72206F757470757417
:101B60002076616C75650070726F66696C650069DE
:101B70006E64657820283020746F203229007361EC
:101B80007665007361766520616E64207265626FB0
:101B90006F74006E616D653D76616C7565206F7266
:101BA00020626C616E6B206F72202A20666F72203B
:101BB0006C6973740073686F772073797374656DE3
:101BC00020737461747573004759524F0041434349
:101BD000004241524F00534F4E4152004750530074
:101BE0004750532B4D4147004144584C3334350046
:101BF0004D505536303530004D4D41383435780034
